S00A000047572E737265637C
S214400000A55AA55A0100000000000000001040005C
S21440100000F0422021144400BD654500BF65450000
S214401010C1654500C3654500C56545000000000044
S214401020000000000000000000000000C76545000A
S214401030FB65450000000000FD654500FF65450076
S21444010047573334342056302E322E352032303250
S214440110332E31312E362031323A30300A0D00003B
S20C4401803412AA5500000000E9
S214440200A55AA55A01000000000000000010440052
S2144402100000000000104400000000000000000041
S2144402200000000000000000000000000000000085
S2144402300000000000000000000000000000000075
S2144402400000000000000000000000000000000065
S2144402500000000000000000000000000000000055
S21444100000F0422021144400BD654500BF654500FC
S214441010C1654500C3654500C56545000000000040
S214441020000000000000000000000000C765450006
S214441030FB65450000000000FD654500FF65450072
S21444104001664500016645000166450001664500A7
S2144410500166450001664500016645000166450097
S2144410600166450001664500016645000166450087
S2144410700166450001664500016645000166450077
S214441400016645000166450000BF00BF00BF00BF3F
S214441410FFF7FABF000000000000000000000000D4
S21444142072B64FF000004FF000014FF000024FF04C
S21444143000034FF000044FF000054FF000064FF055
S21444144000074F4801684FF0807201EA0201002904
S2144414501CD14C4801684FF0807241EA0201016099
S214441460494801684FF0010241EA020101604748D9
S21444147045F6F02101604AF20F5101604048016888
S2144414804FF0807201EA02010029F7D040484149F2
S2144414900160414801684FF00000814200D003E0FB
S2144414A03E4880F3088803E03D4880F3088822E0FD
S2144414B03C484CF2205101604DF6281101603A48F0
S2144414C03A4901600AE03A484CF2205101604DF630
S2144414D028110160374835490160FFE7364800283F
S2144414E009D03649364A521A013A04DD0020002310
S2144414F009C1083AFCDA3348002810D03249086853
S2144415004FF0010240EA020008603049304A521A5D
S214441510013A04DD0020002309C1083AFCDA2D48CC
S214441520002810D02C4908684FF0010240EA020017
S21444153008602A492A4A521A013A04DD0020002348
S21444154009C1083AFCDA274800684FF05A31884205
S214441550F9D0114801684FF00000814200D001E004
S21444156015F050F815F07AF862B615F075F800F0F4
S2144415703BF800BFFEE700BFAFF30080AFF3008048
S21444158010C32D4030C32D4004C32D4000C02D4011
S21444159008ED00E0001043200400264000F04220FE
S2144415A0000043201000274000002740400000FF72
S2144415B010C0464000C046400100000000004020E5
S2144415C0004044200100000094EF00E000000020AA
S2144415D0000001200100000090EF00E00000000041
S2144415E000800000F02440202DE9F04F87B05B4C8B
S2144415F001F066FC5A4816F053FD5A494E20002521
S21444160026F0FEFE58481DF0DBFE58481DF0FCFE52
S21444161001F0C9FB4CF24453E05800F021F901F0C4
S21444162005FE00F045FA00F021FA00F09FF9504913
S214441630002021F041F84F49002021F053F80021C2
S214441640084621F0F9F8002144F62062084621F0C5
S214441650AFF82846013501F063FF062DF9D101F0B5
S2144416609FFB4CF23853444D4FF47A7054F8038041
S214441670E75805F1040BE25854F803900592E258F3
S2144416800292E2580392E2580492E25854F803A0B5
S214441690E6582C46019201F04AFB08F0F9F937481F
S2144416A001F076FC00F0B4F82A6806F57A739A429C
S2144416B002D32E6808F0DBF922680AF1C8039A427E
S2144416C003D3D4F800A008F0CBF9019B2268643316
S2144416D09A4203D32368019308F0AFF9049B226827
S2144416E032339A4201D323680493039B226814330B
S2144416F09A4203D32368039303F0C2FB029B2268F7
S2144417000A339A4203D32368029308F05AF92268AC
S21444171009F105039A4203D3D4F8009008F0CFF8B1
S214441720059B226802339A4203D32368059300F04C
S21444173070F822687B1C9A4200D32768DBF80020A6
S21444174008F101039A4203D3DBF8008008F064F9F9
S21444175008F0A4F90DF054FFA6E700BF7C484120EA
S214441760289F4600E80340206CAC46009CA74600F1
S2144417707417402068174020B40D42208C954600CC
S214441780024B586800F00300704700BF0000264034
S214441790024600F03F00931010B583EA5203540803
S2144417A0534084EA121483EA121384EAD2049B0157
S2144417B084EA521403F0400314F0010F43EA000392
S2144417C00CBF80240024234319B99A4218BFFF2033
S2144417D010BD01290CBF1846FF20F9E73C2A0CD05F
S2144417E07D2A0AD0FE2A08D0BF2A06D092B20144E7
S2144417F0814204D1D043C0B270470022F7E710F8C4
S214441800013B1A4492B2FF2A84BFFF3A92B2EFE7F2
S21444181070470BF08BBF704710B50C4C002001F09E
S214441820E9F92080012001F0E5F9094B2288188067
S214441830084B1A800BF0D9FB0BF0FAFB0BF01CFCA0
S2144418400BF03EFCBDE810400BF05EBC5A1840203E
S2144418505818402004184020704770477047704717
S214441860002110B50446084619F0D4FD0121002095
S21444187019F0D0FD0221002019F0CCFD03210020F0
S21444188019F0C8FD002019F0C1FC0E49002019F0DB
S214441890D3FB0D4BA2B20020197819F00BFD0B496F
S2144418A000201AF07DF80A4900201AF079F8094910
S2144418B000201AF075F808490020BDE810401AF0D8
S2144418C06FB800BFE4A346001CA446006CA54600BF
S2144418D04CA546002CA546000CA54600F8B50D467A
S2144418E006461F4928461F4F0FF0DEF8044670B1DF
S2144418F04CF24453F85806F54553123307EB830726
S2144419007D60032E2BD8DFE806F01A212427002119
S21444191028460FF0BFF880B94CF24453F8580EF0FE
S214441920B9FE29460EF00EFF0EF05EFA00220E4B6C
S2144419300EF0DCFB0EF088FDDDE72046DBE782B2E6
S21444194000210020BDE8F8401AF074BA82B20121A2
S214441950F7E782B20221F4E782B20321F1E7F8BD49
S2144419600000C8427C4841200000594008B503485E
S2144419701EF018FF024B187008BD00BF64AF460047
S214441980BC474020F7B50123104C114D6370A21C90
S214441990EB68A91C0F480235009335F8023C1EF04C
S2144419A0A3FD00222073A01C6178134615F8017B22
S2144419B0013310F8016BDBB2B7421CBF0122002191
S2144419C00A2BF3D102B1617003B0F0BDBC4740208E
S2144419D0B81F402078AF46004B7C062B0AD1012224
S2144419E0054B1A74CA7B1A2A04D1032203F1110147
S2144419F01FF0BAB8704700BFB81F40204B7C062B78
S214441A000AD10122054B1A74CA7B2A2A04D103221E
S214441A1003F111011FF0A8B8704700BFB81F40205B
S214441A201FB500231A210446039301238DF807307B
S214441A301FF0E0F90B4B03930B4B1A7C002AFCD0A7
S214441A401B7C63B102A920461FF0D8F88DF8070026
S214441A50039B5A1E039213B19DF80730F1E704B076
S214441A6010BD00BF006A1800B81F402008B5A1206A
S214441A701DF0ECFC00220A49A1201DF0E6FC094BAF
S214441A80094902220120C3F8F413C3F8982DC3F879
S214441A90F813C3F8902D0549BDE808401EF0D6B9A2
S214441AA0430246000000294004002800D8AE460001
S214441AB008B5A2201DF0CAFC00220B49A2201DF046
S214441AC0C4FC0A4B0A4A01210020C3F8E023C3F8A9
S214441AD0AC1DC3F8E42302220649C3F8A42DBDE88E
S214441AE008401DF0F3BE00BF4902460000002940EE
S214441AF002002800FCAE460010B508221749012013
S214441B004FF480341EF05EFA012308221449002064
S214441B101DF0C8FF002108461EF012F9022801D124
S214441B20013CF7D14FF48034002101201EF054FAD2
S214441B30022801D1013CF7D1094A0823A2F1080042
S214441B4012F8011B013B10F8014BA14204BF0131BE
S214441B5002F8011C13F0FF03F2D110BDCC1F402045
S214441B60D41F402082B00190019B5A1E0192002B44
S214441B70FAD102B07047044B4FF400224FF4FA7087
S214441B80C3F8C022FFF7EEBF00002940044B4FF4D1
S214441B9020124FF4FA70C3F8C022FFF7E3BF00BF29
S214441BA0000029402DE9F04104460D461046002920
S214441BB03ED1DFF8908050260B46C1B2564308F11A
S214441BC010072846BA19B0441BF044F91C484FF491
S214441BD0FB534FF4FB62D8F81410083603FB040397
S214441BE03744D3F8FC3802FB043203F17A0602F594
S214441BF0107C02F5427240F82C1098F8581040F8C1
S214441C002210FB2212FB046200EB4212A94211D8B6
S214441C104FF4FB520133642102FB0404B3FBF1F29C
S214441C2001FB1233C4F8FC3804F521540123236025
S214441C30BDE8F08117F8016B013502F8016BE5E762
S214441C407C484120BC4740202DE9F04104460D46DF
S214441C50104600293ED1DFF8908050260B46C1B28C
S214441C60564308F521670120BA19B0441BF0F2F830
S214441C701C484FF4FB534FF4FB62D8F8141A08364A
S214441C8003FB04033744D3F8FC3802FB043203F165
S214441C907A0602F5107C02F5427240F82C1098F849
S214441CA0581A40F82210FB2212FB046200EB421240
S214441CB0A94211D84FF4FB520133642102FB0404B9
S214441CC0B3FBF1F201FB1233C4F8FC3804F521549B
S214441CD001232360BDE8F08117F8016B013502F853
S214441CE0016BE5E77C484120BC4740202DE9F041A4
S214441CF004460D46104600293ED1DFF89080502613
S214441D000B46C1B2564308F546770220BA19B0448A
S214441D101BF0A0F81C484FF4FB534FF4FB62D8F872
S214441D201C13083603FB04033744D3F8FC3802FB81
S214441D30043203F17A0602F5107C02F5427240F84A
S214441D402C1098F8601340F82210FB2212FB046211
S214441D5000EB4212A94211D84FF4FB5201336421DE
S214441D6002FB0404B3FBF1F201FB1233C4F8FC3863
S214441D7004F5215401232360BDE8F08117F8016B74
S214441D80013502F8016BE5E77C484120B458402011
S214441D902DE9F04104460D46104600293ED1DFF8B1
S214441DA0908050260B46C1B2564308F61857032077
S214441DB0BA19B0441BF04EF81C484FF4FB534FF48A
S214441DC0FB62D8F81C1D083603FB04033744D3F8DB
S214441DD0FC3802FB043203F17A0602F5107C02F565
S214441DE0427240F82C1098F8601D40F82210FB22EE
S214441DF012FB046200EB4212A94211D84FF4FB5284
S214441E000133642102FB0404B3FBF1F201FB1233F9
S214441E10C4F8FC3804F5215401232360BDE8F0815E
S214441E2017F8016B013502F8016BE5E77C48412061
S214441E30B45840202DE9F04104460D46104600298A
S214441E403ED1DFF8908050260B46C1B2564308F583
S214441E50C4670420BA19B0441AF0FCFF1C484FF477
S214441E60FB534FF4FB62D8F82416083603FB0403EE
S214441E703744D3F8FC3802FB043203F17A0602F501
S214441E80107C02F5427240F82C1098F8681640F818
S214441E902210FB2212FB046200EB4212A94211D824
S214441EA04FF4FB520133642102FB0404B3FBF1F20A
S214441EB001FB1233C4F8FC3804F521540123236093
S214441EC0BDE8F08117F8016B013502F8016BE5E7D0
S214441ED07C484120AC6940202DE9F04104460D463B
S214441EE0104600293ED1DFF8908050260B46C1B2FA
S214441EF05643A8F1D8070520BA19B0441AF0AAFFE9
S214441F001C484FF4FB534FF4FB6258F8D41C083675
S214441F1003FB04033744D3F8FC3802FB043203F1D2
S214441F207A0602F5107C02F5427240F82C1018F836
S214441F30901C40F82210FB2212FB046200EB421273
S214441F40A94211D84FF4FB520133642102FB040426
S214441F50B3FBF1F201FB1233C4F8FC3804F5215408
S214441F6001232360BDE8F08117F8016B013502F8C0
S214441F70016BE5E77C484120A47A40204FF4FB52AD
S214441F80054B02FB0033D3F8F808D3F8FC38C31AE1
S214441F9058425841704700BF7C4841202DE9F74FCE
S214441FA0D14D0021D14E4FF4FB692C4641F698782A
S214441FB037464FF0640A0846FFF7E0FF58BBD6F8AA
S214441FC0F83809FB013202F5427257F822C008FB82
S214441FD0014200924FF4FB524A4302EB43123A4406
S214441FE0019200F1010EC0B2844500F2AC8009FBB8
S214441FF00132013385F820C002F5107257F82220CA
S2144420006A624FF0010285F82120B3FBFAF20AFB1C
S2144420101233C6F8F8380131454406F5FB5606290E
S214442020C9D194F82130012B1DD1002340F221223E
S21444203084F82130636A934200F0E68000F29F8081
S21444204040F25512934200F0DC80B3F5AB7F80F04B
S2144420508980422B00F0DE807FD8402B00F0C5807C
S214442060412B00F0C58041F6B973E25C012A0FD1DA
S2144420700022E25441F6BC73E358932B00F0DB8015
S21444208000F2CB80912B00F0D080922B00F0D080D1
S21444209043F65173E25C012A14D10022E25443F61B
S2144420A05473E358962B00F0EE8000F2CF80822BD8
S2144420B000F0E68000F2C280722B00F0EA80732BB8
S2144420C000F0EA8045F6E963E25C012A14D1002276
S2144420D0E25445F6EC63E3589B2B00F0FE8000F296
S2144420E0E9808D2B00F00D8100F2DC80722B00F02D
S2144420F00281732B00F0028147F68163E25C012A79
S2144421000BD10022E25447F68463E358722B00F066
S214442110FE80732B01D102F0D3FD49F61963E25CCD
S214442120012A40F0FC800022E25449F61C63E3583E
S214442130722B00F0EF80732B40F0F18003B0BDE8C3
S214442140F04F02F0EDBD019A02EB000B009A9BF8AB
S21444215040BF02F800B0704643E7992B83D101F0A4
S214442160FBFC80E7B3F5BC7F45D0B3F5BE7F45D0D6
S214442170B3F5BA7F7FF477AF01F038FD73E740F2EA
S214442180855293422BD015D8B3F5AE6F21D00AD8DA
S214442190B3F5407F26D040F2013293427FF463AFDA
S2144421A001F008FE5FE7B3F5B06F7FF45CAF01F073
S2144421B05DFE58E740F2955293420DD040F2777256
S2144421C0934224D0B3F5B26F7FF44DAF01F0C0FE16
S2144421D049E701F0FBFD46E701F0CCFE43E701F09A
S2144421E08FFE40E701F0C6FD3DE701F03AFC3AE7D2
S2144421F001F04AFC37E701F01BFD34E701F03AFDF5
S21444220031E701F0CBFC2EE701F054FD2BE701F05B
S214442210CBFE28E701F05AFC25E740F251129342E0
S2144422207FF436AF01F028FF32E701F0CFFE2FE708
S21444223001F0F2FE2CE701F001FF29E78C2B25D0B4
S214442240922B7FF43FAF02F079F83BE7AA2B26D0D7
S21444225007D89A2B0ED0A02B7FF434AF02F08EF919
S21444226030E7C82B09D0B3F5F36F7FF42BAF02F0F9
S2144422704FFA27E702F042F924E702F00BFA21E787
S21444228001F0CAFF1EE702F0E1F81BE701F0EEFF9B
S21444229018E701F047FF15E701F08CFF12E702F05C
S2144422A0B9F90FE7932B2FD0972B7FF425AF02F085
S2144422B01FFB21E7C92B13D007D8A12B18D0AA2B74
S2144422C07FF41AAF02F0E4FB16E740F299729342A9
S2144422D07FF412AF02F0C2FC0EE702F061FB0BE79C
S2144422E002F016FC08E700BF588740207C4841208F
S2144422F002F096FB00E702F01FFAFDE602F064FAED
S214442300FAE602F043FCF7E602F090FAF4E602F04E
S214442310B9FC02E703B0BDE8F04F02F0E3BC03B0FB
S214442320BDE8F08FEC4BED4A5969DFF8D4C30A4058
S214442330EB492DE9F0475A610022EA4D4FF0000878
S214442340E94E4FF00009DA6583F877209A67E74C40
S214442350DFF8B0E3DFF8B0A3C3E90212197C21F03A
S21444236007011974D96A2940D962996C01F0004171
S2144423709964D96C3140D964196D01F0604141F4D7
S214442380C8211965DA49C3E91512196E01F070417E
S2144423901966596E29405966996E01F0004199664E
S2144423A0B3F86C1001EA0C01A3F86C10B3F8701083
S2144423B001EA0C01A3F87010D96F01F07F41D96788
S2144423C0D3F88000CB49D3F8A070084083F8942013
S2144423D0C3F88000D3F8880000F07F40C3F8880034
S2144423E0D3F88C0000F07F40C3E92302D3F898006A
S2144423F02040C3F89800D3F89C0000F07C40C3F813
S2144424009C00BD480740C3F8A070D3F8A47007F0FA
S2144424104047C3F8A470D3F8A8703740C3E92A727B
S214442420D3F8B0700F40C3F8B070D3F8B47007F068
S2144424304047C3F8B470D3F8BC7007F04047C3F8BD
S214442440BC70D3F8C07007F07F47C3F8C070B3F8C9
S214442450B87083F8C32062F30D07A3F8B87093F8F6
S214442460C47027F0030783F8C470D3F8C870C3F861
S214442470DCA007F00047C3F8C870D3F8CC70074018
S214442480C3F8CC70D3F8D07007F07047C3F8D07058
S214442490D3F8D47007F07F47C3F8D470B3F8D87035
S2144424A007EA0E07A3F8D870D3F8E07007F0404761
S2144424B0C3F8E070D3F8E47007F07847C3E939729C
S2144424C093F8EC7062F3000783F8EC70D3F8F0707E
S2144424D007F07E4747F48037C3F8F070D3F8F470BB
S2144424E03740C3F8F470D3F8107107F04047C3F888
S2144424F01071D3F814713740C3E94572D3F81C7190
S2144425000F40C3E94222C3E94089C3F81C71D3F89B
S2144425102071A3F8302107F0404783F85C21A3F8E4
S2144425207421C3F840A1C3E9487293F8287127F090
S214442530030783F82871D3F82C7107F06047C3F873
S2144425402C71D3F8347107F07047C3F83471D3F85C
S214442550387107F07F47C3F83871B3F83C7107EA1F
S2144425600E0ED3F844710740A3F83CE1C3F8447117
S214442570D3F8487107F07847C3F84871B3F84C71FC
S21444258007F47847A3F84C71D3F8507107F07E47A8
S21444259047F48037C3F85071D3F854713E40C3F8BB
S2144425A05461D3F8586106F06046C3F85861D3F8CE
S2144425B070612E40C3E95889C3F87061D3F87861D6
S2144425C0A3F87C212E40C3F8802183F88821C3F8E1
S2144425D07861D3F8846183F8F02106F07F46C3F827
S2144425E0A821A3F8AC21C3F88461D3F88C61C3F85E
S2144425F0B0212640A3F8B421C3F8B82183F8BC21FF
S214442600C3F8C02183F8C421C3F8C82183F8CC2179
S214442610C3E9636293F8946126F00F0683F89461E5
S214442620D3F8D06106F07C46C3F8D061D3F8D461C1
S2144426300640C3E97A22C3E96622C3E96822C3F89E
S214442640D461D3F8DC6183F8A02206F00046C3F8D0
S214442650382283F83C22C3F8402283F8442283F885
S2144426605E22C3F8482283F84C22C3F8502283F8EB
S2144426703422C3E97762D3F854620640C3F85462FE
S214442680D3F8586206F07E46C3F8586293F8A462BC
S21444269026F01F0646F0010683F8A462B3F8A86243
S2144426A062F30906A3F8A86293F8AC6226F00F0614
S2144426B083F8AC6293F8B06262F3020683F8B062C1
S2144426C0D3F82C6230400D4EC3E98B0293F8B40223
S2144426D062F303001AE000BFD083402000E01FE00E
S2144426E00000E2810000F0FF000080FF0000FEFFD3
S2144426F00080204E0000FCFF0000C0FF00E0FFFF0B
S21444270000C0FFFF00F0FFFF0000C04B83F8B40298
S214442710D3F80C0200F07040C3F80C0283F8102281
S214442720D3F81402A3F8EC2200F00040C3F8F022D9
S214442730C3F81402B3F8180200EA0C0CD3F82002CB
S2144427400540D3F82402A3F818C20840C3F824026C
S214442750D3F8D0022040C3F8D002D3F8B80200F031
S2144427607E40C3F8B802D3F8BC0200F00040C3F879
S214442770BC0293F8C00220F00F0083F8C002D3F8DE
S214442780C40200F07840C3F8C402D3F8C80200F08C
S2144427907F40C3F8C802B3F8CC023040A3F8CC025A
S2144427A0D3F8E80200F00040C3F8E80293F8F402D5
S2144427B062F30000C3E9872583F8F402C5F30745AE
S2144427C0D3F8F80262F3071500F07F4083F82252EC
S2144427D0C3F8F802D3F8FC02D3F80453084005F0D3
S2144427E07845C3F8FC02D3F80803C3F8045300F052
S2144427F07840D3F81453C3E9C20293F8100305F0A3
S214442800784562F30000C3F81453D3F8185383F89A
S2144428101003D3F8000305F07F4500F04040C3F8AA
S2144428201853C3F80003B3F81C033040A3F81C0342
S214442830D3F8200300F07E40C3F82003D3F82403E3
S2144428402040C3E9C90293F82C0362F3000083F8DE
S2144428502C03D3F8300300F07F40C3F83003D3F89A
S21444286034030140C3F83413D3F838130C40D3F878
S214442870581301F07841C3F83843C3E9B689C3E92D
S214442880D61293F86013C3F8642362F30001C3F8C6
S214442890742383F86013D3F8501301F04041C3F80F
S2144428A05013D3F8541301F07841C3F8541393F8F3
S2144428B0681362F3000183F86813D3F86C1301F0CD
S2144428C07F41C3F86C1393F8721321F0030183F825
S2144428D0721393F8781362F3000193F87E2322F080
S2144428E0030283F87813C3E9D08983F87E23BDE8CE
S2144428F0F08741F698730849002258430B1828304D
S214442900DA64084483F848202023013B00F8012B6E
S21444291013F0FF03F9D170475887402041F6987367
S21444292010B558430B4C41F692732218D35A2822BA
S2144429305A43002311185030104421441A46204468
S21444294081F870304B67013300F8012BDBB2202B43
S214442950F9D110BD588740202DE9F8439946234BBA
S2144429600546884603EB00139B6A402B31D8204922
S2144429704FF4FB5303FB001342F644015B5843B346
S21444298041F698761B4C00274FF0280C06FB00F3C4
S214442990E11801F5FC511031F8B248451BD32846DE
S2144429A07543FFF7A6FF41F6907160192826012269
S2144429B0435A06FB035513442C4484F87120C4F848
S2144429C0748084F87090C824B3FBF4F204FB12338A
S2144429D04352BDE8F883088812F807E00CFB003041
S2144429E020443844013780F850E0D5E7B81F4020EB
S2144429F07C4841205887402041F6987241F69273AD
S214442A002DE9F34102FB00F14E4D04466A18D05AB4
S214442A10282202FB00122A4492F87020082A31D851
S214442A20494B082203EB04139A62282341F6947612
S214442A3003FB00F241F6987320466343D118EF181F
S214442A40503329441344414A2B4402EB0412009366
S214442A504B6FB95D1AF086F9012C80462FD143F6A8
S214442A602C711C206B5C0133B3FBF0F200FB123379
S214442A706B54B8F1000F2BD0B8F1020F40D002B01F
S214442A80BDE8F081102A04D82F4B102203EB041320
S214442A90CAE7182A05D82C49182301EB04118B627F
S214442AA0C3E7202A04D82849202301EB0411F6E77B
S214442AB0402ABAD82449402301EB0411EFE7BB5D12
S214442AC00E210133B3FBF1F201FB1233BB55D0E7C1
S214442AD02046FFF723FF41F6987041F69271604313
S214442AE028242E18735A04FB03040133C8202544B3
S214442AF0B3FBF0F200FB123385F871807352BEE7E5
S214442B002046FFF70BFF41F6987041F6927100227B
S214442B10444328202E19735A00FB03440133C8202B
S214442B20254485F87120B3FBF0F200FB1233064AC5
S214442B307352D2E92231013341F10001C2E9223114
S214442B409DE700BF58874020B81F4020DC1F402028
S214442B50F8B500240A4D41F698760A4F06FB04F26F
S214442B602821E0B2D35B01FB03232B4493F8713056
S214442B70012B01D1FFF740FF0134062CEED1F8BDFE
S214442B8058874020EAA6402008B50B21034825F084
S214442B907FFB034B83F8280908BD00BF0217294072
S214442BA0A47A402001290A4628BF0122072819D8BA
S214442BB0DFE800F004070B0D1012141600210A4833
S214442BC001E00A21094825F02ABB0C21F7E7022137
S214442BD00748F8E70D21F2E70E21F0E70F21EEE76C
S214442BE00021F5E7704700BF021729401017294017
S214442BF00017294007281AD8DFE800F004070B0E10
S214442C001013151708210B4801E00B210A4825F03C
S214442C103FBB01210948FAE70B21F4E704210848A1
S214442C20F5E70521FBE70821F9E70A21F7E7FF2046
S214442C30704700BF0617294002172940121729403B
S214442C400417294001284FF002010CBF002201223C
S214442C5010B50446034825F0E2FA034A4CF24053C2
S214442C60D45010BD081729407C48412005281DD85B
S214442C70DFE800F003080C1014180D4A4CF27453A5
S214442C80D05A70470A4A4CF27653F9E7084A4CF24F
S214442C907853F5E7064A4CF27A53F1E7044A4CF285
S214442CA07C53EDE7024A4CF27E53E9E7FF20704737
S214442CB07C48412008B50621002014F030F8024A2A
S214442CC04CF27453D05208BD7C48412010B50221C2
S214442CD0012014F024F8064C4CF276532B21E05293
S214442CE0012014F01CF84CF27E53E05210BD00BF95
S214442CF07C48412010B50321022014F010F8094CFA
S214442D004CF278530421E052022014F008F84CF2B6
S214442D107A530521E052022014F001F84CF27C5319
S214442D20E05210BD7C484120002113F0E5BE084A1D
S214442D304CF2385382B00749D35800930B68009A34
S214442D409B1A0193019B8342F8D902B0704700BF97
S214442D507C484120B40D422038B50F4D0F4C95F8B1
S214442D6090305BB901234CF23C5285F89030A3581E
S214442D700133A350BDE8384006F04EBE0BF0F8F9D8
S214442D804CF23C52002385F89030A3580133A350AC
S214442D904CF23852EBE700BFB81F40207C48412035
S214442DA00020FFF74FBF10B58D20244C1CF04EFB7F
S214442DB0002223498D201CF048FB8F201CF046FB44
S214442DC0002220498F201CF040FB97201CF03EFB3D
S214442DD000221D4997201CF038FB9A201CF036FB35
S214442DE000221A499A201CF030FB194900201EF094
S214442DF075FE184902201EF071FE17490A201EF07F
S214442E006DFE16490D201EF069FE21460122002063
S214442E101FF0E6F804F59671012202201FF0E0F850
S214442E2004F26C5101220A201FF0DAF804F28C51A5
S214442E3001220D20BDE810401FF0D2B8884B412037
S214442E40E9244600EF244600F5244600FB244600C9
S214442E5064B0460038B046000CB04600E0AF4600CA
S214442E6010B48AB90949D1F86C3891F8B848CA18E8
S214442E70013301F6B801DBB282F8584610BC012291
S214442E8041F84C3C1FF0FCB910BC70477C484120CC
S214442E9010B48AB90949D1F8743891F8D848CA1890
S214442EA0013301F6D801DBB282F8584710BC012240
S214442EB041F8643C1FF0E4B910BC70477C4841209C
S214442EC0194B012142F644000022195044F2A470E2
S214442ED0195046F20470195048F2646019504AF288
S214442EE0C45019504CF22450195042F648015A50D6
S214442EF044F2A8715A5046F208715A5048F2686132
S214442F005A504AF2C8515A504CF22851C3E9C12289
S214442F105A504CF248524CF2503199504CF244526A
S214442F204FF44861995070477C48412010B5064B91
S214442F304FF4FB5404FB003042F64803C15042F6BB
S214442F404C03C25010BD00BF7C484120094BD3E916
S214442F50C1218A420BD01A4492F8042202700020FF
S214442F60D3F804230132D2B2C3F8042370470120B5
S214442F70704700BF7C48412007B501220DF1070188
S214442F808DF8070000201EF07FFE03B05DF804FBBA
S214442F900FB470B5C2B0002446AA02AE52F8041B61
S214442FA0304601920FF0A0FC30460CF05BFDC5B2F3
S214442FB0E3B29D4204D842B0BDE8704004B07047C6
S214442FC0305D0134FFF7D8FFF2E708B58E201CF0D9
S214442FD03DFA96201CF03AFA0748FFF7D9FF07490E
S214442FE000201DF0FBFC012005491DF0F7FC0548B8
S214442FF0BDE80840FFF7CCBFE0934600B4AF4600B8
S21444300088AF4600E89346000B2938B5044614D1E9
S21444301042F644030E4D00220E48EA50FFF7B8FF2E
S21444302042F64803EB581BB142F64C02A858984760
S2144430302046BDE838401AF00BBC074B1A6832B13C
S214443040002206481A60BDE83840FFF7A1BF38BDE5
S2144430507C484120EE934600BC7041200A944600CA
S2144430600B2938B505460E4C13D144F2A4730022FE
S2144430700C48E250FFF78CFF44F2A873E3581BB1A8
S21444308044F2AC72A05898472846BDE838401AF037
S214443090DFBB44F2A073E2580AB10022E25038BDC6
S2144430A07C484120299446000B2938B5044614D15F
S2144430B046F204730E4D00220E48EA50FFF768FFAE
S2144430C046F20873EB581BB146F20C72A858984760
S2144430D02046BDE838401AF0BBBB074B1A6832B1ED
S2144430E0002206481A60BDE83840FFF751BF38BD95
S2144430F07C484120459446007CAF4120619446007C
S2144431000B2938B504464FF4FB55134815D105FB37
S214443110040542F6440300221048EA50FFF738FFFD
S21444312042F64803EB581BB142F64C02A85898475F
S2144431302046BDE838401AF08BBB05FB040404F572
S2144431402154236833B1002305482360BDE8384042
S214443150FFF71EBF38BD00BF7C4841207F94460021
S2144431609B9446000B2938B504464FF4FB55134848
S21444317015D105FB040542F6440300221048EA50E4
S214443180FFF706FF42F64803EB581BB142F64C02E3
S214443190A85898472046BDE838401AF059BB05FB66
S2144431A0040404F52154236833B1002305482360FE
S2144431B0BDE83840FFF7ECBE38BD00BF7C48412030
S2144431C0BA944600D69446000B2938B504464FF4C4
S2144431D0FB55134815D105FB040542F6440300226B
S2144431E01048EA50FFF7D4FE42F64803EB581BB1AA
S2144431F042F64C02A85898472046BDE838401AF094
S21444320027BB05FB040404F52154236833B100238B
S21444321005482360BDE83840FFF7BABE38BD00BF56
S2144432207C484120F59446001195460038B50A245A
S2144432303C4D2946002014F083F938B1013C14F083
S214443240FF04F6D121463848FFF7A2FE0A24374D3C
S2144432502946012014F074F938B1013C14F0FF04F7
S214443260F6D101213048FFF793FE0A24304D294613
S214443270022014F065F938B1013C14F0FF04F6D18D
S21444328002212948FFF784FE00222A49B4200A2452
S2144432901CF0DBF800222849B5201CF0D6F80022A2
S2144432A02649B6201CF0D1F8B4201CF0CFF8B5203F
S2144432B01CF0CCF8B6201CF0C9F8002013F0D6FD5C
S2144432C038B1013C14F0FF04F7D121461C48FFF7FF
S2144432D05FFE0A24012013F0C9FD38B1013C14F006
S2144432E0FF04F7D101211648FFF752FE0A240220B4
S2144432F013F0BCFD38B1013C14F0FF04F7D10221B1
S2144433000F48FFF745FE0121002013F031FE01214E
S214443310084613F02DFE01210220BDE8384013F084
S21444332027BE00BF50A346004C954600F4A2460074
S21444333098A246001D7B4500237B4500297B45001B
S2144433403095460038B51C4C054620680430204469
S214443350FFF7FCFD012801D1012038BD2368E2189F
S21444336010790A2810D00D280ED0082815D123B17C
S214443370013B12482360FFF70BFE2368AB42EBD3B6
S21444338025440020E87006E00D48FFF701FE236858
S2144433900020234418712060DFE7A0F120035E2B51
S2144433A0EBD8FFF7E9FD2368E11801330A79236077
S2144433B0303A81F80421E0E77C4841206195460094
S2144433C07095460010B58020FFF7BCFF90B90A4CB4
S2144433D023797BB10949201D0CF03AFB20B90848F3
S2144433E0BDE81040FFF7D4BD211D0648BDE8104097
S2144433F0FFF7CEBD10BD00BF7C4841206595460012
S2144434006B954600739546002DE9F04F082389B026
S214443410002492463B4A054689464FF064081068A5
S214443420EDB2516802AF012622468DF810408DF861
S2144434301C40DFF8E8B0CDE905346B4403C351467D
S214443440484624F0ECFE04AA214640F2555328464A
S214443450CDF8048000978DF81C608DF810400594D4
S2144434601AF0E4F8284B04AA2146284602934FF65D
S21444347007738DF81060ADF80C300623CDE900785C
S21444348005935B461AF0D2F8204A06232146029258
S2144434904FF6FF72059328465B46ADF80C2004AA07
S2144434A08DF81060CDE900781AF0C0F8184A062363
S2144434B021460292284604AA05935B46ADF80C4082
S2144434C08DF81060CDE900781AF0B0F8114B124A26
S2144434D0214628468DF81060CDE90232082304AA16
S2144434E005935B46CDE900781AF0A0F80A20FFF76A
S2144434F01EFC32465146484624F091FE09B0BDE8CB
S214443500F08F00BF7C8946001000500010019FFFDA
S2144435101002C0007102030405060708F100DA1819
S2144435202DE9F0410446002855D16D201BF08EFF4E
S2144435302246C0496D201BF088FF6E201BF086FF94
S2144435402246BD496E201BF080FF01220821BB485D
S21444355024F065FE01220521B84824F060FEB84AEE
S214443560B849204619F0F4FA012120461AF0B2FA76
S21444357022460E2120461AF009F920461AF088FA07
S2144435802346B14A0E21204619F020FC2346AF4A72
S2144435900E21204619F05EFCFEF7C4FE2046FFF7D7
S2144435A0A8F9AB4B012242F644015A5003F5215385
S2144435B01A6041F698700023A64A4443A648A3508E
S2144435C004441A46013384F871202834C82BF9D1B0
S2144435D00020BDE8F081012846D0022840F08980CA
S2144435E074209E4F1BF032FF00229D4974201BF02E
S2144435F02CFF75201BF02AFF00229A4975201BF0E9
S21444360024FF01220421984824F009FE01220621C1
S214443610964824F004FE0025954A20469549DFF84E
S214443620B88219F095FA20461AF032FA05F10E06D9
S21444363058F83530904A0220F6B223F060430135FC
S214443640314619F0C3FB3A46002331460220503730
S21444365019F000FC0B2DE9D17D4B012246F2047192
S2144436605A5003F5CE43A3E77120844F1BF0EEFE79
S2144436700022834971201BF0E8FE72201BF0E6FE10
S2144436800022804972201BF0E0FE2246072177483C
S21444369024F0C5FD22460221734824F0C0FD0025CF
S2144436A0794A20467949DFF8348219F051FA20469F
S2144436B01AF0EEF905F11C0658F83530744A012024
S2144436C0F6B223F060430135314619F07FFB3A46A3
S2144436D0002331460120503719F0BCFB042DE9D1B4
S2144436E044F2A4715A4B01225A5044F2A0715A50E3
S2144436F05FE7032859D0042800F0F48005287FF4B7
S21444370058AF7B20634D1BF0A1FE002262497B200C
S2144437101BF09BFE7C201BF099FE00225F497C2018
S2144437201BF093FE01220E21504824F078FD01221E
S2144437305B48114624F073FD5A4A5B49204619F00B
S21444374007FA20461AF0A4F9012255492046FFF705
S2144437505BFE564A5449204619F0FAF920461AF0B8
S21444376097F92B68524A0E2123F06043204619F0FD
S2144437702DFB00234F4A0E21204619F06BFBAB6805
S2144437804B4A0F2123F06043204619F01FFB0023C9
S214443790494A0F21204619F05DFB4CF224512C4B2C
S2144437A001225A504CF22051A1E77720434F1BF098
S2144437B04DFE0022424977201BF047FE78201BF03E
S2144437C045FE00223F4978201BF03FFE012200219F
S2144437D03D4824F024FD01223B4800251146DFF8ED
S2144437E0008124F01CFD394A3949204619F0B0F9C5
S2144437F020461AF04DF905F10E0658F83530354A8C
S2144438000320F6B223F060430135314619F0DEFA60
S2144438103A46002331460320503719F01BFB0A2D45
S214443820E9D148F264610A4B01225A5048F2606179
S2144438305DE700BF4DF2450053F2450008172940A6
S21444384044A74600884140204C2040202C4C402031
S2144438507C484120E8A64020588740202C604020E1
S21444386095F245009BF245000E1729400C17294057
S21444387094A64600383840206C2040208C5A40207D
S21444388077F245007DF24500ECA64600E03C402039
S2144438905C2040209C8C4600D7F24500DDF2450073
S2144438A01017294084894600402A40208CA54600AB
S2144438B09C2040202C7E40207C7E40202C6A402049
S2144438C0B3F24500B9F24500061729403CA6460027
S2144438D0903340207C2040200C8D4600648D46006A
S2144438E0BC8C46007920294D1BF0B0FD00222849A7
S2144438F079201BF0AAFD7A201BF0A8FD002225495A
S2144439007A201BF0A2FD01220A21234824F087FCDA
S21444391001220921204824F082FC204A20492046DE
S21444392019F016F920461AF0B3F809221A49204627
S214443930FFF76AFD1B4A1A49204619F009F9204642
S2144439401AF0A6F82B68184A0E2123F06043204646
S21444395019F03CFA0023154A0E21204619F07AFA4B
S214443960AB68114A0F2123F06043204619F02EFA23
S21444397000230F4A0F21204619F06CFA4AF2C4512C
S2144439800C4B01225A504AF2C051B0E6AC8C460069
S214443990C5F24500CBF24500081729408489460005
S2144439A0E82E4020E4A546008C2040202C7440207D
S2144439B07C7440207C48412041F69872084B02FBB8
S2144439C0003310B503EB8104E278A07800EB0220C4
S2144439D0627802EB002213F8210000EB022010BDAF
S2144439E05887402010B5094B41F6987404FB0030C4
S2144439F0130A00EB810181F8282081F82930130C42
S214443A00120E81F82A3081F82B2010BD58874020AA
S214443A1013B502AB044603E9060041F69871094A19
S214443A209DF8043001FB0022009903F03F0321F087
S214443A306041FEF791FF204602B0BDE81040FEF715
S214443A4058BF00BF80874020FDF708BF70477047C7
S214443A507047704770477047704770477047704765
S214443A607047074B074A196858799160197941EAB3
S214443A70002191819979DB799173D373704700BFA4
S214443A8058874020D08340200E490F4810B54A78C6
S214443A900B7802F0010443EA0423C2F34104C2F360
S214443AA0C10243EA442343EAC2238A7843EA4233C0
S214443AB0CA7843EA4253426902F060421343436180
S214443AC010BD00BF58874020D0834020074B08498C
S214443AD01B7803F003021B0903F0040313430A7C18
S214443AE022F0070213430B74704700BF58874020E8
S214443AF0D08340200549064B0A7E1B7822F01F02DD
S214443B0003F01F0313430B76704700BFD083402057
S214443B10588740200549064B0A7F1B7822F01F022F
S214443B2003F01F0313430B77704700BFD083402036
S214443B30588740200649074B91F820201B7822F0EE
S214443B400F0203F00F03134381F82030704700BF81
S214443B50D0834020588740200E4A0F4990785378A7
S214443B6043EA0023A1F825301079D37843EA0023AA
S214443B7090790B8553794A8D43EA0023C0F380102D
S214443B8002F40042C3F30D0343EA803313434B85E8
S214443B90704700BF58874020D0834020114B1248BE
S214443BA010B55A78997802F003041B7843EA042344
S214443BB0C2F3810443EA8423C2F30114920943EA1C
S214443BC0043343EA823301F00302C1F3810143EA3A
S214443BD00243C26A120D43EA814312051343C36289
S214443BE010BD00BF58874020D08340200E4B0F4A5C
S214443BF05878197841EA002158791186997801F065
S214443C000F0182F83210D97882F83310197941EAD4
S214443C10002191869979DB7901F00F0182F83730DB
S214443C2082F83610704700BF58874020D083402023
S214443C300E4B0F4A5878197841EA00215879118773
S214443C40997801F00F0182F83A10D97882F83B103F
S214443C50197941EA002191879979DB7901F00F01BE
S214443C6082F83F3082F83E10704700BF58874020A5
S214443C70D08340200D4B0E4A5878197841EA0021EB
S214443C805879A2F84010997801F00F0182F8421052
S214443C90197941EA0021A2F844109979DB7901F0B8
S214443CA00F0182F8473082F8461070475887402004
S214443CB0D08340202D492E4A10B50B78487803F01F
S214443CC07F0343EAC013887843EAC033C87843EA9C
S214443CD0C053906C00F00040034348799364C0F3AB
S214443CE040040B79897982F84C3000F001031B02BA
S214443CF043EA4423C0F3800443EA8423C0F3C00465
S214443D0043EAC423C0F3001443EA0433C0F3401424
S214443D1043EA4433C0F38014C00943EA843343EA95
S214443D20C03301F0010043EA0043C1F3400043EAD4
S214443D304043C1F3800043EA8043C1F3C00043EAF2
S214443D40C043C1F3001043EA0053C1F34010C1F32B
S214443D50801143EA405343EA8153D16C21F4FF0176
S214443D6021F4FE410B43D36410BD00BF5887402066
S214443D70D08340200D4A0E4810B55178137801F090
S214443D800F04C1F3001143EA042343EA0133917854
S214443D9043EA4133D17843EA4153016D01F060412F
S214443DA00B4303655368436510BD00BF58874020E6
S214443DB0D0834020034A044B116852689965DA65FB
S214443DC0704700BF58874020D0834020244A254966
S214443DD070B55578137805F003069078D47843EA9E
S214443DE00623C5F3810643EA8623C5F30116AD09C7
S214443DF043EA063343EA8533C0F3011543EA0543F1
S214443E00850900F00F0043EA854304F0030543EABE
S214443E100553C4F3810543EA8553C4F30115A40945
S214443E2043EA056343EA84630C6E04F07044234318
S214443E3054790B661379D27981F86430230104F0FF
S214443E40030403F4706343EA02334A6E43EA0050C1
S214443E50054B40EA046013401843486670BD00BFF3
S214443E6058874020D0834020FF0000FC70B5224D88
S214443E70224A2C78E878C4F3401604F00F032979D4
S214443E8043EA0613C4F38016E40943EA461343EAB6
S214443E9084136C7843EAC413AC7843EAC43300F022
S214443EA0030443EAC453C0F3810443EA4463C0F3BF
S214443EB00114800943EAC46343EA4073906E00F0F9
S214443EC00040034301F0030093668B0803F00403A9
S214443ED00343880800F0080003438808C90900F033
S214443EE01000034343EA411392F86C1021F03F015B
S214443EF00B4382F86C3070BD58874020D0834020F6
S214443F00114A124810B55178137801F0030443EA75
S214443F100423C1F3810443EA8423C1F301148909C9
S214443F2043EA043343EA8133A0F870305388A0F858
S214443F3072309388A0F87430937980F87630D379C9
S214443F4080F8773010BD00BF58874020D08340208B
S214443F50064B074A1968587991671979DB7941EA1B
S214443F60002182F87E30A2F87C10704758874020A3
S214443F70D0834020094A0A491378907881F88030E3
S214443F8053781843D378074A9B0443EA0023D1F86E
S214443F90800002401343C1F8803070475887402061
S214443FA0D0834020FF0000FC08B5054B18880CF071
S214443FB075FB04490CF0C6FB034BC3F8840008BDEC
S214443FC058874020CDCCCC3DD0834020104B41F682
S214443FD09871104A595C82F8881041F69B71585C77
S214443FE041F69A71595C41EA0021A2F8891041F6DB
S214443FF09D71585C41F69C71595C41EA0021A2F8D7
S2144440008C1041F69F715B5C82F88E30704700BF1F
S21444401058874020D0834020064A41F69871064B84
S2144440205158C3F8901041F69F71525C83F894201F
S214444030704700BF58874020D08340200C4A41F642
S2144440409F730C4910B541F69974D05C41F6987349
S214444050D35C125D02F0010243EA0223D1F89820B1
S214444060520C43EA402352041343C1F8983010BD1F
S21444407058874020D0834020284941F69973284ADF
S21444408070B5C85C41F69A73CD5C41F69B7300F0FC
S2144440900306CC5C41F69873CB5C43EA0623C0F334
S2144440A0810643EA8623C0F30116800943EA0633B1
S2144440B043EA803305F00300C5F3810543EA004331
S2144440C004F0030043EA854343EA0053C4F3810003
S2144440D0A40943EA8053D2F89C0043EA046300F000
S2144440E07C40034341F69F70C2F89C3041F69C7373
S2144440F0CB5C82F8A03041F69D73CB5C095C1B0216
S21444410003F47C5343EA8133D2F8A01021F47F11A0
S21444411021F47C510B43C2F8A03070BD5887402030
S214444120D0834020214843F63073214930B5C35AE2
S2144441305BBAA1F8A43043F63373C25C43F63273D9
S214444140C2F30115C45C930943EA850304F00F05E2
S214444150240943EA051343F63675455DED0843EAFC
S2144441600523C2F3800543EA4533B1F8A65005F467
S21444417040452B43A1F8A63043F63473C55C43F65A
S2144441803573C35C43EA0523A1F8A830C2F3C003E1
S214444190520143EA440302F060021A4391F8AA30FB
S2144441A023F07F031A4381F8AA2030BD5887402065
S2144441B0D0834020164A43F63073164910B5D35A76
S2144441C05BBAA1F8AC3043F63273D05C43F6337333
S2144441D0D35C43EA0023A1F8AE3043F63673D05C92
S2144441E043F63473D45C43F63573D35C43EA042213
S2144441F000F00103C0F3400043EA4203D1F8B02084
S214444200920C43EA404392041343C1F8B03010BDC5
S21444421058874020D0834020124A43F63071124BD0
S214444220515A49BAA3F8B41043F63271505C43F677
S2144442303371515C41EA0021B3F8B60061F30D00D6
S21444424043F63671A3F8B60043F63770515C125CF9
S21444425042EA0122B3F8B81062F30D01A3F8B8108D
S214444260704700BF58874020D083402030B543F67F
S2144442703073304C3049E35A5BBAA1F8BC3043F64D
S2144442803673E05C43F63773E25C43F63273E55CC0
S21444429000F0030343EA8503C0F3800543EA85231D
S2144442A0C2F3800543EAC523850943EA0533B1F8DA
S2144442B0BE5005F440452B43C2F3C005A1F8BE30BA
S2144442C043F63373E35C81F8C030C0F3C0031B028B
S2144442D043EA452302F0030543EA852343F634754F
S2144442E0655D43EA0533C0F30015C0F3401043EA66
S2144442F00553C2F3001543EA45539509120943EAA8
S2144443008553D1F8C05002F0020225F47F050243DB
S21444431025F47F452B43C1F8C03043F63573E35C40
S21444432081F8C33091F8C43023F003031A4381F86C
S214444330C42030BD58874020D0834020F0B543F693
S2144443403273404F404DFE5C43F63473F95C43F69B
S2144443503373C6F3801CF85C43F63573FC5C43F653
S2144443603673FA5CF30943EA4C0343F6317C42EA7B
S214444370042217F80CC043EA8C03C6F3401C43EAF5
S2144443808C23C6F3001C43EACC23C1F3400C43EA17
S2144443900C3343F6307C17F80C7043EA4733C6F3C5
S2144443A0C00743EA4753C6F3800743EA8753C0F33C
S2144443B0001743EAC753470943EA0763C4F30117A0
S2144443C0A40943EAC763C6F3400706F0010643EA76
S2144443D0477343EA8673D5F8C86006F0004633430D
S2144443E001F00106C5F8C830C2F30903C0F3C002A1
S2144443F043EA862343EAC223C0F3800243EA0233F5
S214444400C0F3400200F0010043EA4233C1F3C00265
S21444441043EA803343EAC433C1F3001443EA4443D3
S2144444208C09C1F3800143EA844343EA025343EAD6
S2144444304151D5F8CC309B0D9B051943C5F8CC109B
S214444440F0BD00BF58874020D0834020284843F61C
S214444450307343F636722749F0B5C35A43F632757D
S214444460845C43F635725BBA455D825CA709A1F865
S214444470D03043F6337347EA820743F63772C65C56
S21444448043F63473825CC35CB009B1F8D2C042EAE6
S214444490042240EA8500C6F3810543EA0623C6F3B0
S2144444A0011640EA8520144DC3F309030CEA050CB3
S2144444B043EA862340EA0C0043EA0733A1F8D200D5
S2144444C0C4F38100C4F3011443EA8053D1F8D40002
S2144444D000F07F400343C1F8D430C2F30903B1F877
S2144444E0D82043EA842315402B43A1F8D830F0BDA6
S2144444F058874020D083402000F0FFFF1D4943F6F4
S21444450030731D48F0B5CB5A43F632745BBA0E5D31
S214444510A0F8DC3043F63373CA5C43F63573CD5C9F
S214444520C2F3810443F634732F09CB5C44EA870410
S21444453043F6367743EA0223C95D41EA052144EA55
S2144445408111A0F8DE10C3F30901C2F3001343EA55
S21444455041039109C2F3401243EAC62343EAC163C6
S21444456043EA4273D0F8E02002F040421343C0F8D6
S214444570E030F0BD58874020D083402070B52349B2
S21444458043F6367443F6357543F630730C5D4E5D2C
S214444590CB5AA5091E485BBA45EA860543F63776E4
S2144445A0A0F8E43043F633738E5DCA5C43F6347346
S2144445B046EA042443F63276CB5C8E5D910943EAA0
S2144445C0022341EA8601C2F38006C3F3090341EAA3
S2144445D08621B0F8E66006F478463143A0F8E61043
S2144445E0C2F3C00143EA8123C2F30011520943EAED
S2144445F0C52343EA415343EA8453C0F8E83090F86D
S214444600EC3062F3000380F8EC3070BD58874020ED
S214444610D08340201D4A43F630731D4870B5D35AA4
S2144446205BBAA0F8F03043F63273D45C43F6347386
S214444630D55C43F63373D15C2B09C5F3C00543EA16
S214444640011143F63673D65C43F63573D35CDB0010
S21444465043EA5612C4F3400343EA450304F0010513
S214444660A40843EA850343EAC403B0F8F24004F4DA
S2144446707E442343A0F8F23041EA0233D0F8F420D3
S214444680D20DD2051343C0F8F43070BD588740208D
S214444690D08340201B4943F631731B4830B5CB5C6E
S2144446A080F8F83043F63273CA5C43F63573CD5C13
S2144446B043F63473CC5C43F63073C95C93091B02EF
S2144446C043EA8123C2F3401143EA8143C2F38001A3
S2144446D0C2F3C00243EAC143D0F8F81043EA025397
S2144446E02A0905F00F0543EA4253084A43EA45635C
S2144446F00A401343C0F8F830230943EA041480F808
S214444700FC4030BD58874020D0834020FF0000E066
S214444710074943F63073074ACB581BBAC2F80831E8
S21444472043F63473CB581BBAC2F80C31704700BFFB
S21444473058874020D0834020214845F6C863214905
S21444474030B5C35A5BBAA1F8103145F6CB63C25CA8
S21444475045F6CA63C2F30115C45C930943EA85036C
S21444476004F00F05240943EA051345F6CE65455D76
S214444770ED0843EA0523C2F3800543EA4533B1F81E
S214444780125105F440452B43A1F8123145F6CC634B
S214444790C55C45F6CD63C35C43EA0523A1F81431F2
S2144447A0C2F3C003520143EA440302F060021A43D0
S2144447B091F8163123F07F031A4381F8162130BD51
S2144447C058874020D0834020164A45F6C863164989
S2144447D010B5D35A5BBAA1F8183145F6CA63D05C13
S2144447E045F6CB63D35C43EA0023A1F81A3145F679
S2144447F0CE63D05C45F6CC63D45C45F6CD63D35CDF
S21444480043EA042200F00103C0F3400043EA4203B3
S214444810D1F81C21920C43EA404392041343C1F856
S2144448201C3110BD58874020D0834020F0B545F653
S214444830CA632D4F2D4CFD5C45F6CC63F95C45F6BA
S214444840CB63C5F3801CFE5C45F6CD63F85C45F649
S214444850CE63FA5CEB0943EA4C0345F6C96C42EA7C
S214444860002217F80CC0C2F3090243EA8C03C5F3CE
S214444870401C43EA8C23C5F3001C43EACC23C1F313
S214444880400C43EA0C3345F6C86C17F80C7043EA00
S2144448904733C6F30017760943EA475343EA865339
S2144448A0C0F30116800943EA4663C5F3400605F0A3
S2144448B0010543EAC66343EA0573D4F82C5105F070
S2144448C060452B43C4F82C3101F0010342EA8322AD
S2144448D042EAC020C1F30012890940EA423040EA65
S2144448E08131A4F83011F0BD58874020D083402051
S2144448F0284845F6C86345F6CE622749F0B5C35AFC
S21444490045F6CA65845C45F6CD625BBA455D825C15
S214444910A709A1F8343145F6CB6347EA820745F642
S214444920CF62C65C45F6CC63825CC35CB009B1F822
S21444493036C142EA042240EA8500C6F3810543EACA
S2144449400623C6F3011640EA8520144DC3F3090333
S2144449500CEA050C43EA862340EA0C0043EA073394
S214444960A1F83601C4F38100C4F3011443EA80532A
S214444970D1F8380100F07F400343C1F83831C2F320
S2144449800903B1F83C2143EA842315402B43A1F89C
S2144449903C31F0BD58874020D083402000F0FFFFD4
S2144449A01D4945F6C8631D48F0B5CB5A45F6CA645A
S2144449B05BBA0E5DA0F8403145F6CB63CA5C45F65B
S2144449C0CD63CD5CC2F3810445F6CC632F09CB5C42
S2144449D044EA870445F6CE6743EA0223C95D41EAC2
S2144449E0052144EA8111A0F84211C3F30901C2F338
S2144449F0001343EA41039109C2F3401243EAC62333
S214444A0043EAC14343EA4253D0F84421920D920507
S214444A101343C0F84431F0BD58874020D08340202B
S214444A20184845F6C863184930B5C35A5BBAA1F866
S214444A30483145F6CC63C55C45F6CA63C45C45F666
S214444A40CB63C35C43EA042245F6CD63E409C35C06
S214444A50B1F84A0143EA0523ED09C3F3090343EADF
S214444A6085230A4D28400343A1F84A31C2F309037B
S214444A70B1F84C2143EA84232A401343A1F84C312D
S214444A8030BD00BF58874020D083402000F8FFFF49
S214444A901D4A45F6C8631D4870B5D35A5BBAA0F89C
S214444AA0503145F6CA63D45C45F6CC63D55C45F6CE
S214444AB0CB63D15C2B09C5F3C00543EA011145F627
S214444AC0CE63D65C45F6CD63D35CDB0043EA561230
S214444AD0C4F3400343EA450304F00105A40843EA4B
S214444AE0850343EAC403B0F8524104F47E442343A6
S214444AF0A0F8523141EA0233D0F85421D20DD205FF
S214444B001343C0F8543170BD58874020D0834020AA
S214444B101B4945F6C9631B4830B5CB5C80F8583111
S214444B2045F6CA63CA5C45F6CD63CD5C45F6CC63B0
S214444B30CC5C45F6C863C95C93091B0243EA8123EF
S214444B40C2F3800143EA8143C2F3C001C2F3401278
S214444B5043EAC143D0F8581143EA02532A0905F000
S214444B600F0543EA4253084A43EA45630A4013435F
S214444B70C0F85831230943EA041480F85C4130BD38
S214444B8058874020D0834020FF0000E030B545F6EB
S214444B90C863304C3049E35A5BBAA1F8203145F635
S214444BA0CE63E05C45F6CF63E25C45F6CA63E55CFB
S214444BB000F0030343EA8503C0F3800543EA8523F4
S214444BC0C2F3800543EAC523850943EA0533B1F8B1
S214444BD0225105F440452B43C2F3C005A1F82231C7
S214444BE045F6CB63E35C81F82431C0F3C0031B0273
S214444BF043EA452302F0030543EA852345F6CC659C
S214444C00655D43EA0533C0F30015C0F3401043EA3C
S214444C100553C2F3001543EA45539509120943EA7E
S214444C208553D1F8245102F0020225F47F0502434D
S214444C3025F47F452B43C1F8243145F6CD63E35C28
S214444C4081F8273191F8283123F003031A4381F879
S214444C50282130BD58874020D0834020074945F658
S214444C60C863074ACB581BBAC2F8683145F6CC63CA
S214444C70CB581BBAC2F86C31704700BF58874020E7
S214444C80D08340200C4947F664630C48CA5C47F618
S214444C906563CB5C43EA022247F66263CB5C03F06F
S214444CA00F0343EA0213D0F87021120D1205134382
S214444CB0C0F87031704700BF58874020D0834020EA
S214444CC0064A47F66263D15C47F66363D35C044A9C
S214444CD043EA0123A2F87431704700BF5887402046
S214444CE0D08340200C4949F6FC530C48CA5C49F62C
S214444CF0FD53CB5C43EA022249F6FA53CB5C03F0FD
S214444D000F0343EA0213D0F87821120D1205134319
S214444D10C0F87831704700BF58874020D083402081
S214444D20064A49F6FA53D15C49F6FB53D35C044A27
S214444D3043EA0123A2F87C31704700BF58874020DD
S214444D40D083402010B51A4C20890BF0A7FC194993
S214444D500BF0F8FC184BA27B1860184B60891A605D
S214444D600BF09CFC16490BF0EDFC16490BF0E0FBEF
S214444D700BF03AF80CA3D3E900230AF0D5FE0BF067
S214444D8083FB114B114A1860E37BA08903F00F03A1
S214444D9013600BF083FC0E490BF0D4FC0D490BF06A
S214444DA0C7FB0D4B186010BDC3F5285C8FC2D53FBA
S214444DB0D0834020CDCCCC3DB41F40209C1F402007
S214444DC00AD7A33C00C02344A81F4020981F402075
S214444DD0ACC52737ACC5A73EA01F4020124A13498E
S214444DE0137D03F003000860C3F3830010499B0956
S214444DF0086010490B60537D0F49C3F341000860B7
S214444E00C3F3C1000D4903F0010308700C490B605D
S214444E1053690C49C3F347330B60D38A0A4AC3F336
S214444E2047131360704700BFD0834020881F40203C
S214444E30841F4020801F4020781F4020741F40203D
S214444E407C1F4020681F4020701F4020074B084AA4
S214444E501B7CC3F300011170C3F34001054AC3F33E
S214444E6080031170044A1370704700BFD0834020FB
S214444E70661F4020651F4020641F4020FFF7E6BFA2
S214444E8008B5FFF7E3FFBDE80840FCF7E5BC10B5FE
S214444E90124CB4F825000BF001FC11490BF052FCFF
S214444EA0104B1860208D0BF0F9FB0F490BF04AFCB1
S214444EB00E490BF03DFB0E4B1860608DC0F30D00A1
S214444EC00BF0ECFB08490BF03DFC0A4B0A4A186011
S214444ED094F82B30C3F38013137010BDD083402056
S214444EE0CDCCCC3D601F40200AD7233C000048432D
S214444EF05C1F4020581F4020541F4020164A174924
S214444F0092F82C3003F003000860C3F38100144980
S214444F100860C3F3011013499B09086012490B60EB
S214444F2092F82D30114903F003000860C3F3810062
S214444F300F490860C3F301100E499B0908600E49E7
S214444F400B6092F82E300D4A03F00301C3F381033D
S214444F5011600B4A13607047D08340207C1A40206F
S214444F60781A4020741A4020701A40206C1A402048
S214444F70681A4020641A4020601A40205C1A402078
S214444F80581A402010B5194C208E0BF087FB184950
S214444F900BF0D8FB17490BF0CBFA174B174A18609F
S214444FA094F83230A08E03F00F011B091160144AA6
S214444FB0136094F83330134A323B13600BF06EFBA5
S214444FC011490BF0BFFB11490BF0B2FA104B114AD2
S214444FD0186094F8363003F00F011B0911600E4A2E
S214444FE0136094F837200D4B1A6010BDD0834020D0
S214444FF00AD7A33B0AD72343501F40204C1F4020C8
S214445000481F4020441F40200AD7A33AF8D32342DF
S214445010401F40203C1F4020381F4020341F402063
S21444502010B5194C208F0BF039FB18490BF08AFB4E
S21444503017490BF07DFA174B174A186094F83A3024
S214445040A08F03F00F011B091160144A136094F8F3
S2144450503B20134B1A600BF021FB12490BF072FBFA
S21444506011490BF065FA114B114A186094F83E301A
S21444507003F00F011B0911600E4A136094F83F2099
S2144450800D4B1A6010BD00BFD08340200AD7A33B07
S2144450900AD72343301F40202C1F4020281F40207F
S2144450A0241F40200AD7A33AF8D32342201F402087
S2144450B01C1F4020181F4020141F402010B5184CB9
S2144450C0B4F840000BF0EAFA16490BF03BFB1649DD
S2144450D00BF02EFA154B164A186094F84230B4F882
S2144450E0440003F00F011B091160124A13600BF0D1
S2144450F0D5FA11490BF026FB10490BF019FA104B60
S214445100104A186094F8463003F00F011B091160EA
S2144451100D4A136094F847200C4B1A6010BD00BF2C
S214445120D08340200AD7A33B0AD72343101F4020EE
S2144451300C1F4020081F40200AD7A33AF8D3234226
S214445140041F4020001F4020FC1E4020F81E402024
S21444515010B53E4C3E4A94F84830B4F8480003F044
S2144451600101C0F3C7101160C3F34001394A11600E
S214445170C3F38201384AC3F341131160374A1360BC
S2144451800BF08CFA36490BF0DDFA0BF0A1FC354BEC
S2144451901860A06CC0F3C7300BF080FA30490BF0AF
S2144451A0D1FA0BF095FC304B1860B4F84A00C0F3C3
S2144451B0C7100BF073FA2D490BF0BAF90BF088FCC4
S2144451C02B4B94F84C2018602A4B1A6094F84D30B8
S2144451D0294A03F001011160C3F34001274A1160D4
S2144451E0C3F38001264A1160C3F3C001254A116007
S2144451F0C3F30011244A1160C3F34011234A1160DB
S214445200C3F38011224ADB091160224A136094F8E2
S2144452104E30214A03F001011160C3F340011F4A96
S2144452201160C3F380011E4A1160C3F3C0011D4AD6
S2144452301160C3F300111C4A1160C3F340111B4AAA
S214445240C3F3801311601A4A136010BDD083402004
S214445250F41E4020F01E4020EC1E4020E81E402055
S2144452600AD7233CE41E4020E01E40200000204293
S214445270DC1E4020D81E4020D41E4020D01E402095
S214445280CC1E4020C81E4020C41E4020C01E4020C5
S214445290BC1E4020B81E4020B41E4020B01E4020F5
S2144452A0AC1E4020A81E4020A41E4020A01E402025
S2144452B09C1E402038B5264D264B95F8504004F0A9
S2144452C00102C4F302101A60C4F34002224B1A606F
S2144452D0C4F38002214B1A60C4F3C002204BE40995
S2144452E01A600BF0D7F91F4B1F4A18601F4B286DE6
S2144452F01C6095F85130C0F3473003F00F01C3F3F8
S2144453000013323811601A4A13600BF0C7F9194B70
S2144453101860B5F85200C0F3471032380BF0BEF9A7
S214445320154B1860B5F85400A0F500400BF0B6F9DC
S214445330124B1860B5F856000BF0B0F910490BF054
S21444534001FA10490BF0F4F80F4B186038BD00BF53
S214445350D0834020981E4020941E4020901E40201B
S2144453608C1E4020881E4020801E4020841E4020E4
S2144453707C1E4020781E4020741E4020701E402014
S2144453800AD7233C000048436C1E40207047304BED
S214445390304A10B593F86140C4F381011170C4F3E8
S2144453A001112D4A1170C4F301012C4AA40911704D
S2144453B093F860202A49C2F381100870C2F30110A2
S2144453C028490870C2F381002749C2F301020870D5
S2144453D026490A7093F865202549C2F38100C2F332
S2144453E00102087023490A7093F866202249C2F3E2
S2144453F003120A7093F867202049C2F301020A7028
S21444540093F862201E4902F003000860C2F381004C
S2144454101C490860C2F301101B49920908601B49E5
S2144454200A6093F863201A4902F00300C2F381022B
S2144454300860184993F864000A700BF02FF916496F
S2144454400BF080F9154B1860154B1C6010BD00BF5F
S214445450D0834020681E4020671E4020661E4020A1
S214445460651E4020641E4020631E4020621E40206D
S214445470611E4020601E402070184020281E402098
S214445480581E4020541E4020501E40204C1E402093
S214445490481E402069184020CDCCCC3D401E4020BC
S2144454A05C1E4020264A274992F8683003F00700DD
S2144454B00860C3F3C00024490860C3F300102349BE
S2144454C00870C3F340102249C3F38013087021497F
S2144454D00B70B2F868302049C3F3C7130B60936E61
S2144454E01E49C3F3C7330B60B2F86A301C49C3F392
S2144454F0C1130B6092F86B301A49C3F3410008603D
S214445500C3F3C1001849C3F34113086017490B603D
S21444551092F86C30164A03F003011160C3F380011D
S214445520144A1160C3F3C001134A1160C3F3001157
S214445530124AC3F340131160114A1360704700BF08
S214445540D0834020241E4020201E40201E1E402083
S2144455501D1E40201C1E4020181E4020141E4020A5
S214445560101E40200C1E4020081E4020041E4020D2
S214445570001E4020FC1D4020F81D4020F41D402005
S214445580F01D402010B5194C194A94F8703094F820
S2144455907200C3F38101C3F301131170154A1370EB
S2144455A094F87130144AC3F301011170C3F38101B6
S2144455B0124AC3F381131170114A13700BF06AF840
S2144455C0104B186094F873000BF064F80E4B94F884
S2144455D0742018600D4B1A7094F875200C4B1A7092
S2144455E094F876200B4B1A7010BD00BFD083402031
S2144455F0E61D4020D51D4020E51D4020D41D4020FA
S214445600E41D4020E01D4020DC1D4020D81D4020E5
S214445610D71D4020D61D402010B50C4CB4F87A0057
S2144456200BF03CF80A490BF08DF80A4B1860B4F8B6
S21444563078000BF033F806490BF084F8064BB4F8C0
S2144456407C201860054B1A8010BD00BFD0834020D4
S214445650CDCCCC3DD01D4020CC1D4020CA1D402082
S214445660084B0949B3F88220C2F387020A70D3F87C
S21444567080200649C2F309220A8093F88020044B0E
S2144456801A707047D0834020C81D4020C61D402055
S214445690C41D402010B5124C124B94F88820B4F820
S2144456A089001A600AF0FAFF0F490BF04BF80F49CD
S2144456B00AF03EFF0E4B1860B4F88C000AF0EEFF7A
S2144456C00C490BF03FF80C4B0C4A186094F88E309B
S2144456D003F00F011B091160094A136010BD00BF97
S2144456E0D0834020C01D4020ACC52737ACC5A73E5C
S2144456F0BC1D4020CDCCCC3DB81D4020B41D402020
S214445700B01D402010B5114CB4F890000AF0C6FF06
S2144457100F490BF017F80F490AF00AFF0E4B1860B2
S214445720B4F892000AF0BAFF09490BF00BF809499D
S2144457300AF0FEFE094B0A4A186094F8943003F0C7
S2144457400F011B091160074A136010BDD083402027
S2144457500AD7A33C00C02344AC1D4020A81D4020CB
S214445760A41D4020A01D4020114A124992F89830AA
S21444577003F003000860C3F381000F490860C3F3D5
S21444578001100E499B0908600D490B6092F8993048
S2144457900C4903F00100C3F3430308600A490B6055
S2144457A0D2F89830094AC3F343331360704700BFB6
S2144457B0D08340209C1D4020981D4020941D4020AE
S2144457C0901D40208C1D4020881D4020841D402074
S2144457D0194A1A4992F89C3003F003000860C3F350
S2144457E0810017490860C3F3011016499B090860F5
S2144457F015490B6092F89D30144903F00300086085
S214445800C3F3810012490860C3F3011011499B0990
S214445810086011490B6092F89E30104903F003006B
S214445820C3F3810308600E490B60D2F8A0300D4ADA
S214445830C3F3833313607047D0834020801D4020D9
S2144458407C1D4020781D4020741D4020701D402043
S2144458506C1D4020681D4020641D4020601D402073
S2144458605C1D4020581D402010B50E4C0E4B94F83D
S214445870A70094F8A42000F01F001A6000EB8000F4
S2144458800AF00CFF094B1860B4F8A8000AF006FFAB
S21444589007490AF057FF07490AF04AFE064B1860C4
S2144458A010BD00BFD0834020541D40203C1D4020E6
S2144458B0CDCC4C3D00C0CC44381D402010B50C4CDB
S2144458C0B4F8AE000AF0EAFE0A490AF03BFF0A4979
S2144458D00AF02EFE094B1860D4F8B000C0F34F000F
S2144458E0A0F5FF407F380AF0D9FE054B186010BD7E
S2144458F0D08340200AD7A33C00C02344281D402020
S214445900201D402010B50D4CB4F8B600C0F30D0071
S2144459100AF0C4FE4FF07A510AF014FF084B1860A0
S214445920B4F8B800C0F30D000AF0B8FE4FF07A5150
S2144459300AF008FF034B186010BD00BFD083402018
S214445940181D4020141D402070470B4A0B49B2F8DE
S214445950CC0008B5B2F8C830C0F30900C3F38703D7
S2144459600B700AF09BFE06490AF0ECFE05490AF065
S214445970DFFD054B186008BDD0834020101D402035
S214445980CDCCCC3D9A994C420C1D402010B5174CBA
S214445990B4F8D200C0F309000AF080FE14490AF0B5
S2144459A0D1FE144B1860B4F8D400C0F309000AF0D2
S2144459B075FE0F490AF0C6FE0F4B1860D4F8D400A3
S2144459C0C0F309300AF06AFE09490AF0BBFE0B4BE5
S2144459D01860B4F8D800C0F309000AF05FFE044922
S2144459E00AF0B0FE064B186010BD00BFD0834020BE
S2144459F0CDCCCC3D081D4020041D4020001D402039
S214445A00FC1C402038B5154DB5F8DE0080090AF078
S214445A1045FE13490AF096FE12490AF089FDB5F888
S214445A20E040114BC4F34904186020460AF036FEA1
S214445A300E490AF087FE0E4B1860D5F8E000C0F316
S214445A40CF200AF02BFE0B490AF07CFE0A4B186066
S214445A500A4B1C600A4B1C6038BD00BFD0834020F4
S214445A60CDCC4C3D66667241F81C40209A99193E4E
S214445A70F41C40200AD7233CF01C40207C1C4020C9
S214445A801C1B402010B5164CB4F8E600C0F30900C1
S214445A900AF004FE13490AF055FE134B1860B4F896
S214445AA0E800C0F309000AF0F9FD0E490AF04AFE80
S214445AB00E4B1860D4F8E800C0F3C9200AF0EEFD97
S214445AC008490AF03FFE0A4B1860B4F8EA00800919
S214445AD00AF0E4FD03490AF035FE064B186010BD93
S214445AE0D08340209A99193EEC1C4020E81C402064
S214445AF0E41C4020E01C402010B5134CB4F8F200DF
S214445B00C0F3C5000AF0CAFD10490AF01BFE10494E
S214445B100AF00EFD0F4B1860B4F8F400C0F30B0007
S214445B200AF0BCFD0C490AF00DFE0C4B1860D4F884
S214445B30F400C0F30A300AF0B1FD04490AF002FE4C
S214445B40074B186010BD00BFD0834020CDCCCC3D61
S214445B50CDCC4C40DC1C40200AD7233CD81C4020EB
S214445B60D41C40207047704710B50E4C0E4B94F82A
S214445B70130194F8102100F01F001A6000EB800017
S214445B800AF08CFD094B1860B4F814010AF086FD3F
S214445B9007490AF0D7FD07490AF0CAFC064B1860C5
S214445BA010BD00BFD0834020D01C4020CC1C4020D9
S214445BB0CDCC4C3D00C0CC44C81C402010B50C4C49
S214445BC0B4F81A010AF06AFD0A490AF0BBFD0A490C
S214445BD00AF0AEFC094B1860D4F81C01C0F34F0021
S214445BE0A0F5FF407F380AF059FD054B186010BDFC
S214445BF0D08340200AD7A33C00C02344C41C402082
S214445C00C01C402070470B4A0B49B2F8300108B517
S214445C10B2F82C31C0F30900C3F387030B700AF0C3
S214445C203DFD06490AF08EFD05490AF081FC054B08
S214445C30186008BDD08340209C1C4020CDCCCC3D71
S214445C409A994C42981C402010B5174CB4F836012B
S214445C50C0F309000AF022FD14490AF073FD144B00
S214445C601860B4F83801C0F309000AF017FD0F496C
S214445C700AF068FD0F4B1860D4F83801C0F30930B9
S214445C800AF00CFD09490AF05DFD0B4B1860B4F8A8
S214445C903C01C0F309000AF001FD04490AF052FD34
S214445CA0064B186010BD00BFD0834020CDCCCC3D01
S214445CB0941C4020901C40208C1C4020881C402073
S214445CC010B5134CB4F8420180090AF0E7FC1149B8
S214445CD00AF038FD10490AF02BFC104B1860B4F853
S214445CE04401C0F349000AF0D9FC0D490AF02AFDE4
S214445CF00AF0EEFE0B4B1860D4F84401C0F3C720FC
S214445D000AF0CCFC08490AF01DFD084B186010BD8B
S214445D10D0834020CDCC4C3D66667241BC1C4020AE
S214445D209A99193EB41C40200AD7233CB81C4020FC
S214445D3010B50C4CB4F84A01C0F309000AF0AEFCA6
S214445D4009490AF0FFFC094B1860B4F84C01C0F34B
S214445D5009000AF0A3FC04490AF0F4FC044B18605A
S214445D6010BD00BFD08340209A99193EB01C4020F5
S214445D70AC1C402008B5FEF7E5FFFFF72FF8FFF709
S214445D8086F8FFF7BBF8FFF7E3F9FFF793FAFFF758
S214445D90FEFAFFF787FBFFF7F5FBFFF73DFCFFF73F
S214445DA05FFCFFF7EFF8FFF73BF9FFF787F9FFF7DC
S214445DB071FCFFF7A7FCFFF7D7FCFFF709FDFFF7D9
S214445DC0E5FDFFF71FFEFFF75DFEFFF73DFFFFF71C
S214445DD077FFBDE80840FFF7ABBF10B5124CB4F8E8
S214445DE05201C0F3C5000AF059FC10490AF0AAFC57
S214445DF00F490AF09DFB0F4B1860B4F85401C0F3EA
S214445E000B000AF04BFC0C490AF09CFC0B4B186048
S214445E10D4F85401C0F30A300AF040FC03490AF0AF
S214445E2091FC074B186010BDD0834020CDCCCC3DB0
S214445E30CDCC4C40A81C40200AD7233CA41C402070
S214445E40A01C402008B5FFF757FEBDE80840FFF702
S214445E50C4BF7047704708B5084BD3F87001C0F309
S214445E600F100AF01BFC06490AF06CFC05490AF0C0
S214445E705FFB0AF02DFE044B186008BDD08340201B
S214445E80CDCC4C3D00C0CC44C41B402008B5084B88
S214445E90B3F874010AF002FC06490AF053FC0649BA
S214445EA00AF046FB0AF014FE044B186008BD00BF17
S214445EB0D08340200AD7A33C00C02344C81B4020BC
S214445EC008B5094BD3F87801C0F30F100AF0E6FB87
S214445ED006490AF037FC06490AF02AFB0AF0F8FDA0
S214445EE0044B186008BD00BFD0834020CDCC4C3D49
S214445EF000C0CC44B81B402008B5084BB3F87C011E
S214445F000AF0CCFB06490AF01DFC06490AF010FBD1
S214445F100AF0DEFD044B186008BD00BFD083402065
S214445F200AD7A33C00C02344B81B402008B5FFF75B
S214445F309BFCFFF7C3FCFFF7E5FCFFF706FDFFF706
S214445F4013FEFFF73BFEFFF75EFEFFF784FFFFF707
S214445F509DFFFFF7B5FFBDE80840FFF7CDBF1A4BDE
S214445F60186810B5C830194C0AF094FB18490AF062
S214445F709DFC09F039FF0EF03FFF0AF065FA154B19
S214445F801549A4F8800118680AF0D4FA13490AF0AF
S214445F908DFC09F029FF0EF02FFF0AF055FA104B3E
S214445FA0A4F882011B68A4F884310E4B186809F0E3
S214445FB01BFF0EF021FF0AF047FA0B4B84F88601CC
S214445FC01B6884F8873110BD841C4020D083402051
S214445FD0CDCCCC3D801C402000C023440AD7A33CF3
S214445FE07C1C4020781C4020741C40202F4B304A98
S214445FF03049126810B5304C12021B7802F44072D5
S21444600084F88C312D4B1B689B0203F48063134346
S2144460102B4A1268D20202F4C0521343294A126829
S214446020520302F4C0421343274A1268D20302F4CE
S214446030C0321343D4F88C2122F4FF3222F4807207
S2144460401343C4F88C31214B18680AF073FA20497C
S2144460500AF02CFC09F0C8FE0EF0CEFE0AF0F4F965
S2144460601C4BA4F8920118680AF014FB11490AF074
S21444607061FA17490AF01AFC09F0B6FE0EF0BCFEA7
S2144460800AF0E2F9144B154A1B781268DB00A4F8B0
S214446090900102F0070203F00803134394F8942196
S2144460A022F00F02134384F8943110BDD61D4020CD
S2144460B0641C4020ACC5A73ED0834020601C4020D2
S2144460C05C1C4020581C4020541C4020501C40203F
S2144460D0ACC527374C1C40201E1E4020241E4020A2
S2144460E0184B1949186810B50AF0E0FB174C09F02C
S2144460F07BFE0EF081FE0AF0A7F9154B1249A4F870
S214446100980118680AF0D2FB09F06EFE0EF074FE91
S2144461100AF09AF90F4B0C49A4F89A0118680AF049
S214446120C5FB09F061FE0EF067FE0AF08DF90A4BD6
S214446130A4F89C011B7884F89F31084B1B7884F89C
S2144461409E3110BDCC1D4020CDCCCC3DD0834020CC
S214446150D01D4020401E4020C81D4020C41D402065
S214446160174B184A1B7812785B0002F0010203F0C2
S21444617002031343144A1278920002F004021343B3
S214446180124A1278D20002F008021343104A1278D8
S214446190120102F0100213430E4A1278520102F022
S2144461A0200213430C4A1278920102F04002134331
S2144461B00A4A127843EAC213094A82F8F031704711
S2144461C0291C40202A1C4020281C4020271C4020F4
S2144461D0261C4020251C4020241C40207C174020A0
S2144461E0D083402038B5254B254D1968254B186873
S2144461F00AF0A0F9244B0446244918680AF09AF990
S21444620023490AF053FB09F0EFFD0EF0F5FD0AF0C2
S2144462101BF9204B2049A5F8F40118680AF08AF9BE
S2144462201E490AF043FB09F0DFFD0EF0E5FD0AF0D7
S2144462300BF91B49A5F8F60120460AF037FB09F08E
S214446240D3FD0EF0D9FD0AF0FFF8164BA5F8F80179
S21444625018880AF023FA14490AF028FB09F0C4FD0A
S2144462600EF0CAFD114B1C780AF0EEF8C0F30D0090
S214446270A4030443A5F8FA4138BD00BFA017402044
S214446280D0834020B41F4020A41740200000484339
S2144462900AD7233C9C17402000C023440AD7A33C7B
S2144462A0CDCCCC3D7A174020CDCC4C3E79174020FF
S2144462B01C4B1D49186810B50AF0F8FA1B4C09F037
S2144462C093FD0EF099FD0AF0BFF8194BA4F8A0010F
S2144462D0186809F089FD0EF08FFD0AF0B5F8154BE5
S2144462E01549A4F8A20118680AF024F913490AF0DB
S2144462F0DDFA09F079FD0EF07FFD0AF0A5F8104BA3
S2144463001049A4F8A40118680AF014F90E490AF0D2
S214446310CDFA09F069FD0EF06FFD0AF095F8A4F881
S214446320A60110BDAC1F4020CDCCCC3DD083402030
S214446330B8194020A418402000C023440AD7A33CE0
S2144463405C1B4020000048430AD7233C114B1249AB
S214446350186810B50AF0AAFA104C09F045FD0EF07C
S2144463604BFD0AF071F80E4B0E491B78A4F8A801B1
S214446370A4F8AA310C4B18680AF0DCF80B490AF06A
S21444638095FA09F031FD0EF037FD0AF05DF8A4F8F1
S214446390AC0110BD08194020CDCCCC3DD083402064
S2144463A01219402000C023448C1840200AD7A33C2E
S2144463B0184B1949186810B50AF0BCF817490AF082
S2144463C075FA174C09F010FD0EF016FD0AF03CF86D
S2144463D0144B1549A4F8B00118680AF0ABF81349F1
S2144463E00AF064FA09F000FD0EF006FD0AF02CF8F7
S2144463F00F4BA4F8B2011B6884F8B4310D4B1A68ED
S2144464000D4B1B6803F00F0343EA021384F8B531BF
S21444641010BD00BF281D402000C023440AD7A33C1B
S214446420D0834020381D402000C0CC44CDCC4C3DC9
S2144464302C1C4020DC1B4020E01B4020164B1749F8
S214446440186810B50AF076F815490AF02FFA154C74
S21444645009F0CAFC0EF0D0FC09F0F6FF124B1349C3
S214446460A4F8B80118680AF065F811490AF01EFA4B
S21444647009F0BAFC0EF0C0FC09F0E6FF0D4BA4F898
S214446480BA011A680C4B1B6803F00F0343EA021365
S21444649084F8BC3110BD00BFC41C402000C0234457
S2144464A00AD7A33CD0834020C81C402000C0CC441C
S2144464B0CDCC4C3DCC1B4020D01B4020174B1868FD
S2144464C010B500F28F20164C0AF0E4F815490AF08D
S2144464D0EDF909F089FC0EF08FFC09F0B5FF124B7C
S2144464E0A4F8C001186800F266600AF0D3F80F49B1
S2144464F00AF0DCF909F078FC0EF07EFC09F0A4FF03
S2144465000B4BA4F8C2011A680A4B1B6803F00F032E
S21444651043EA021384F8C43110BD00BFC81B4020B0
S214446520D08340200AD7A33CC41B4020CDCC4C3D4E
S214446530BC1B4020C01B4020174B186810B500F207
S2144465408F20164C0AF0A6F815490AF0AFF909F060
S2144465504BFC0EF051FC09F077FF124BA4F8C8012F
S214446560186800F266600AF095F80F490AF09EF93A
S21444657009F03AFC0EF040FC09F066FF0B4BA4F819
S214446580CA011A680A4B1B6803F00F0343EA021356
S21444659084F8CC3110BD00BFB81B4020D0834020C7
S2144465A00AD7A33CB41B4020CDCC4C3DAC1B40206A
S2144465B0B01B40200A4A0B4B126883F8E8210A4A6B
S2144465C0126883F8E921094A126883F8EA21084ADE
S2144465D0126883F8EB21074A1268C3F8EC21704727
S2144465E0A81B4020D0834020A41B4020A01B402052
S2144465F09C1B4020981B40202B4B2C4930B51D78C3
S2144466002B4B05F003051C782A4B04F0030418783A
S214446610294B00F003001B8881F8D431274B1A68B5
S214446620274B92001B6802F00C0203F003031A4344
S214446630244B1B681B0103F030031A43224B1B6890
S2144466409B01DBB21A43214B1B681B0203F44073C5
S2144466501A431F4B1B689B0203F440631A431D4BAB
S2144466601B681B0303F440531A431B4B1B689B03D2
S2144466709BB21A43194B1B681B0403F440331A435A
S214446680174B1B689B0403F440231343D1F8D021D3
S21444669043EA055302F07C4243EA845343EA0063E8
S2144466A01343C1F8D03130BD2A1B4020D08340204C
S2144466B02B1B40202C1B4020281B4020901B402096
S2144466C0941B40208C1B4020881B4020841B402069
S2144466D0801B40207C1B4020781B4020741B40209D
S2144466E0701B4020124B13491B7803F00302124BD5
S2144466F01B7803F0030343EA8203104A127802F03D
S214446700030243EA02130E4A127802F0030243EAF3
S21444671082130C4A127802F0030243EA0223B1F8C9
S214446720D82102F47C421343A1F8D831704700BF05
S2144467306B1B4020D08340206C1B40206A1B4020AB
S214446740691B4020681B4020094B0A491A680A4BBB
S21444675002F001021B6803F0030343EA820391F844
S214446760E42122F00702134381F8E431704700BF66
S214446770601B4020D0834020641B402038B5344BF7
S214446780344D1868C83009F085FF33490AF08EF84E
S21444679009F02AFB0EF030FB304B1C68304B64008B
S2144467A01B6804F0020403F001031C432D4B1B68D2
S2144467B09B0003F004031C432B4B1B68DB0003F0D5
S2144467C008031C43294B1B681B01DBB21C43284BA4
S2144467D01B681B0203F440731C43264B1B689B0236
S2144467E003F4E0531C43244B1B685B0303F4C0438D
S2144467F01C4309F029FE214B214903EAC0331C43BC
S214446800D5F8DC3103F000431C431E4BC5F8DC418D
S214446810186809F08FFE10490AF048F809F0E4FABF
S2144468200EF0EAFA09F010FE174B1549A5F8E001F8
S214446830186809F07FFE08490AF038F809F0D4FAD7
S2144468400EF0DAFA09F000FEA5F8E20138BD00BF02
S214446850341B4020D08340200AD7233C501B402082
S214446860541B40204C1B4020481B4020441B4020C7
S214446870401B40203C1B4020381B40200080FF7FAC
S21444688000004843301B40205C1B4020274B2849CF
S214446890186810B509F04EFE26490AF007F8264C4B
S2144468A009F0A2FA0EF0A8FA09F0CEFD234B2449CB
S2144468B0A4F85002186809F03DFE224909F0F6FF94
S2144468C009F092FA0EF098FA09F0BEFD1E4BA4F8B1
S2144468D052021B68A4F854321C4B1A681C4B02F034
S2144468E003021B6803F0010343EA4203194A126891
S2144468F002F0030243EAC203174A126802F0010296
S21444690043EA4213154A126802F00F0243EA82131E
S214446910134A126802F00F0243EA8223B4F856225E
S21444692002F440421343A4F8563210BD6C1E402075
S214446930000048430AD7233CD0834020281D4020EB
S21444694000C023440AD7A33C1C1B40205C1C4020A8
S214446950141B4020541C4020081B4020041B40208D
S214446960001B4020244B4FF08E41244A1B6812687B
S2144469701B0102F00F02DBB21343214A12681202D3
S21444698002F4706213431F4A1268120302F48052E0
S21444699013431D4A1268520302F4C04213431B4A6F
S2144469A01268D20302F4C0321343194A12685204DE
S2144469B010B502F0FF72174C1343D4F8582202F075
S2144469C07E421343C4F85832134B186809F0B2FD9C
S2144469D009F00AFA0EF010FA09F036FD0F4BA4F847
S2144469E05C021A680E4B1B6803F00F0343EA02135B
S2144469F084F85E3210BD00BFF81A4020FC1A4020CE
S214446A00F41A4020F01A4020581C4020E81A40202F
S214446A10181E4020D0834020701E4020E01A40209C
S214446A20E41A4020144B10B5186809F0DDF9134CED
S214446A300EF0E2F909F008FD114B84F860021B6879
S214446A4084F861320F4B1B68A4F862320E4B186808
S214446A5009F0CAF90EF0D0F909F0F6FC0B4BA4F88D
S214446A6064021A680A4B1B6803F00F0343EA0213D6
S214446A7084F8663210BD00BF781C4020D083402086
S214446A80741C40204C1C4020501C4020C81A4020F7
S214446A90CC1A40201C4A136DC3F3473382F898320D
S214446AA0B2F85230C3F3471382F89932B2F84A30F8
S214446AB0C3F3C71382F89A3292F8643082F89B3252
S214446AC0124B1968124B01F007011B6803F00103CF
S214446AD043EA41030F49097801F0010143EA0113EF
S214446AE00D49096801F00F0143EA41130B4909684F
S214446AF001F00F0143EA4123B2F89C1201F46041CD
S214446B000B43A2F89C327047D0834020241E40207A
S214446B10F01D40201E1E4020C41A4020C01A4020AB
S214446B20FFF7B8BF174B184A1B7812785B0002F081
S214446B30010203F002031343144A1278920002F04F
S214446B4004021343124A1278D20002F00802134396
S214446B50104A1278120102F0100213430E4A1278B9
S214446B60520102F0200213430C4A1278920102F0BA
S214446B70400213430A4A127843EAC213094A82F887
S214446B80A0327047291C40202A1C4020281C402044
S214446B90271C4020261C4020251C4020241C402026
S214446BA07C174020D0834020174B186810B500F25D
S214446BB08F20164C09F06EFD154909F077FE09F052
S214446BC013F90EF019F909F03FFC124BA4F8300201
S214446BD0186800F2666009F05DFD0F4909F066FE2C
S214446BE009F002F90EF008F909F02EFC0B4BA4F854
S214446BF032021A680A4B1B6803F00F0343EA021377
S214446C0084F8343210BD00BFBC1A4020D0834020E4
S214446C100AD7A33CB81A4020CDCC4C3DB01A4020ED
S214446C20B41A4020174B186810B500F28F20164C43
S214446C3009F030FD154909F039FE09F0D5F80EF093
S214446C40DBF809F001FC124BA4F83802186800F28D
S214446C50666009F01FFD0F4909F028FE09F0C4F8E4
S214446C600EF0CAF809F0F0FB0B4BA4F83A021A6887
S214446C700A4B1B6803F00F0343EA021384F83C32C2
S214446C8010BD00BFAC1A4020D08340200AD7A33C96
S214446C90A81A4020CDCC4C3DA01A4020A41A40202F
S214446CA0174B186810B500F28F20164C09F0F2FC0A
S214446CB0154909F0FBFD09F097F80EF09DF809F028
S214446CC0C3FB124BA4F84002186800F2666009F051
S214446CD0E1FC0F4909F0EAFD09F086F80EF08CF85D
S214446CE009F0B2FB0B4BA4F842021A680A4B1B6825
S214446CF003F00F0343EA021384F8443210BD00BF86
S214446D009C1A4020D08340200AD7A33C981A40209F
S214446D10CDCC4C3D901A4020941A4020174B18680E
S214446D2010B500F28F20164C09F0B4FC154909F052
S214446D30BDFD09F059F80EF05FF809F085FB124BDB
S214446D40A4F84802186800F2666009F0A3FC0F49EC
S214446D5009F0ACFD09F048F80EF04EF809F074FB63
S214446D600B4BA4F84A021A680A4B1B6803F00F033D
S214446D7043EA021384F84C3210BD00BF8C1A4020FC
S214446D80D08340200AD7A33C881A4020CDCC4C3D23
S214446D90801A4020841A40204C4B4FF084412DE901
S214446DA0F04FDFF864A187B01B788AF8C432484BAA
S214446DB01B788AF8C532474B186809F0BBFB4FF07E
S214446DC0834109F0BFFC09F00FF80EF015F8424B6A
S214446DD08046894618684FF0844109F0ABFB4FF073
S214446DE0834109F0AFFC08F0FFFF0EF005F83B4B7B
S214446DF006460F4693F800B0394B3A490BF0010B60
S214446E00186809F097FB384909F050FD08F0ECFF84
S214446E100DF0F2FF354B364A1B78CDE90001106879
S214446E203449059309F086FB334909F03FFD08F0E1
S214446E30DBFF0DF0E1FF314A1478314A04F00104D7
S214446E401578240305F00105CDE90201494640467C
S214446E5009F0FAFAC0F30900AD0239460543BAF818
S214446E60C60200F4784005433046AAF8C6524FEAB4
S214446E708B2509F0E9FAC0F3090BDDE9000109F0B6
S214446E80E3FA204A059B45EA0B0B02EAC02203F0CC
S214446E9001034BEA020BDAF8C8224BEAC35302F06A
S214446EA07F421343DDE90201CAF8C83209F0CCFA3E
S214446EB0C0F30B000443BAF8CC0200F46040044329
S214446EC0AAF8CC4207B0BDE8F08F00BF5D19402059
S214446ED05C19402058194020501940204C19402035
S214446EE04819402033336F410AD7233C4419402085
S214446EF040194020CDCCCC42CDCC4C3D3C19402012
S214446F005419402000F87F00D0834020124B1A8E3C
S214446F10C3F86822114A1168114A01F00F01126839
S214446F2002F00F0242EA011293F8331042EA0122B9
S214446F30A3F86C229A8EC3F870220A4A11680A4A49
S214446F40126802F00F0242EA011283F87422074ADA
S214446F50126883F875227047D0834020481F40202B
S214446F604C1F4020381F40203C1F4020341F4020E8
S214446F70114B1A8FC3F87822104A1168104A1268C7
S214446F8002F00F0242EA011283F87C220D4A12688C
S214446F9083F87D229A8FC3F880220B4A11680B4AE5
S214446FA0126802F00F0242EA011283F88422084A69
S214446FB0126883F885227047D0834020281F4020DB
S214446FC02C1F4020241F4020181F40201C1F4020F8
S214446FD0141F4020104BB3F84020C3F888220F4AB1
S214446FE011680F4A126802F00F0242EA011283F84F
S214446FF08C22B3F84420C3F890220A4A11680A4AFD
S214447000126802F00F0242EA011283F89422074AF9
S214447010126883F895227047D0834020081F40208A
S2144470200C1F4020FC1E4020001F4020F81E40201D
S214447030334B3449F0B51E78334B06F0030691F8CB
S21444704064201D78314B42EA062205F003051C688D
S2144470502F4B42EA8522240318682E4BA4B2000420
S2144470601B78224300F4702003F003072A4B104396
S2144470701B7803F0030343EA8703284F3F7807F05F
S214447080030743EA0713264F3F7807F0030743EA0C
S2144470908713244F3F7807F0030743EA0723224F1A
S2144470A03F7807F0030743EA8723204F3F7807F0EB
S2144470B0030743EA07331E4F3F68BF03BFB23B4351
S2144470C01C4F43EA06433F7843EA864307F00307E8
S2144470D043EA065343EA865343EA066343EA87632E
S2144470E0D1F80C7207F070473B43C1F80C32D1F824
S2144470F010321B0D1B051843C1F81002F0BD00BF2B
S214447100601E4020D0834020611E4020101A40203C
S2144471100C1A4020631E4020621E4020641E4020FD
S214447120651E4020661E4020681E4020671E402084
S2144471305C1E402069184020204B214A70B51C68CC
S214447140204BB2F8685004F00F04186892F8683080
S21444715005F4FF4592F86C1000F00F0003F07F032F
S2144471602B43956E05F4FF052B43B2F86A50C5F3DE
S214447170C11543EAC55392F86B50C5F3410643EA3A
S2144471804663C5F3C106C5F3411543EAC66343EAFD
S2144471904573D2F8145205F000452B43C2F8143216
S2144471A001F03F03B2F8181243EA841301F4404155
S2144471B043EA80230B43A2F8183270BDEC1D4020EE
S2144471C0D0834020E81D40201D4B1E4A1B68126891
S2144471D09B001D4902F0030203F00C0313431B4AB1
S2144471E01268120102F030021343194A12689201DF
S2144471F0D2B21343174A1268120202F4407213437F
S214447200154A1268920202F440621343134A126803
S214447210120302F440521343114A1268920302F4D2
S214447220703213430F4A1268920402F470121343E6
S214447230D1F82C22920D92051343C1F82C32704794
S214447240FC194020001A4020D0834020F8194020E2
S214447250F4194020F0194020EC194020E819402049
S214447260E4194020E01940201A4B1B49186810B511
S21444727009F01CFB194C08F0B7FD0DF0BDFD09F0F4
S214447280E3F8174B1449A4F81C02186809F00EFBDF
S21444729008F0AAFD0DF0B0FD09F0D6F8114BA4F89D
S2144472A01E02188809F0FAF90B4909F0FFFA08F0AB
S2144472B09BFD0DF0A1FD09F0C7F80B4BA4F8200286
S2144472C01A680A4B1B6803F00F0343EA021384F858
S2144472D0223210BDCC1D4020CDCCCC3DD0834020A6
S2144472E0D01D4020CA1D4020301E4020341E402061
S2144472F0134A92F8803010B582F82432114BD2F8F3
S21444730024421878B2F88230C3F38701D2F880302A
S214447310C3F309231B0243EA81430B49097801F06E
S2144473200F0143EA8163094921400B43C2F82432E2
S21444733092F8283260F3030382F8283210BD00BF67
S214447340D0834020DA194020DB194020FF0000C0DB
S214447350094B0A491A680A4B02F007021B6803F0F5
S214447360030343EA820391F8A42222F01F02134344
S21444737081F8A432704700BF5C1C4020D083402074
S214447380501B4020064B10B5064C186809F0A0FB6D
S214447390B4F8A83260F30903A4F8A83210BD00BFBD
S2144473A0781C4020D0834020094B0A4A1B78127828
S2144473B09B00094902F0030203F00C03134391F8BF
S2144473C0AC2222F00F02134381F8AC32704700BF60
S2144473D0D6194020D7194020D0834020044B054975
S2144473E093F8B022097861F3020283F8B02270471A
S2144473F0D0834020D5194020044B054993F8B42245
S214447400097861F3030283F8B4227047D08340209E
S214447410D4194020F8B53D4B3D4D1B783D4985F881
S214447420B8323D4B186809F041FA08F0DDFC0DF01F
S214447430E3FC09F009F8394A394B03EA402310685B
S214447440D5F8B822000200F4807003433548104053
S2144474500343C5F8B832344B1B7885F8BC32334BFB
S2144474601C68334B04F003041F68324B07F00107D3
S2144474701E68314B44EA870406F00106186809F092
S21444748009F94FF0814109F05DF909F021FB2B4AD7
S2144474902B4B44EAC606D5F8BC1203EA0023106810
S2144474A0284A800595F8C04200F4800024F00F0472
S2144474B003431068244A2643C005126800F40000BB
S2144474C085F8C0621206034302F0407213431F4A13
S2144474D01268920602F0406213431D4A126812076D
S2144474E002F0805213431B4A1268520702F00052BD
S2144474F01343194A1268920702F080421343174A0C
S2144475000A401343C5F8BC32F8BD00BF7C1940207E
S214447510D0834020CDCCCC3DAC194020B01940207F
S21444752000FEFF01FF0000FE7D1940208819402020
S2144475308419402080194020A8194020A4194020CE
S21444754000FF3F00A01940205C1C402098194020B2
S21444755094194020901940208C194020FF00008048
S214447560084A094B1278094983F8D022084A097810
S214447570127883F8D12293F8D22261F3000283F87A
S214447580D2227047C6194020D0834020C4194020D8
S214447590C5194020114B12491B6810B5114C84F88C
S2144475A0F032114B1B6884F8F132104B186808F01F
S2144475B0C1FF0F4909F07AF908F016FC0DF01CFCDF
S2144475C008F042FF0B4A94F8F4321278A4F8F20218
S2144475D062F3000384F8F43210BD00BFC0194020A3
S2144475E000C02344D0834020BC194020B819402012
S2144475F00AD7A33CB4194020F8B5204B204D186850
S21444760009F048F84FF0814109F09CF809F060FA17
S2144476101C4B04461F681C4BC4F30D0407F00107BB
S2144476201E681A4B44EA8734186844EAC63409F09C
S21444763031F84FF0814109F085F809F049FA144AC7
S214447640C0F30D03A5F8EC421068124A800300F418
S214447650804003431068104AC003126800F4FF00D9
S214447660D205034302F0FF421343D5F8E82202F062
S21444767000421343C5F8E832F8BD00BF68194020FD
S214447680D083402064194020601940207819402057
S21444769074194020701940206C1940200D4B0E4A36
S2144476A01B780E4982F8FC320D4B09781B7801F0A2
S2144476B0010182F8FD320B4B1B785B0003F002039A
S2144476C00B4392F8FE1221F003010B4382F8FE327C
S2144476D0704700BF3B194020D083402039194020D2
S2144476E03A194020381940200C4B0D4A1B680D4966
S2144476F082F8F8320C4B09781B6801F0030182F8D3
S214447700F9320A4B1B789B0003F00C030B430849E1
S214447710097843EA011382F8FA3270473419402054
S214447720D08340202F194020301940202E19402065
S2144477302D194020F8B5254B254C1B78254F84F849
S2144477400033254B1B7884F80133244B18783230A9
S21444775008F0A4FF014608F0EDFE09F0B9F9204907
S21444776084F802030E781F493F780D781E4907F0C7
S21444777001071E4B08781E491A78303009781D4B8D
S21444778049001B7801F03E01394394F8037327F00F
S2144477903F07394384F8031303F03F0102F01F0305
S2144477A006F00F0243EA411343EAC22305F03F02C0
S2144477B043EAC23300F03F0243EA4253D4F8042378
S2144477C002F078421343C4F80433F8BD2C19402021
S2144477D0D0834020291940202B1940202A194020C4
S2144477E025194020241940202319402027194020D9
S2144477F0281940202619402038B50C4B0C4C5D689F
S214447800284608F0F1FA0DF0F7FA08F01DFE09498B
S214447810C4F8E402284609F049F808F0E5FA0DF001
S214447820EBFA08F011FEC4F8E00238BD30464020BA
S214447830D0834020000008422DE9F74F374D384E9C
S214447840686809F045F986F80803A86809F040F91D
S214447850344986F80903686908F06CFE324909F031
S21444786025F809F035F98346A86909F031F92D4918
S2144478700446E86908F05EFE2B4909F017F8CBF396
S214447880090B09F025F98246286A09F021F92549A9
S2144478908146686A08F04EFE234909F007F809F065
S2144478A017F98046A86A09F013F91E4900F0010743
S2144478B0E86808F03FFE1C4908F0F8FF09F008F9AC
S2144478C0C0F309032869019309F002F9019B00F00B
S2144478D0010043EA8023B6F80A0300F478400343E1
S2144478E01248A6F80A33A30200EACA2A03F48063BD
S2144478F04FEA495043EA0B0300F4001043EA0A03F4
S214447900034343EA8853C6F80C3396F8103367F3B8
S214447910000386F8103303B0BDE8F08F30464020AD
S214447920D083402066667241CDCC4C3D00F81F00A3
S214447930084A094B1278094983F83823084A0978D3
S214447940127883F8392393F83A2361F3000283F8D4
S2144479503A23704722194020D083402020194020E3
S21444796021194020114B124A1B68124910B5124C7B
S214447970127884F82833114B1B6884F8293394F81A
S2144479802C3362F3000384F82C330D4B186808F04C
S214447990D1FD0C4908F08AFF08F026FA0DF02CFABF
S2144479A008F052FDA4F82A0310BD00BF1C1940205D
S2144479B01219402000C02344D08340201819402088
S2144479C0141940200AD7A33C284B294910B5294C02
S2144479D01B7884F82033284B186808F067FF08F0B3
S2144479E003FA0DF009FA08F02FFD244A244B03EA63
S2144479F040231068D4F82023000200F48070034328
S214447A0020481040204A03431268C4F82033120228
S214447A101E4B02F480721B7884F824331C4B1B687C
S214447A205B0203F4C06313431A4A1268D20202F498
S214447A30C0521343184A1268520302F400521343C6
S214447A40164A1268920302F480421343144A126898
S214447A50D20302F4C0321343D4F8242322F4FF3270
S214447A6022F480721343C4F8243310BD1019402006
S214447A70CDCCCC3DD0834020081940200C19402062
S214447A8000FEFF01FF0000FE0419402011194020AB
S214447A9000194020FC184020F8184020F4184020D4
S214447AA0F01840203A4B4FF084412DE9F047394EC8
S214447AB01B7886F81433384B1B7886F81533374BC7
S214447AC0186808F037FD4FF0834108F03BFE08F095
S214447AD0FFFF334B0446334993F800A0324B0AF079
S214447AE0010A186808F026FD304908F0DFFE08F061
S214447AF0EFFF2F4B81462F4993F800802E4B08F01A
S214447B000108186808F016FD2C4908F0CFFE08F066
S214447B10DFFF2B4B05464FF084411F78294BC5F3B6
S214447B200B0507F00107186808F004FD4FF0834181
S214447B3008F008FE08F0CCFF234BC0F3090245EAE0
S214447B4007351878C4F3090300F0010043EA8A2392
S214447B5042EA8022B6F8160300F4784002431B48F3
S214447B6000EAC929A6F81623D6F8182343EA0903D7
S214447B7002F07F4243EAC8531343C6F81833B6F8B4
S214447B801C3303F460431D43A6F81C53BDE8F0873A
S214447B90ED184020D0834020EC184020E0184020C8
S214447BA0DC18402033336F41D81840200AD7233C92
S214447BB0D4184020CDCCCC42D0184020CDCC4C3D1F
S214447BC0CC184020E8184020E418402000F87F00F5
S214447BD02DE9F74F374D384E686808F079FF86F838
S214447BE05803A86808F074FF344986F8590368694E
S214447BF008F0A0FC324908F059FE08F069FF8346B5
S214447C00A86908F065FF2D490446E86908F092FC27
S214447C102B4908F04BFECBF3090B08F059FF82467C
S214447C20286A08F055FF25498146686A08F082FCB0
S214447C30234908F03BFE08F04BFF8046A86A08F04C
S214447C4047FF1E4900F00107E86808F073FC1C492A
S214447C5008F02CFE08F03CFFC0F3090328690193A2
S214447C6008F036FF019B00F0010043EA8023B6F893
S214447C705A0300F4784003431248A6F85A33A30242
S214447C8000EACA2A03F480634FEA495043EA0B03E6
S214447C9000F4001043EA0A03034343EA8853C6F851
S214447CA05C3396F8603367F3000386F8603303B0BA
S214447CB0BDE8F08F30464020D0834020666672414F
S214447CC0CDCC4C3D00F81F000D4B0E4A1B780E4998
S214447CD082F834330D4B09781B7801F0010182F8A1
S214447CE035330B4B1B785B0003F002030B4392F8CF
S214447CF0361321F003010B4382F83633704700BF36
S214447D00CB184020D0834020C9184020CA184020B1
S214447D10C81840200C4B0D4A1B680D4982F8303376
S214447D200C4B09781B6801F0030182F831330A4B87
S214447D301B789B0003F00C030B430849097843EA7D
S214447D40011382F832337047C4184020D083402051
S214447D50BC184020C0184020BB184020BA18402009
S214447D60F8B5254B254C1B78254F84F85033254BC6
S214447D701B7884F85133244B1878323008F08EFC44
S214447D80014608F0D7FB08F0A3FE204984F85203C6
S214447D900E781F493F780D781E4907F001071E4BA1
S214447DA008781E491A78303009781D4B49001B78EC
S214447DB001F03E01394394F8537327F03F073943A3
S214447DC084F8531303F03F0102F01F0306F00F023A
S214447DD043EA411343EAC22305F03F0243EAC2336F
S214447DE000F03F0243EA4253D4F8542302F0784268
S214447DF01343C4F85433F8BDB9184020D083402008
S214447E00B6184020B8184020B7184020B218402072
S214447E10B1184020B0184020B4184020B51840206F
S214447E20B318402008B5FFF785FCBDE80840FFF7C7
S214447E3097BF38B50C4B0D4C5D68284607F0D4FF09
S214447E400CF0DAFF08F000FB0949C4F84C03284656
S214447E5008F02CFD07F0C8FF0CF0CEFF08F0F4FA4B
S214447E60C4F8480338BD00BF30464020D083402085
S214447E700000084208B5FEF772F8FEF7B7F8FEF7BA
S214447E802FF9FEF76DF9FEF7ADF9FEF791FAFEF716
S214447E90D5FAFEF713FBFEF74FFBFEF78BFBFEF718
S214447EA0ABFBFEF71FFCFEF74FFCFEF767FCFEF746
S214447EB0EDFCFEF757FDFEF7B5FDFEF733FEFEF785
S214447EC073FEFEF7AFFEFEF7EBFEFEF727FFFFF767
S214447ED01DF8FFF74DF8FFF77DF8FFF7A9F8FFF711
S214447EE02BF9FFF7C1F9FFF703FAFFF76DF9FFF730
S214447EF02FFAFFF747FAFFF757FAFFF76FFAFFF73D
S214447F007BFAFEF749FFFFF777FCFFF7CBFDBDE8AA
S214447F100840FFF78EBF114B11491B6810B5114C32
S214447F2084F86433104B1B6884F865330F4B186829
S214447F3008F000FB0E4908F0B9FC07F055FF0CF0BA
S214447F405BFF08F081FA0B4A94F868331278A4F879
S214447F50660362F3000384F8683310BDAC1840200F
S214447F6000C02344D0834020A8184020A4184020B2
S214447F700AD7A33CA11840200D4B0E4A1B780E4945
S214447F8082F870330D4B09781B7801F0010182F8B2
S214447F9071330B4B1B785B0003F002030B4392F8E0
S214447FA0721321F003010B4382F87233704700BF0B
S214447FB0A0184020D08340209E1840209F18402080
S214447FC09D1840200C4B0D4A1B780D4982F86C33A3
S214447FD00C4B09781B7801F0030182F86D330A4B89
S214447FE01B789B0003F00C030B430849097843EACB
S214447FF0011382F86E3370479C184020D08340208B
S2144480009A1840209B1840209918402098184020E1
S214448010114B12491B6810B5114C84F87433114B3C
S2144480201B6884F87533104B186808F083FA0F49B8
S21444803008F03CFC07F0D8FE0CF0DEFE08F004FA2C
S2144480400B4A94F878331278A4F8760362F3000364
S21444805084F8783310BD00BF9418402000C02344F1
S214448060D0834020901840208C1840200AD7A33C48
S214448070881840200D4B0E4A1B780E4982F87C33F4
S2144480800D4B09781B7801F0010182F87D330B4BC8
S2144480901B785B0003F002030B4392F87E1321F037
S2144480A003010B4382F87E33704700BF8718402095
S2144480B0D0834020851840208618402084184020CD
S2144480C00C4B0D4A1B680D4982F880330C4B0978DB
S2144480D01B6801F0030182F881330A4B1B789B002E
S2144480E003F00C030B430849097843EA011382F86A
S2144480F08233704780184020D0834020791840202F
S2144481007C184020781840207718402008B5FFF7A0
S21444811027FAFFF73FFAFFF77DF9FFF76DFAFFF707
S2144481208BFBFFF7BBFAFFF7DFFAFFF701FCFFF71D
S21444813019FCFFF749FCFFF74BFDFFF7C5FDFFF7BA
S214448140E9FDFFF7E8FEFFF717FFFFF73BFFFFF7F2
S2144481505FFFFFF78FFFBDE80840FFF7B1BF074A50
S2144481600020074BD2F88011D2F884219962DA6253
S214448170044B93E80600FBF74BBC00BFD08340207B
S21444818058874020DC894600144A154892F88D11D9
S21444819092F88C3110B4C1F3010480F8283001F011
S2144481A01C03C1F34111234380F82930D2F88C31A3
S2144481B0C3F3C13492F89431C3F3C003DB0143EAFA
S2144481C084030B4380F82A30D2F89031C3620020EF
S2144481D0044B10BC93E80600FBF71ABCD08340203F
S2144481E058874020E48946000B4A00200B4BD2F8BF
S2144481F098119962B2F89C1183F82C1092F89E114B
S21444820092F89F2183F82D1083F82E20044B93E890
S2144482100600FBF7FDBB00BFD083402058874020B4
S214448220EC894600084B002093F8F031C3F3000273
S21444823003F0FE031343054A82F82830044B93E8C0
S2144482400600FBF7E5BB00BFD0834020588740209C
S214448250F48946000D480E4AD0F8F4319362B0F8DB
S214448260F8319385B0F8FA31C3F30D0190F8FB3139
S214448270002003F0C00382F82E1043EA112382F84C
S2144482802F30044B93E80600FBF7C2BBD083402054
S21444829058874020248A460008B50A4B50200A4A8C
S2144482A0D3F8B01193F8B431283211600821137111
S2144482B004F0DAFA054B002093E80600BDE80840CF
S2144482C0FBF7A6BBD083402058874020FC89460055
S2144482D0094B00200949D3F8B82193F8BC318A6287
S2144482E003F0F002C3F30303134381F82F30044B27
S2144482F093E80600FBF78CBBD08340205887402089
S214448300048A4600094B00200949D3F8C02193F853
S214448310C4318A6203F0F002C3F30303134381F8C3
S2144483202F30044B93E80600FBF772BBD083402003
S214448330588740200C8A4600094B00200949D3F848
S214448340C82193F8CC318A6203F0F002C3F30303E6
S214448350134381F82F30044B93E80600FBF758BBD1
S214448360D083402058874020148A46000A4A00207A
S2144483700A4BD2F8E81192F8EC21996283F82C2043
S21444838083F82D2083F82E2083F82F20044B93E87F
S2144483900600FBF73DBB00BFD083402058874020F3
S2144483A01C8A4600254A264992F8D031C3F3010078
S2144483B003F0FC03034310B481F8283092F8D1311B
S2144483C0C3F3010003F0FC03034392F8D20181F89F
S2144483D02930C0F3010400F00C0323438409C0F39E
S2144483E0011081F82A3092F8D33103F003039B013D
S2144483F043EA8403034381F82B3092F8D43181F85E
S2144484002C3092F8D53103F03800C3F3020303430B
S21444841081F82D3092F8D631C3F38300D2F8D431A4
S214448420C3F3833343EA0013002081F82F30054B0F
S21444843010BC93E80600FBF7EBBA00BFD08340209D
S214448440588740202C8A46000B490C4A91F8D8316C
S214448450C3F3010003F0FC030343002082F82830F2
S21444846091F8D931C3F3010382F82930044B93E8D9
S2144484700600FBF7CDBA00BFD08340205887402083
S214448480348A4600084B002093F8E43103F0040293
S214448490C3F301031343054A82F82830044B93E898
S2144484A00600FBF7B5BA00BFD0834020588740206B
S2144484B03C8A46001049114A91F8DC31C3F3000067
S2144484C003F0FE03034382F8283091F8DD3103F0CD
S2144484D07C00C3F301030343002082F82930D1F81B
S2144484E0DC31C3F3CF335385D1F8E031D362044B48
S2144484F093E80600FBF78CBAD08340205887402088
S214448500448A460019491A48D1F8502200F5FE53C9
S21444851010B41A6041F6C473B1F85422C25291F8AA
S2144485205622C2F3C103C2F341041B0143EA840347
S214448530C2F30004C2F34012234343EA821341F6D3
S214448540C672835491F85732C3F38302B1F8563255
S214448550C3F3831343EA021341F6C77283540120DC
S214448560044B10BC93E80600FBF752BAD083402075
S214448570588740206C8A46001F49204B91F8580281
S21444858003F5FE5210B500F0F004C0F30300204398
S214448590107091F8590200F07004C0F303002043B1
S2144485A041F6C174185541F6C274D1F85802C0F366
S2144485B0C130185541F6C374B1F85A02C0F34700A7
S2144485C0185541F6C470B1F85C4291F85E121C52DC
S2144485D001F0F000C1F30301014341F6C77019549A
S2144485E00821142004F0A9FA054B012093E806005C
S2144485F0BDE81040FBF70CBAD08340205887402093
S214448600748A46001149124B01F5FE52D3F86002B3
S21444861010B5B3F86442106041F6C47093F86632FD
S2144486200C5203F0F000C3F30303034341F6C77050
S2144486300B540821152004F080FA064B012093E8D9
S2144486400600BDE81040FBF7E3B900BF588740205A
S214448650D08340207C8A460015491648D1F8983283
S21444866000F5FE5210B5136091F89C3203F01E04D8
S214448670C3F30003234341F6C474035591F89D3273
S214448680C3F34304B1F89C3241F6C771C3F34313B2
S21444869043EA041343540821162004F04EFA064BCA
S2144486A0012093E80600BDE81040FBF7B1B900BFCF
S2144486B0D083402058874020848A4600FFF7CCBFAA
S2144486C008B5FDF7BFFBF9F7C8F8FEF7E3F9BDE8D0
S2144486D00840FFF7C1BF084B012093F8A032C3F30C
S2144486E0000203F0FE031343044A1370044B93E85A
S2144486F00600FBF78DB900BFD083402018A7402062
S2144487008C8A460008B50E480E4B00F5FE52D3F848
S214448710301293F83432116003F0F001C3F30303CC
S2144487200B4341F6C77143540821502004F005FA20
S214448730054B012093E80600BDE80840FBF768B9FE
S21444874058874020D08340204C8A460008B50E48BF
S2144487500E4B00F5FE52D3F8381293F83C321160B3
S21444876003F0F001C3F303030B4341F6C7714354CC
S2144487700821512004F0E1F9054B012093E8060056
S214448780BDE80840FBF744B958874020D0834020D2
S214448790548A460008B50E480E4B00F5FE52D3F8F0
S2144487A0401293F84432116003F0F001C3F303031C
S2144487B00B4341F6C77143540821602004F0BDF9C9
S2144487C0054B012093E80600BDE80840FBF720B9B6
S2144487D058874020D08340205C8A460008B50E481F
S2144487E00E4B00F5FE52D3F8481293F84C32116003
S2144487F003F0F001C3F303030B4341F6C77143543C
S2144488000821612004F099F9054B012093E80600FD
S214448810BDE80840FBF7FCB858874020D08340208A
S214448820648A4600174B184A03F5FE51B2F86802AC
S214448830088092F86C1201F0F000C1F30301014382
S21444884041F6C270195441F6C37192F86D025854F9
S21444885041F6C471B2F87002585292F8741201F09C
S214448860F000C1F30301014341F6C67019540120D8
S21444887092F8751241F6C7729954044B93E8060071
S214448880FBF7C6B858874020D0834020948A4600D9
S214448890174B184A03F5FE51B2F87802088092F84E
S2144488A07C1201F0F000C1F30301014341F6C270AB
S2144488B0195441F6C37192F87D02585441F6C47176
S2144488C0B2F88002585292F8841201F0F000C1F3D4
S2144488D00301014341F6C6701954012092F88512EB
S2144488E041F6C7729954044B93E80600FBF790B8D8
S2144488F058874020D08340209C8A4600174B184A0D
S21444890003F5FE51B2F88802088092F88C1201F002
S214448910F000C1F30301014341F6C270195441F615
S214448920C370D2F890121954090A41F6C470195407
S21444893092F8941201F0F000C1F30301014341F6AA
S214448940C6701954012092F8951241F6C77299548C
S214448950044B93E80600FBF75BB800BF58874020FB
S214448960D0834020A48A46002848294990F80C32EF
S21444897001F5FE5270B5C3F3010403F0FC03234330
S214448980137090F80D32C3F3010403F0FC03234341
S21444899041F6C1740B5541F6C27390F80E42250158
S2144489A0A609C4F30114CD5490F80F5205F00303FE
S2144489B0C5F381051B0143EA8603234341F6C3748A
S2144489C043EA85130B5541F6C47390F81042CC54D1
S2144489D041F6C57490F8113290F812021D01C3F3A3
S2144489E0031300F00F000D5543EA001341F6C77019
S2144489F00B5408214FF4AE6004F09FF8054B012059
S214448A0093E80600BDE87040FBF702B8D0834020E8
S214448A1058874020CC8A46002D4991F8140238B530
S214448A20C0F3001500F008032A4C43EA4513C0F38C
S214448A30020504F5FE522B43C0F34015C0F38010E4
S214448A4043EA851343EAC01341F6C1701370B1F884
S214448A501432C3F3C713235441F6C270D1F8143208
S214448A60C3F3C733235491F81702C0F3C103C0F3CA
S214448A704105C0F341101B0143EA8503B1F8165281
S214448A80C5F3C1152B4343EA801341F6C370235400
S214448A9041F6C47091F818329B00235491F8193269
S214448AA0C3F38300B1F8183241F6C771C3F3831396
S214448AB043EA00134FF4B0606354082104F03DF8D1
S214448AC0054B012093E80600BDE83840FAF7A0BFFE
S214448AD0D083402058874020D48A460018491948F5
S214448AE091F82C3200F5FE5210B5C3F3010403F09E
S214448AF0FC032343137091F82D3203F03C04C3F374
S214448B000103234341F6C174035591F82E32C3F34F
S214448B108304D1F82C3241F6C771C3F3833343EA56
S214448B2004134354082140F2855004F006F8064BDB
S214448B30012093E80600BDE81040FAF769BF00BF7D
S214448B40D083402058874020DC8A46001149124B87
S214448B5001F5FE52D3F81C0210B5B3F8204210605B
S214448B6041F6C47093F822320C5203F0F000C3F37B
S214448B700303034341F6C7700B5408214FF4B26015
S214448B8003F0DBFF054B012093E80600BDE81040E8
S214448B90FAF73EBF58874020D0834020EC8A4600F0
S214448BA0104810B5104C90F8243204F5FE52137059
S214448BB090F8283203F00F0190F8273240F295508F
S214448BC0C3F3830343EA011341F6C7716354082190
S214448BD003F0B3FF054B012093E80600BDE81040C0
S214448BE0FAF716BFD083402058874020F48A4600C0
S214448BF0084B0120084993F8A43203F01C02C3F33F
S214448C000103134341F6C3728B54044B93E80600A6
S214448C10FAF7FEBED083402058874020AC8A4600F0
S214448C20084B41F6C271B3F8A822074BC2F30120A1
S214448C30585441F6C37101205A54044B93E8060035
S214448C40FAF7E6BED083402058874020B48A4600D0
S214448C50054B0120054A93F8AC321B011370044BB4
S214448C6093E80600FAF7D4BED083402018A74020E5
S214448C70BC8A4600074B41F6C1720749012093F867
S214448C80B03203F007039B008B54044B93E8060072
S214448C90FAF7BEBED083402058874020C48A460098
S214448CA0074B41F6C1720749012093F8B432C3F327
S214448CB003038B54044B93E80600FAF7A9BE00BF9F
S214448CC0D083402058874020E48A46000D4843F627
S214448CD05872B0F8D01208B549BA0B4B99521A4498
S214448CE090F8D21243F65A70C9011954032132201F
S214448CF003F0BAFD054B022093E80600BDE80840A1
S214448D00FAF786BED083402058874020FC8A460027
S214448D10114B43F65870114AB3F8F01249BA10B5DD
S214448D20115243F65A74B3F8F21293F8F43249BA2D
S214448D3003F00103115343F65C719B015354024400
S214448D400521402003F019FC054B022093E8060059
S214448D50BDE81040FAF75CBED083402058874020D8
S214448D60048B46003048314A90F8BC3290F8B8122A
S214448D7070B543F6587590F8BF42535543F6597349
S214448D80D15443F65A71D0F8B832C3F34F235BBA82
S214448D905352C4F3801304F0100141EAC301C4F3F0
S214448DA00103194390F8B93203F0010341EA431131
S214448DB0C4F3810304F0200441EA831143F65C7350
S214448DC0D15490F8C012C1F3800601F00803C1F3F1
S214448DD0010143EA06130B4390F8BE12D0F8BC02D6
S214448DE02343CC09C1F3801143EA841343F65D74EC
S214448DF01355C0F30D2343F65E74C0F305409B0041
S214448E001055642043EA410343F65F7153542A44A1
S214448E10082103F029FD064B022093E80600BDE82E
S214448E207040FAF7F5BD00BFD083402058874020F5
S214448E300C8B46001F4843F658721F4BB0F8EA1294
S214448E40C1F3C71170B5995443F65974D0F8E81273
S214448E501A44B0F8E852C1F3C731C5F3052619558C
S214448E6090F8ED4204F08001C4F38014314343F695
S214448E705A76995543F65B715D54B0F8EC5290F8C7
S214448E80E912C5F3052001F04001014343F65C7046
S214448E9041EAC411195443F65D716A205D540621B3
S214448EA003F0E2FC054B022093E80600BDE8704060
S214448EB0FAF7AEBDD083402058874020148B460036
S214448EC038B52C4B43F658702B4AB3F8C412B3F853
S214448ED0CC5249BA115293F8CA12CC09C5F30321AD
S214448EE041EA041193F8CD42C4F3001441EA441114
S214448EF093F8C742C4F3800441EA841193F8C94204
S214448F00C4F3800441EAC41143F65A74115543F637
S214448F105B71B3F8C642555443F65C71C4F3090515
S214448F20C4F387045454B3F8C812D3F8C832C1F310
S214448F300904C1F3051141EA851143F65D7551559F
S214448F40C3F3CB21C3F3C34343EA041343F65E742B
S214448F50135543F65F73D15402440821702003F03E
S214448F6083FC064B022093E80600BDE83840FAF737
S214448F704FBD00BFD0834020588740201C8B4600FE
S214448F80284A43F658702849B2F808335BBA30B4D6
S214448F900B5243F65A73B2F80A03B2F80C53C0F3B2
S214448FA00904C0F38700C854C5F3012092F80B3374
S214448FB003F00403034392F80D03C0F3800043EA2E
S214448FC0C00392F80E03C0F3401043EA001392F82D
S214448FD0100300F0010043EA401343F65B7043EA93
S214448FE0841343F65D740B5443F65C73D2F80C0357
S214448FF0CD54C0F3C923B2F80E23C0F347309B01C7
S2144490000855900943EA923343F65E728B5443F60E
S2144490105F73C8540220054B30BC93E80600FAF749
S214449020F7BC00BFD083402058874020248B46009E
S214449030104843F65871104A08B5B0F8FC325BBA8B
S214449040535290F8FE3203F00100C3F3400343EA60
S214449050400343F65A7013540A444FF444700321B1
S21444906003F08BFA054B022093E80600BDE808405F
S214449070FAF7CEBCD0834020588740202C8B46003D
S214449080134843F65872134BB0F8F81249BA10B561
S21444909099521A4490F8FA1243F65A70C1F30104EE
S2144490A01C54C1F3031443F65B70C1F381011C5492
S2144490B043F65C70195405214FF4547003F05DFA7E
S2144490C0054B022093E80600BDE81040FAF7A0BC22
S2144490D0D083402058874020348B4600254943F6A9
S2144490E05872B1F8000338B540BA234B91F803439D
S2144490F098521A44D1F8040304F00105C4F3440416
S214449100C0F3C53040EAC51043F65A75585543F681
S2144491105B75B1F80403C0F34510585543F65C75C7
S21444912091F80403C0F304005855B1F80603C0F39D
S214449130022500F4FC6045EAC40443F65D755C55BC
S21444914091F80543C4F3C304204343F65E741855AC
S21444915091F8020343F65F71585408214FF4617046
S21444916003F082FB054B022093E80600BDE8384036
S214449170FAF74EBCD0834020588740203C8B4600AC
S214449180094943F65870094AD1F8E0321BBA1350DD
S2144491900220D1F8E43243F65C711BBA5350044BB8
S2144491A093E80600FAF734BCD08340205887402022
S2144491B0448B46000E4845F6F062B0F8381308B5BE
S2144491C049BA0C4B99521A4490F83A1345F6F26051
S2144491D0C1F3000119540321332003F045FB064B29
S2144491E0032093E80600BDE80840FAF711BC00BF28
S2144491F0D0834020588740204C8B4600114B45F680
S214449200F060114AB3F8281349BA10B5115245F61E
S214449210F264B3F82A1393F82C3349BA03F00103E3
S214449220115345F6F4619B015354024405214020F2
S21444923003F000FA054B032093E80600BDE810400F
S214449240FAF7E6BBD083402058874020548B46002C
S2144492502248234A90F8201338B590F8243345F62C
S214449260F064135545F6F163D15445F6F261D0F8EF
S2144492702033C3F34F235BBA535290F82513C1F3FC
S2144492804013C1F380151B0143EAC503C1F34105EE
S2144492902B4390F8215305F0010543EA4513C1F3E7
S2144492A0C10501F0010143EA851345F6F4655355BB
S2144492B0D0F824336520C3F3C13343EA811145F61D
S2144492C0F563D1542244082103F0CEFA054B03201B
S2144492D093E80600BDE83840FAF79ABBD0834020AE
S2144492E0588740205C8B460038B52C4B45F6F060DA
S2144492F02B4AB3F81413B3F81C5349BA115293F8D3
S2144493001A13CC09C5F3032141EA041193F81D430B
S214449310C4F3001441EA441193F81743C4F3800499
S21444932041EA841193F81943C4F3800441EAC41112
S21444933045F6F264115545F6F361B3F816435554B1
S21444934045F6F461C4F30905C4F387045454B3F8EA
S2144493501813D3F81833C1F30904C1F3051141EACD
S214449360851145F6F5655155C3F3CB21C3F3C34385
S21444937043EA041345F6F664135545F6F763D154A9
S21444938002440821712003F06FFA064B032093E849
S2144493900600BDE83840FAF73BBB00BFD083402008
S2144493A058874020648B460008B5FEF7D8FEFEF783
S2144493B0EBFEFEF719FFFEF735FFFEF76DFFFEF7EF
S2144493C087FFFEF7D3FFFEF7EDFFFFF73DF8FFF705
S2144493D059F8FFF76FF8FEF73DFFFFF793F8FFF7EE
S2144493E0CBF8FFF70FF9FFF776F9FFF7AFF9FFF77A
S2144493F0D1F9FFF7F3F9FFF785F9FFF713FAFFF70B
S21444940047FAFFF77BFAFFF7AFFAFFF705FBFFF7DC
S2144494109DFBFFF763FBFFF7C3FBFFF7E9FBFFF793
S214449420FFFBFFF715FCFFF725FCFFF739FCFFF7BA
S21444943047FDBDE80840FFF757BF284A45F6F060A9
S2144494402749B2F858335BBA30B40B5245F6F26348
S214449450B2F85A03B2F85C53C0F30904C0F3870069
S214449460C854C5F3012092F85B3303F00403034366
S21444947092F85D03C0F3800043EAC00392F85E03AB
S214449480C0F3401043EA001392F8600300F0010072
S21444949043EA401345F6F36043EA841345F6F5641D
S2144494A00B5445F6F463D2F85C03CD54C0F3C92399
S2144494B0B2F85E23C0F347309B010855900943EA4F
S2144494C0923345F6F6628B5445F6F763C854032048
S2144494D0044B30BC93E80600FAF79ABAD08340208F
S2144494E0588740206C8B4600104845F6F061104A79
S2144494F008B5B0F834335BBA535290F8363303F0B9
S2144495000100C3F3400343EA400345F6F2601354B4
S2144495100A444FF44470032103F08CF8054B0320AF
S21444952093E80600BDE80840FAF772BAD0834020B4
S21444953058874020748B4600134845F6F062134B18
S214449540B0F8301349BA10B599521A4490F8321309
S21444955045F6F260C1F301041C54C1F3031445F606
S214449560F360C1F381011C5445F6F4601954052197
S2144495704FF4547003F05EF8054B032093E806005E
S214449580BDE81040FAF744BAD083402058874020BC
S2144495907C8B4600254945F6F062B1F8500338B551
S2144495A040BA234B91F8534398521A44D1F8540383
S2144495B004F00105C4F34404C0F3C53040EAC510C2
S2144495C045F6F265585545F6F365B1F85403C0F3CD
S2144495D04510585545F6F46591F85403C0F3040015
S2144495E05855B1F85603C0F3022500F4FC6045EA2A
S2144495F0C40445F6F5655C5591F85543C4F3C30475
S214449600204345F6F664185591F8520345F6F7613B
S2144496105854082140F2853003F026F9054B0320C0
S21444962093E80600BDE83840FAF7F2B9D083402004
S21444963058874020848B460008B5FFF74FFDBDE8A9
S2144496400840FFF7A7BF08B5F8F709F9FEF7EAFBA5
S214449650BDE80840FFF7F0BF094945F6F060094AFF
S214449660D1F848331BBA13500320D1F84C3345F68F
S214449670F4611BBA5350044B93E80600FAF7C8B992
S214449680D0834020588740208C8B4600114B47F6A9
S2144496908860114AB3F8641349BA10B5115247F6B4
S2144496A08A64B3F8661393F8683349BA03F001033F
S2144496B0115347F68C619B015354024405214020C4
S2144496C003F016F8054B042093E80600BDE8104066
S2144496D0FAF79EB9D083402058874020948B4600A2
S2144496E0104847F68861104A08B5B0F870335BBA3C
S2144496F0535290F8723303F00100C3F3400343EA35
S214449700400347F68A6013540A444FF444700321D6
S21444971002F0EEFF054B042093E80600BDE808403F
S214449720FAF776B9D0834020588740209C8B460071
S214449730134847F68862134BB0F86C1349BA10B511
S21444974099521A4490F86E1347F68A60C1F301049E
S2144497501C54C1F3031447F68B60C1F381011C54B7
S21444976047F68C60195405214FF4547002F0C0FF3C
S214449770054B042093E80600BDE81040FAF748B9C4
S214449780D083402058874020A48B460008B50A4B17
S21444979049F6226209494020B3F876335BBA8B52C5
S2144497A00521074A03F002F8064B052093E8060015
S2144497B0BDE80840FAF72CB9D083402058874020AB
S2144497C078254120AC8B4600134849F62062134B5B
S2144497D0B0F8801349BA10B599521A4490F88213D7
S2144497E049F62260C1F301041C54C1F3810449F6CE
S2144497F02360C1F303111C5449F62460195405210F
S2144498004FF4547002F0D2FF054B052093E806004F
S214449810BDE81040FAF7FCB8D08340205887402073
S214449820BC8B4600104849F62061104A08B5B0F88B
S2144498307C335BBA535290F87E3303F00100C3F393
S214449840400343EA400349F6226013540A444FF463
S2144498504470032102F0AAFF054B052093E8060056
S214449860BDE80840FAF7D4B8D08340205887402053
S214449870B48B460008B5FFF729FAFFF749FAFFF715
S21444988071FAFFF7D7FAFFF7D3FBFFF7F9FBFFF7B9
S21444989091FCFFF7B3FCFFF7DBFCFFF725FEFFF771
S2144498A04BFEFFF7F3FEFFF71BFFFFF741FFFFF703
S2144498B06DFFFFF7B7FFBDE80840FFF785BF08B563
S2144498C0FCF734FBF7F7A7FFFEF720FCBDE808409B
S2144498D0FFF7D0BF7047704770477047064AB2F8E4
S2144498E02C32B2F8701003F44043C1F30D010B431D
S2144498F0A2F82C32704700BFD0834020044BB3F804
S2144499001A21A3F83022B3F81421A3F83222704760
S214449910D0834020044BB3F8AE20A3F83822B3F8E3
S214449920A820A3F83A227047D08340207047704757
S214449930054BB3F87421A3F84022D3F87021C2F340
S2144499400F12A3F842227047D0834020054BB3F849
S2144499507C21A3F84822D3F87821C2F30F12A3F847
S2144499604A227047D0834020054BB3F87421A3F8AD
S214449970C021D3F87021C2F30F12A3F8C221704756
S214449980D0834020054BB3F87C21A3F8C821D3F8F4
S2144499907821C2F30F12A3F8CA217047D08340201F
S2144499A008B5FFF7E1FFFFF7EDFFFFF797FFFFF777
S2144499B0A5FFFFF7AFFFFFF7BBFFBDE80840FFF783
S2144499C0C5BF08B5FCF7D6F9F7F726FFFEF752FAF7
S2144499D0FFF7E6FFBDE80840FFF7E6BC7047704770
S2144499E0704770470B4AD2F8D031D2F89C101B0D02
S2144499F0C1F313011B050B43D2F8A010C2F8D031B3
S214449A0001F47F11D2F8D43123F47F130B43C2F808
S214449A10D4317047D083402008B5F9F799F8BDE8AB
S214449A200840F8F7BBBA7047F7F7F3BEFFF747BFEF
S214449A30FFF7C7BFFBF724BA7047074A1378632B70
S214449A4096BF01330023DBB21370044A1368013314
S214449A501360FEF735BE00BF78484120F82040200A
S214449A6008B5F9F7F1FFBDE8084002F055BB08B564
S214449A70FFF7E9FD4CF24053044AD058B0FA80F060
S214449A80BDE808404009F9F7DDB800BF7C484120EE
S214449A90014900201EF038BE90B0460000201EF05B
S214449AA02FBE0022114610461EF032BE704700BF3D
S214449AB02DE9F04FB84CE5B0D4E904230DF5987879
S214449AC0CDE93023DDE93001D4E9562306F02EF8FB
S214449AD0A1A3D3E9002306F0DFF906460F46A0A368
S214449AE0D3E90023D4E9580106F0D6F902460B46DA
S214449AF03046394606F01AF89BA3D3E9002306F00D
S214449B00F5FA95A3D3E90023D4E94E56D4E950ABED
S214449B10CDE95823CDE9005695A3D3E90023D4E9EB
S214449B205245CDE91201CDE95E23002000220023F0
S214449B309A49CDE9024552AC0025CDE95201CDE91A
S214449B405423CDE95623CDE95A01CDE95C23CDE92A
S214449B506023CDE96201CDE90A01CDE90623A14699
S214449B605046594608340135D9E9062306F094F997
S214449B7006460F46D9E90023DDE9000106F08CF9D4
S214449B8002460B463046394605F0D0FF06460F4699
S214449B90D4E90A23DDE9020106F07EF902460B46C3
S214449BA03046394605F0C2FF032DE8E80201D6D117
S214449BB0794C236D0293636D0493DDE94E23DDE90E
S214449BC04CABCDE90023DDE95023CDE90823DDE99C
S214449BD008010022002306F05FF9002280468946E9
S214449BE00023DDE9000106F057F952465B4605F0CE
S214449BF09DFF42464B4605F099FF02460B460298A7
S214449C00049905F091FF002206460F46002350466D
S214449C10594606F041F9DDE9002305F087FF424640
S214449C204B4605F083FF02460B46DDE9120105F07C
S214449C307BFF02460B46CDE90C234FA3D3E9002312
S214449C4006F02AF980468946304639464CA3D3E97D
S214449C50002306F021F902460B464046494605F0E5
S214449C6065FF52465B4605F061FF00220023C4E9C7
S214449C704E013046394606F00FF98046894642A3DF
S214449C80D3E90023DDE90C0106F006F902460B464B
S214449C904046494605F04AFFDDE9002305F046FF05
S214449CA002460B46CDE94201C4E9502330463946C4
S214449CB037A3D3E9002306F0EFF806460F46002202
S214449CC00023DDE90C0106F0E7F802460B46304671
S214449CD0394605F02BFFDDE9082305F027FFD4E9D4
S214449CE01A23D4E902ABC4E95201CDE91A235046FB
S214449CF000222B4B594606F055FB002840F00482C0
S214449D00D4E91267D4E90C453046394622462B46F8
S214449D1006F03EFB08B926462F4600224FF0804305
S214449D20DDE91A0106F020FB0022002800F0EF814E
S214449D3000233046394606F0AFF802460B46CDE9D6
S214449D400823154BD3E9AA4522462B4605F0ECFEDC
S214449D5006460F4626E000BFFCA9F1D24D62603F9E
S214449D60D9D6F61FCE4EE43F2DBA9CBB926FE43F45
S214449D7049DC63E9431794BF7B14AE47E17A843FDA
S214449D80E71DA7E8482ED33F386744696FF0EF3F96
S214449D903CBD5296218EB5BF000E42200000F03FD7
S214449DA000004940B0A3D3E9002306F005FB002891
S214449DB000F0AF8120462946ABA3D3E9002305F043
S214449DC0B5FECDE90801DDE90834B94E0022C6E9FE
S214449DD0AA34D6E95A45B74B2046294606F0ECFA4B
S214449DE0002840F0A8810022B34B2046294606F0BE
S214449DF0C5FA002840F0A28196F823330BB1C6E991
S214449E005C45AB4B20462946D3E95C6732463B4625
S214449E1005F08AFE04460D4695A3D3E9002306F0D2
S214449E20CBFA002840F08D812046294692A3D3E9F8
S214449E30002306F0A3FA002840F0878122462B46EA
S214449E403046394605F072FE02460B46DFF88882F5
S214449E50CDE936238AA3D3E9002306F01DF8044649
S214449E600D460BF011F806460F46204629460AF0E2
S214449E707DFF04460D46D8E90823D8E9060106F0D6
S214449E800BF822462B4606F007F80022002306F07D
S214449E9003F804460D4630463946D8E90A2305F009
S214449EA0FBFF02460B462046294605F03FFE76A3B6
S214449EB0D3E9002305F0F0FF75A3D3E9002305F0AA
S214449EC0EBFF00227D4B04460D4606F075FA00284B
S214449ED040F03F81002200232046294606F04EFAF1
S214449EE008B100240025724B93F824230AB1C3E931
S214449EF05E45D3E95E672046294632463B4605F032
S214449F0013FE04460D4664A3D3E9002306F054FA30
S214449F10002840F021812046294661A3D3E9002346
S214449F2006F02CFA002840F01B8122462B46304689
S214449F30394605F0FBFD02460B46CDE944235AA3B9
S214449F40D3E9002305F0A8FF594BCDE93801D3E9FE
S214449F500E45D3E9601220460023CDE900120022C4
S214449F60294606F001FA002800F0FE80002200236D
S214449F700298049906F00CFA50B10022504B504611
S214449F80594606F00FFA18B100230024CDE90034F0
S214449F90474CD4E90023CDE90C2394F82133002B15
S214449FA040F03181012384F8213384F82233DFF8EA
S214449FB000810022434DDDE90634DDE90001C8E9AD
S214449FC0D434414B06F0D0F9031E4FF000025946F4
S214449FD018BF0123504618933C4B06F0D9F9041E8B
S214449FE04FF000024FF0804318BF0124DDE908011A
S214449FF006F0CEF9189B00280CBF2046601C0024AF
S21444A000184405F0DFFE0022314B05F08FFDD8E9F9
S21444A010D62305F08BFD00222E4B06F0C3F9002212
S21444A020D8E9B867002800F00D8100233046394649
S21444A03006F09AF918B1DDE90623C8E9BE231C4E9A
S21444A040DDE90A23C6E9BA45D6E9BE45C6E9B823DA
S21444A050204600221C4B294606F090F900284AD098
S21444A0603CE000BFAFF30080FCA9F1D24D62703FE4
S21444A070FCA9F1D24D62603FFCA9F1D24D6260BFAB
S21444A080399D52A246DF913FE3A59BC420B0D23F00
S21444A090578C22C76075B53FFCA9F1D24D62903FFC
S21444A0A07B14AE47E17AC4BF9A9999999999E93F46
S21444A0B0000E422000002040000020C000004E4019
S21444A0C00000594000408F400000084000003440E3
S21444A0D00000F03F00001440088E46002046294603
S21444A0E0DDE93823C6E9BC2373A3D3E9002305F08E
S21444A0F01DFDC6E9BE01DDE90A34C6E9D4340023B1
S21444A100814CCDE9103419E10026002705E67F4B43
S21444A1100FE66BA3D3E900233046394606F02EF902
S21444A12000283FF450AE2046294667A3D3E90023CF
S21444A13005F0FAFC45E60024754D5DE60024754DB1
S21444A1405AE663A5D5E9004578E663A5D5E9004512
S21444A15074E60024704DC6E661A5D5E90045E4E6FC
S21444A16061A5D5E90045E0E6DDE9000106F044F9DD
S21444A17003283FF60DAFDFE800F002191D19002250
S21444A18000230298049906F003F900283FF400AF30
S21444A19000225E4B2046294606F0E6F878BB0022AD
S21444A1A05E4B2046294606F0DFF840BB00224FF0BF
S21444A1B080431AE0002200230298049906F0E8F847
S21444A1C000283FF4E5AE0022554B5046594606F06B
S21444A1D0E9F800283FF4DCAE00224C4B20462946E2
S21444A1E006F0C2F840B900224C4B2046294606F0F9
S21444A1F0BBF800283FF4CCAECDE90045C8E60023C2
S21444A2004FF08044C2E694F82233012B0DD100224D
S21444A210444BDDE90C0106F0B1F808B10223C4E66C
S21444A220DDE90623C4E9D623C1E631A3D3E90023F6
S21444A230DDE90C0106F0C0F808B10123B5E6DDE916
S21444A2400A23EFE7314B3046394606F08DF80028AE
S21444A25000F01082D8E9BC23D8E9100106F0A2F831
S21444A260002863D0D8E9BA4523A3D3E9002320467F
S21444A270294605F011FE02460B462046294605F0BF
S21444A28053FC04460D461EA3D3E9002306F076F895
S21444A29028B9C8E9BA45244BD3E9BA3431E7DDE9ED
S21444A2A00634C8E9BA34C8E9B834C8E9BC34C8E99D
S21444A2B0BE34F0E7AFF300807B14AE47E17A743FD8
S21444A2C0FCA9F1D24D6280BFFCA9F1D24D62803F19
S21444A2D0FCA9F1D24D62603FFCA9F1D24D6260BF49
S21444A2E0FCA9F1D24D62903F7B14AE47E17AC4BFDD
S21444A2F00000000000C062409A9999999999A93F34
S21444A3007B14AE47E17A843F00408F400000F03F24
S21444A31000002040000020C000004E4000000840DE
S21444A32000005940000049C0000E4220DDE90A23DF
S21444A330C8E9BA45C8E9D423CDE91045049C029837
S21444A34024F000410024B2A3D3E9002306F016F813
S21444A350002840F09281C04DDFF80483AEA3D3E9D1
S21444A3600023DDE9120105F097FD02460B46002066
S21444A370002105F0D9FB22462B4605F08DFD02460A
S21444A3800B46CDE932230022B44B05F085FDA4A349
S21444A390D3E90023CDE93A01D8E9620105F07CFD12
S21444A3A006460F46A0A3D3E90023DDE9320105F0B3
S21444A3B073FD02460B463046394605F0B7FB064663
S21444A3C00F46D8E96423DDE93A0105F0ADFB0022E7
S21444A3D0002305F061FD02460B463046394605F03B
S21444A3E0A5FB02460B46CDE91C2391A3D3E90023E3
S21444A3F005F0E2FF002840F042818FA3D3E9002312
S21444A400DDE91C0105F0BAFF002840F03C81DDE997
S21444A4101C23CDE91623DDE916232046294605F0FC
S21444A4203BFD8F4B04460D46D3E9AC6732463B466C
S21444A43005F07AFB00224FF080438046894605F0BB
S21444A440BBFF0022002800F022814FF080433046B4
S21444A450394605F06BFB04460D46814B0022C3E9A2
S21444A460AC45DDE900017F4B05F07EFF002800F097
S21444A4701F810020784922462B4605F00DFD0246F2
S21444A4800B46CDE934230022002305F08BFF18B990
S21444A49000230024CDE93434714C0022724BD4E9B5
S21444A4A0660105F0F9FC94F828332C902E9153B9A4
S21444A4B00123029A84F82833049BC4E93C23DDE94B
S21444A4C00623C4E9C423664E02980499B246D6E9E4
S21444A4D03C4522462B4605F027FB59A3D3E90023E7
S21444A4E005F0DAFC2B46224605F020FB96F8293385
S21444A4F004460D46C6E93C4523B90123C6E9C6458C
S21444A50086F82933DAE9C6894FA3D3E90023CAE992
S21444A510C645DAE9C40105F0BFFC424606460F4686
S21444A5204B462046294605F0FFFA49A3D3E90023C3
S21444A53005F0DCFD02460B463046394605F0F6FA91
S21444A54003460C460022CDE90601CAE9C4342C98D9
S21444A550464B2E9905F0A0FC002204460D463E4B81
S21444A560DDE9000105F000FF189B00284FF00002CB
S21444A5702046294608BF1E463D4B18BF4FF0FF36BF
S21444A58005F01AFF002840F096800022002320465B
S21444A590294605F0F3FE08B100240025304605F0B0
S21444A5A011FC22462B4605F077FC2D4B82468B4603
S21444A5B0D3E9AE4522462B4605F0B6FA0022294B8F
S21444A5C006460F4605F0F8FE0022002876D0254BB6
S21444A5D02046294605F0AAFA82468B46204B00229E
S21444A5E050465946C3E9AEAB214B05F0E5FE00287C
S21444A5F040F08080002200235046594605F0BEFEB7
S21444A60000287BD04FF0000A4FF0000B76E000BFE6
S21444A6109A9999999999B93F00000000007097401B
S21444A6209A9999999999C93FEC51B81E85EBB13FCF
S21444A63000000000008AAB40000000000088A3C071
S21444A640FA189C8FC1F9983F3A2BD5996DF4EC3F94
S21444A650FCA9F1D24D62603F0000F03F00407F40CD
S21444A660000E4220000008400000B03F000054C0E6
S21444A67000408F400023002443E500256CE616A3E3
S21444A680D3E90023C5E616A3D3E90023C1E64FF079
S21444A69040434046494605F071FE00283FF4DDAE8F
S21444A6A000224FF080433046394605F03DFAD2E664
S21444A6B000200021DFE600240B4D6FE70B4B3046AD
S21444A6C0394605F05BFE002888D00022084B204619
S21444A6D0294605F029FA7FE700000000008AAB40CF
S21444A6E0000000000088A3C000408F40000008C05F
S21444A6F0000008404FF0000ADFF848B30022002369
S21444A700DDE9000105F030FE0646002840F0B68339
S21444A71000224FF08043DDE9000105F025FE58B9DC
S21444A720C74B0022DDE9000105F01EFE189B0028F9
S21444A7300CBF1E464FF0FF360022C24BDDE908012F
S21444A74005F0AAFB9AA3D3E9002305F0CFFC9AA30D
S21444A750D3E9002305F0A0FB0022BB4B05F09CFB8D
S21444A76097A3D3E9002305F0C1FC04460D463046C2
S21444A77005F028FB02460B462046294605F08CFB8E
S21444A78002460B46CDE90E23B04BD3E9B0452246EC
S21444A7902B4605F0C9F906460F468BA3D3E900239A
S21444A7A005F00AFE002800F06B832046294686A35F
S21444A7B0D3E9002305F0BAF9CDE90E01A34CDDE94F
S21444A7C00E23DDE90E01C4E9B023D4E9682305F07D
S21444A7D0ADF97FA3D3E9002305F05EFB06460F469A
S21444A7E07DA3D3E90023D4E96A0105F055FB02466C
S21444A7F00B463046394605F099F979A3D3E9002348
S21444A80005F074FC02460B46CDE90A23D4E96C23D2
S21444A81005F08AF900228B4B05F03EFBD4E96E2303
S21444A82005F082F902460B46CDE91E23D4E970238F
S21444A83005F07AF90022834B05F02EFBD4E9722307
S21444A84005F072F902460B46CDE92023D4E9742379
S21444A85005F06AF900227B4B05F01EFBD4E976230B
S21444A86005F062F960A3D3E90023CDE93C01DDE9B4
S21444A8700A0105F011FB06460F465DA3D3E9002303
S21444A880DDE91E0105F008FB32463B4605F04EF96D
S21444A8908046894658A3D3E90023DDE9200105F024
S21444A8A0FBFA02460B464046494605F03FF9DDE9C9
S21444A8B03C2305F03BF952A3D3E9002305F0ECFA18
S21444A8C0D4E97823CDE922011046194605F02EF93D
S21444A8D0DDE9222305F02AF9D4E93E2305F026F9DA
S21444A8E049A3D3E9002305F0D7FA8046894648A30E
S21444A8F0D3E90023D4E97A0105F0CEFA02460B46A2
S21444A9004046494605F012F98046894642A3D3E9B3
S21444A9100023D4E9420105F0BFFA02460B464046FE
S21444A920494605F001F93EA3D3E9002305F0DEFBD2
S21444A93002460B46CDE92423D4E97C2305F0F6F8F9
S21444A94023A3D3E9002305F0A7FA8046894636A315
S21444A950D3E90023D4E97E0105F09EFA02460B466D
S21444A9604046494605F0E2F831A3D3E9002305F012
S21444A970BDFBDDE90C23CDE93E01DDE90A0105F026
S21444A980D3F80022324B04460D4605F015FD002848
S21444A99040F088822046294627A3D3E9002305F0C1
S21444A9A0EDFC002840F08F8254E000BFAFF30080F7
S21444A9B0000000000020AC405C8FC2F528DC274035
S21444A9C0B46155D0CC38FB3F9A9999999999D93F17
S21444A9D0FCA9F1D24D62603FB428207983A6BA3FE1
S21444A9E054434F56A8ACBB3F9A999999999963405A
S21444A9F09A99999999996A40CDCCCCCCCCCC35408F
S21444AA00E3F36EFB79D0E33E277845D92444D93F17
S21444AA10FB50D7647BD71C403043BB3975F10440A8
S21444AA206D0D4BFEC9AF1840EBF33CDE4AA2813FA6
S21444AA30E9C8B5C771D3893F0000000000409FC0F5
S21444AA400000F03F00408F4000004E40000E422081
S21444AA5000409F400022C64B2046294605F0ACFCE9
S21444AA60002800F022820022C14B2046294605F0E9
S21444AA705BF880468946BF4CDDE90A01D4E9802369
S21444AA8005F052F80022BC4B05F006FAD4E98223BE
S21444AA9005F04AF802460B46CDE92623D4E984233A
S21444AAA005F042F80022B44B05F0F6F9D4E98623C3
S21444AAB005F03AF802460B46CDE92823D4E9882324
S21444AAC005F032F80022AC4B05F0E6F9D4E98A23C7
S21444AAD005F02AF88AA3D3E90023CDE94001DDE94D
S21444AAE0260105F0D9F932463B4605F01FF80646DE
S21444AAF00F4685A3D3E90023DDE9280105F0CCF908
S21444AB0002460B463046394605F010F8DDE9402348
S21444AB1005F00CF87EA3D3E9002305F0BDF9D4E98B
S21444AB20B22305F001F802460B46CDE94623D4E9A4
S21444AB308C2304F0FBFF78A3D3E9002305F0ACF99B
S21444AB4006460F4676A3D3E90023D4E98E0105F0E2
S21444AB50A3F902460B463046394604F0E7FF72A393
S21444AB60D3E9002305F0C2FAD4E99023CDE91401D1
S21444AB701046194604F0DAFFDDE9142304F0D6FF44
S21444AB80D4E9462304F0D2FF69A3D3E9002305F0B1
S21444AB9083F906460F4668A3D3E90023D4E9920115
S21444ABA005F07AF902460B463046394604F0BEFFB5
S21444ABB006460F4662A3D3E90023D4E94A0105F0CA
S21444ABC06BF902460B463046394604F0ADFF5EA3A9
S21444ABD0D3E9002305F08AFA0022684BCDE92A011E
S21444ABE00298049905F0CAFB002840F075810022BB
S21444ABF0624B0298049904F097FF55A3D3E90023C7
S21444AC0005F04AF900225E4B06460F4605F0CAFB9D
S21444AC1008B100265A4F50A3D3E90023DDE92A01A0
S21444AC2005F03AF90022574B05460C4605F0A6FBBC
S21444AC300C90002840F053810022534B284621466E
S21444AC4005F0BAFB002840F04D8104F1004440462C
S21444AC50494643A3D3E9002305F01EF9DDE93E2324
S21444AC6004F064FF8046894632463B4628462146E1
S21444AC7005F012F902460B464046494604F056FF94
S21444AC8002460B46CDE90C230022404B05F094FBCC
S21444AC90002840F02A8100223D4BDDE90C0105F0F6
S21444ACA06DFB002840F02681324C3A4D2EA3D3E962
S21444ACB00023D4E9380105F0EFF806460F460AF0BB
S21444ACC0E3F8D5E9042305F0E7F8CDE94A01304630
S21444ACD039460AF04BF806460F46D5E90223D5E92D
S21444ACE0000105F0D9F832463B4605F0D5F80AA3EC
S21444ACF0D3E90023CDE948014EE000BFAFF300801E
S21444AD009A99999999996A40CDCCCCCCCCCC35407B
S21444AD10E3F36EFB79D0E33EFCA9F1D24D62603F8B
S21444AD205ED817C2038C9E3F6F216A9B4B52A13F4D
S21444AD302ED7D19C0A49373F7119ABB745FF1F4000
S21444AD40ECBC164D8E930F401988C921F33610403B
S21444AD509A9999999999C93FCDCCCCCCCCCCEC3F17
S21444AD603B08AA2A23DCA63F399D52A246DF913FE0
S21444AD7000004940000E422000408F40000014402E
S21444AD800000F03F00003EC000003E40000054403B
S21444AD90000054C0088E4600D4E9C00104F0C6FE44
S21444ADA094F9203306460F46012BC4E9C06700F0E9
S21444ADB0A480022B40F0A58053A1D1E900012C9A2F
S21444ADC02E9B04F0B3FE00225F4B05F065F8044664
S21444ADD00D464FA3D3E90023DDE9060105F05CF8F0
S21444ADE002460B462046294604F0A0FE0AF092F896
S21444ADF00022564B04F09AFE0022554B05F04CF8C0
S21444AE0045A3D3E9002304F091FE00220023044620
S21444AE100D4605F0C7FA002800F0808600224B4B0A
S21444AE202046294605F0B4FA002800F0E9860022B8
S21444AE30484B2046294605F0BFFA48B138A3D3E923
S21444AE4000233046394605F0ADFA002840F0968097
S21444AE500022414B2046294605F090FA002800F08F
S21444AE60DB862FA3D3E900233046394605F09AFA09
S21444AE70002800F0D186394B022281E000265BE4AC
S21444AE8029A3D3E900233046394605F077FA00284B
S21444AE903FF494AC2046294625A3D3E9002304F086
S21444AEA043FE89E400242E4DDDE500222D4B20464A
S21444AEB0294605F077FA50B900222B4B20462946FE
S21444AEC004F034FED5E51CA5D5E90045F4E74FF07B
S21444AED000084FF00009CEE5002600279BE6002533
S21444AEE0224CB4E60C9D224CB1E60023214CCDE91D
S21444AEF00C34D9E60023204CF9E711A1D1E900012E
S21444AF005DE7002000215AE77B14AE47E17AB4BFE0
S21444AF107B14AE47E17A943F9A9999999999A93FB7
S21444AF20B81E85EB51B8AE3F9A9999999999E9BF5D
S21444AF309A9999999999E93F0000000000409FC06A
S21444AF407B14AE47E17AB43F000014400000F03F63
S21444AF500000E03F0000E83F0000D03F000E4220E3
S21444AF6000409F40000049C00000494000003E4069
S21444AF7000003EC000005440000054C0BE4B0122B6
S21444AF80002183F820230022C3E9C012DFF8E882B8
S21444AF9020462946D8E9C26732463B4604F0C4FDFB
S21444AFA0A5A3D3E9002304F077FF32463B4604F0DA
S21444AFB0BDFD03460C46C8E9C2342E9CA0A3D3E983
S21444AFC00023CDE906012C9824F0004105F08EF8C4
S21444AFD00022002306460D4605F0DAF9002840F024
S21444AFE0A185A64AAA4304D1C5F31303334340F0CC
S21444AFF099850022A24B3046294605F0D3F908B17C
S21444B00000269F4D00220023DDE9480104F044FF5A
S21444B010DDE94A2304F08AFD8BA3D3E9002304F038
S21444B0203BFF8BA3D3E9002304F036FF002280467F
S21444B03089460023DDE9000105F096F90446002818
S21444B04040F0748500224FF08043DDE9000105F0AE
S21444B0508BF958B98A4B0022DDE9000105F084F9E2
S21444B0600028189B18BF4FF0FF331C460022854B20
S21444B0704046494605F0A0F9002840F05A8500228B
S21444B08000234046494605F079F918B14FF00008C8
S21444B0904FF00009784B93F8E830002B00F04F85CA
S21444B0A00022774BDDE9080105F07CF9002800F022
S21444B0B046850020724942464B4604F0EDFEDDE9E3
S21444B0C00C2304F033FD80468946204604F07AFE7D
S21444B0D002460B464046494604F0DEFE0022002364
S21444B0E08046894605F05EF918B94FF000084FF0DF
S21444B0F0000942464B46DDE9060104F0CDFE3246E1
S21444B1002B4604F0C9FE002280468946002350465A
S21444B110594605F047F918B94FF0000A4FF0000BAE
S21444B12000205749DDE9062304F0FEFC52465B4600
S21444B13004F0B2FE32462B4604F0AEFE0022002354
S21444B140CDE906014046494605F036F9C0B100222D
S21444B1500023DDE9060105F02FF988B142464B4647
S21444B160DDE9060105F00AF93BA3D3E900230028EC
S21444B17000F0E984DDE9060104F08EFECDE906011F
S21444B18037A3D3E900234046494605F0F7F818B1FB
S21444B1904FF000084FF0000931A3D3E90023DDE95E
S21444B1A0060105F0EBF818B100230024CDE9063477
S21444B1B000224FF08043DDE91A0105F0D5F8002857
S21444B1C000F0C9840022304B0298049904F064FECF
S21444B1D006460F4624A3D3E9002305F0EDF80028DD
S21444B1E040F0C184002200233046394605F0C6F8B4
S21444B1F008B1002600270022214BDFF87CA0DDE9B9
S21444B200080105F0CFF848B919A3D3E90023DAE9D1
S21444B210320105F0C7F8002800F0BD8400221B4B1D
S21444B220DAE910452046294605F0BCF8002800F027
S21444B230B2842DE0AFF30080111111111111A13F1A
S21444B2409A9999999999D93FE3A59BC420B0D23F3E
S21444B250578C22C76075B53F333333333333E33FBC
S21444B260333333333333D33F000000000088A340E6
S21444B2707B14AE47E17A843F000E42200000F07F04
S21444B2800000F03F00004E400000594000002440BB
S21444B290A5A3D3E90023DDE9120105F083F80028CD
S21444B2A000F079840022B64B0298049905F07AF8A7
S21444B2B0002800F070840022B24B3046394605F030
S21444B2C067F8002800F06784DAE9B623DAE908016B
S21444B2D0CDE9182396A3D3E9002304F0DDFDDDE988
S21444B2E0422304F023FC94A3D3E9002304F0D4FDC2
S21444B2F002460B462046294604F0F8FE04460D4610
S21444B3000022A14BCAE9544505F056F8002800F03F
S21444B310398400229D4B2046294605F02FF8002804
S21444B32000F0308420462946DDE9182304F0FCFB6F
S21444B33021F0004CDDE91823614604F0D7FE7AA3D9
S21444B340D3E9002305F01AF8002800F01B847CA3F8
S21444B350D3E90023DDE9180104F09EFD7AA3D3E97E
S21444B3600023CDE92C012946204604F095FD0246EB
S21444B3700B46DDE92C0104F0D9FB02460B46CAE92C
S21444B380B623DDE9182304F0CFFB21F00045002264
S21444B3907F4B294604F0F2FF002800F0E98301239E
S21444B3A08AF827337B4B00204FF08041C3E9F001F5
S21444B3B0784CD4E9B623DDE91A01C4E9EE23C4E99E
S21444B3C0CC6700224FF08043C4E9EA6704F0CCFF20
S21444B3D00022002800F0E6836F4BD4E9200104F0F5
S21444B3E0C3FF002800F0EB8300226B4BD4E9220114
S21444B3F004F0BAFF002800F0E28302984FF00008F9
S21444B400049953A3D3E9002304F070FE0022634B4F
S21444B41004F0D2FF002800F0D483DFF884915D4C1A
S21444B42000225D4BD4E91E0104F09EFF002840F044
S21444B430CB8342464B46C4E9D223DDE9340146A3D6
S21444B440D3E90023C4E9EC8904F026FD44A3D3E9F8
S21444B450002304F04BFEDDE90623C4E9DE01C4E91B
S21444B460DC23DDE91C01DDE9162304F05DFBDDE9A0
S21444B4701023CDE92C01C4E9DA23DDE90023DDE914
S21444B4803001C4E9E423DDE93823C4E9D023DDE907
S21444B4903623C4E9D823D4E9942304F047FB32A3E3
S21444B4A0D3E9002304F0F8FC06460F4630A3D3E95C
S21444B4B00023D4E9960104F0EFFC02460B463046DE
S21444B4C0394604F033FB2CA3D3E9002304F00EFEE4
S21444B4D0D4E99823CDE91A01D4E9060104F026FB01
S21444B4E021A3D3E9002304F0D7FC06460F4620A345
S21444B4F0D3E90023D4E99A0104F0CEFC02460B4675
S21444B5003046394604F012FB1BA3D3E9002304F06B
S21444B510EDFDD4E99C23CDE90401D4E9080104F007
S21444B52005FB3FE0AFF300809A9999999999C93FF2
S21444B5307B14AE47E17A843F8462BF15623E973FF0
S21444B5405C8FC2F5285CEF3F7B14AE47E17A943FAC
S21444B550CDCCCCCCCCCC0C400E9F7422C154D13F25
S21444B5605C8FC2F528DC2740FCA9F1D24D62603FCF
S21444B570FEF2469F2892AF3F1F94D22C39CFB03F5D
S21444B5800000F83F0000244000407F4000409F40B9
S21444B59000001440000E42200000F03F0000E03F50
S21444B5A0000054C0B0A3D3E9002304F075FC06465B
S21444B5B00F46AFA3D3E90023D4E99E0104F06CFC04
S21444B5C002460B463046394604F0B0FAAAA3D3E9FD
S21444B5D0002304F08BFDDDE90423CDE90601104683
S21444B5E0194604F059FC04460D46DDE90623104688
S21444B5F0194604F051FC02460B462046294604F000
S21444B60095FA09F0FDFC0022002304460D4604F09A
S21444B610ABFE48B922462B46DDE91A0104F066FD26
S21444B62009F01AFA04460D46974E20462946974F87
S21444B630D6E95A23CDE9102391A3D3E9002304F095
S21444B6402BFC02460B46DDE9100104F06DFAD6E900
S21444B6500A34CDE91C01CDE91634DDE91601D6E9F4
S21444B660A22304F063FA80A3D3E9002304F014FC75
S21444B67004460D467EA3D3E90023D6E9A40104F08C
S21444B6800BFC02460B462046294604F04FFA7AA3A2
S21444B690D3E9002304F02AFDD6E91445CDE9180180
S21444B6A022462B46DDE9080104F03EFA0022784B98
S21444B6B0CDE92E012046294604F0EEFB02460B4611
S21444B6C00020744904F030FA0022704B0C460546BC
S21444B6D004F054FE002808BF284663A3D3E9002399
S21444B6E016BF00202146394604F0D6FB96F825338B
S21444B6F082468B46D6E916010BB1C6E9A601D6E9C1
S21444B700A623CDE9022304F00FFA00228046894698
S21444B7105E4B2846214604F031FE002840F057820E
S21444B72004F1004442464B465046594604F026FE31
S21444B730002840F04F82284621464BA3D3E90023F5
S21444B74004F0AAFB06460F4602460B4640464946C8
S21444B75004F014FE08B946464F4632463B46DDE9F9
S21444B760020104F0E3F9484B0A46CDE902010146DA
S21444B770C3E9CE12C3E9E81293F82623D3E91801A5
S21444B7800AB1C3E9A801D3E9A88942464B4604F066
S21444B790CBF906460F4602460B465046594604F039
S21444B7A0EDFD78B9284621462FA3D3E9002304F0BB
S21444B7B073FB32463B4682468B4604F0FDFD08B991
S21444B7C0B246BB4652465B464046494604F0AEF94E
S21444B7D02D4C02460B46C4E9E02300220023CDE963
S21444B7E00801C4E9E623D4E91C0100222A4B04F0EC
S21444B7F0BBFD68B90022284BD4E91E0104F0B4FD11
S21444B80030B90022244BD4E9280104F0ADFD18B128
S21444B8100022214BC4E9E6231B4C00221E4BD4E9EC
S21444B8202A0104F0A1FDA0B900221B4BD4E92C0147
S21444B83004F09AFD68B90022174BD4E92E0104F0AF
S21444B84093FD30B90022144BD4E9300104F08CFD4A
S21444B85088B30D4E00220023D6E91A4520462946D1
S21444B86004F082FD1AE000BFFCA9F1D24D62603FAD
S21444B870FEF2469F2892AF3F1F94D22C39CFB03F5A
S21444B880F8C1631ADCA54C40000E4220008061409B
S21444B89000001A40000079400000F03F38B900220A
S21444B8A04FF080432046294604F05EFD18B100233D
S21444B8B08D4CC6E9E6348D4C00228B4BD4E92001EE
S21444B8C004F052FD40B90022874BD4E9220104F02B
S21444B8D04BFD002800F08181844B0021824AC3E955
S21444B8E0E612DFF808A20022DAE9A067DDE912349E
S21444B8F0DAE90489CAE9583430467D4B3946CAE900
S21444B900568904F0C9FA04460D460022794BDDE90F
S21444B9101C0104F0C1FA02460B462046294604F0B0
S21444B92005F902460B46DDE9180104F0FDF86CA360
S21444B930D3E9002304F0B0FADDE9102304F0F6F866
S21444B940DDE93634CAE95A01CAE95C34DDE94434EF
S21444B950DDE93201CAE95E34DDE90034CAE960341F
S21444B960DAE9B42304F0E0F85DA3D3E9002304F055
S21444B97093FADAE9622304F0D9F80022DDE93A348E
S21444B980CAE96201CAE96434DAE966015A4B04F04A
S21444B99083FADDE92E2304F0C9F8DDE90E34CAE95A
S21444B9A06601CAE96834DDE90A34CAE96A34CAE990
S21444B9B06C34DDE91E34CAE96E34CAE97034DDE914
S21444B9C02034CAE97234CAE97434DDE93C34CAE93D
S21444B9D07634DDE92234CAE97834DAE94023CAE920
S21444B9E03E23DDE92234CAE94034DDE92434CAE999
S21444B9F07A34DAE94423CAE94223DDE92434CAE93D
S21444BA004434CAE97C34DDE93E34CAE97E34DDE9AF
S21444BA100C34CAE9B234DDE90A34CAE98034DDE9D3
S21444BA202634CAE98234CAE98434DDE92834CAE9CA
S21444BA308634CAE98834DDE94034DDE91C01CAE9C4
S21444BA408A34DDE94634CAE99489CAE98C34DDE9A6
S21444BA501434CAE98E34CAE99034DAE94823CAE988
S21444BA604623DDE91434CAE94834DDE92A34CAE910
S21444BA709234DAE94C23CAE94A23DDE92A34CAE98E
S21444BA804C34DDE92C34CAE9B434DDE91A34CAE965
S21444BA909634DAE90623CAE99823DDE90434CAE988
S21444BAA09A34DAE90823CAE99C23DDE90634CAE96C
S21444BAB09E340BA3D3E9002304F0EEF93B4632460A
S21444BAC004F034F8DDE91634CAE9A001CAE9A23420
S21444BAD0DDE91834CAE9A434DDE902340EE000BFD7
S21444BAE0FCA9F1D24D62603F0000F03F000E4220B8
S21444BAF000001440000059400000EE3FCAE9A63456
S21444BB0000238AF82333AAF824338AF82633DDE957
S21444BB100834CAE9A83465B0BDE8F08F002400258F
S21444BB20FFF79FB900263546FFF76CBA0024FFF7A7
S21444BB309DBA4FF00008DFF82091FFF7ABBA00201B
S21444BB400021FFF7B8BA4046494604F0A5F98046B6
S21444BB508946FFF715BBDDE90623DDE9100103F04E
S21444BB60E5FFFFF735BB34A7D7E90067FFF743BBCC
S21444BB709AF82733002B7FF415AC0023324CCAE9DD
S21444BB80F03415E40022314B002183F827232E4A53
S21444BB90C3E9F0120CE400222C4B002183F827233F
S21444BBA00022F5E72A4B4046494604F005FC0028A7
S21444BBB03FF435AC4FF00008DFF894902FE44FF094
S21444BBC000084FF000092AE40022002333E400254D
S21444BBD0204CA7E556465F46BFE500221A4BD4E9FB
S21444BBE0240104F0C1FB00283FF47BAE0022164B30
S21444BBF0D4E9260104F0B8FB00287FF46DAE70E665
S21444BC000FA3D3E900233046394600240E4D04F0F2
S21444BC10C9FB00287FF4B2A93046394608A3D3E9C5
S21444BC20002304F0BFFB00283FF4B0A9074B0022D2
S21444BC3083F82023FFF7AAB9000000000088A34039
S21444BC40B81E85EB51B8AE3F0000F03F000E4220D0
S21444BC5000005440008061C000004E4000221C4B4F
S21444BC60104619461B4A10B51B4CC4E9F2011B4941
S21444BC70C4F8F0230122C4F8D013194984F82323C6
S21444BC8084F82623C4E9F6014FF0FF41C4F8E013D4
S21444BC901449C4E9FA0140F20111A4F8241308A196
S21444BCA0D1E90001C4E9C00100200F49C4E9C2013A
S21444BCB005A1D1E90001C4E9B60110BDAFF3008087
S21444BCC00000000065CDCD410000000000709740A4
S21444BCD00000F8FF000080FF000E42200000C0FF76
S21444BCE00000F07F0000F0FF0000E03FF8B55B4B3B
S21444BCF000265B4C0027186804F076F8594B1D68FC
S21444BD00C4E90001284604F04DF8574BC4E91A012B
S21444BD10186804F069F8554BC4E91401186804F02F
S21444BD2063F8534BC4E90401186804F05DF8514BBA
S21444BD30C4E90601186804F057F84F4BC4E90801F3
S21444BD40186804F051F84D4BC4E90A01186804F029
S21444BD504BF84B4BC4E93201186804F045F8494B9C
S21444BD60C4E93601186804F03FF8474BC4E90201B9
S21444BD70186804F039F8454BC4E91001C4E934673F
S21444BD80186804F031F8424B1B78003B18BF012377
S21444BD90C4E9380184F8E830C4E92A67C4E92C6762
S21444BDA0C4E92E67C4E93067C4E91C67C4E91E6762
S21444BDB0C4E92067C4E92267C4E92467C4E926675E
S21444BDC0C4E9286725BB334B186804F00DF8324B9A
S21444BDD0C4E90201186803F0E5FF00222F4BC4E9CA
S21444BDE012232F4BC4E90C01C4E93267186803F0E8
S21444BDF0D9FF2C4BC4E90E01186803F0F5FF2A4B13
S21444BE00C4E91601186803F0EFFFC4E91801F8BD49
S21444BE10012D1CD1254B186803F0C4FF244BC4E9FC
S21444BE200C01C4E93267186803F0BCFF214BC4E92F
S21444BE301201186803F0B6FF1F4BC4E90E011868D8
S21444BE4003F0D2FFC4E91867C4E91601DFE7023DF0
S21444BE50012DDCD8C4E90C67D9E700BF701E40202A
S21444BE60000E4220581C4020781C4020201F4020B2
S21444BE70401F4020041F4020101F4020A01F402089
S21444BE80501C4020B41F40206C1E4020581F4020A9
S21444BE90541F4020B81D4020C01D40200000444090
S21444BEA0901D4020AC1D4020A81D40209C1F4020D3
S21444BEB0681F4020841F4020A81F4020784B2DE94F
S21444BEC0F04FD3F800A085B0764B774CC3F800A06B
S21444BED0764BDFF834921B68754FC9F80030754EC0
S21444BEE0DFF828B2D4E9040104F0CEFA724B1860A5
S21444BEF0D4E9020104F0C8FA054638603060D4E953
S21444BF00140104F0C1FA6D4ACBF800008046106074
S21444BF10D4E9180104F098FA694901900860D4E914
S21444BF20220104F091FA67490880D4E9240104F018
S21444BF308BFA65490870D4E91A0104F085FA634916
S21444BF400870D4E9200104F09FFA61490860D4E9F6
S21444BF501E0104F099FA5F490860D4E91C0104F014
S21444BF6093FA5D49086028465C490C68214604F00B
S21444BF70A5FD524A029210B13C6034600DE004F1D3
S21444BF8000442846214604F07BFD0028F4D121468F
S21444BF90284604F075FD0028EFD1514940460391E8
S21444BFA004F08CFD28B10399029BCBF8001019606D
S21444BFB006E04C494046039104F062FD0028F2D165
S21444BFC0494B4A4C1B68002B4DD1494B1968019B81
S21444BFD023F00205012D04D1504604F0ABFA20604C
S21444BFE000E02160434D2068294604F05DFD00B121
S21444BFF0256023680022DFF818813F4D3F4CC8F87F
S21444C00000302B603E4BD4E9200104F0ADF910B16A
S21444C0100023C8F800300022394BD4E9220104F04A
S21444C020A3F908B100232B600022354BD4E9240140
S21444C03004F09AF908B100233B600022304BD4E95F
S21444C040260104F091F908B10023336000222C4BFA
S21444C050D4E9280104F088F910B100233B6033602A
S21444C06005B0BDE8F08F012B0BD1264B1968019B18
S21444C07023F00205012DAFD000232160C9F800301B
S21444C080B0E7022B03D11F4B51461868A5E7032B94
S21444C090A8D10023C9F800301A4B1B682360A1E7D7
S21444C0A0601F4020A41F4020301142205C1F4020C7
S21444C0B0B819402014194020B41740208C1840204A
S21444C0C05C1C40207A17402079174020A81740204F
S21444C0D0A4174020A01740209C174020AC174020AF
S21444C0E000004843000048C3581C4020AC1F402072
S21444C0F0B81D402000401C4508194020000E422030
S21444C1000000F03FB41F40205C1B4020A418402091
S21444C110AC19402000000000F8B5174B174C1E68B9
S21444C120174D66B1012E19D000210020F5F7D6FB35
S21444C13000210120F5F7D2FB00232B700CE0267873
S21444C140002EF1D100213046F5F7C8FB0D490120F9
S21444C150F5F7C4FB01232E702370F8BD2F78002F0B
S21444C160E2D108493846F5F7B9FB00213046F5F7E1
S21444C170B5FB2E702770F0E7581C4020E817402087
S21444C180E91740200000C84208B5114B186803F070
S21444C1902BFE0DA3D3E9002304F0FAF890B90D4B17
S21444C1A04FF07E51186804F07FFC003818BF012019
S21444C1B0094B1860094B1B685A1E53425341084AA0
S21444C1C0136008BD0120F3E7666666666666E6BFEA
S21444C1D0201F4020B41F4020941B40205C1C40205D
S21444C1E0801B402008B5FFF7CFFF104B1A68104B52
S21444C1F01A60104B1A68104B1A60104B1A68104B92
S21444C2001A60104B1A68104B1A60104B1A68104B81
S21444C2101A60104B1A68104B1A60104B1A68104B71
S21444C2201A60104B1A68104B1A6008BD5C1A4020FE
S21444C230741B4020741A40208C1B4020701A4020E7
S21444C240881B4020601A4020781B4020781A4020E3
S21444C250901B40206C1A4020841B4020641A4020C7
S21444C2607C1B4020581A4020701B402008B5FFF71E
S21444C2708BFF104B1A68104B1A60104B1A68104B01
S21444C2801A60104B1A68104B1A60104B1A68104B01
S21444C2901A60104B1A68104B1A60104B1A68104BF1
S21444C2A01A60104B1A68104B1A60104B1A68104BE1
S21444C2B01A6008BD601D4020741B4020781D402035
S21444C2C08C1B4020741D4020881B4020641D402049
S21444C2D0781B40207C1D4020901B4020701D402031
S21444C2E0841B4020681D40207C1B40205C1D402051
S21444C2F0701B402000230B4A012113600A4A136036
S21444C3000A4A13600A4A13600A4A13600A4A1360C8
S21444C3100A4A13600A4A13600A4A11600A4A1360BA
S21444C320704700BF941B4020901B40208C1B40202D
S21444C330881B4020841B4020801B40207C1B4020C0
S21444C340781B4020741B4020701B402002230B4A5D
S21444C35013600B4A136000230A4A13600A4A1360A8
S21444C3600A4A13600A4A13600A4A13600A4A136068
S21444C3700A4A13600A4A1360704700BF941B402061
S21444C380901B40208C1B4020881B4020841B402050
S21444C390801B40207C1B4020781B4020741B402080
S21444C3A0701B40202C4B2D491A6810B542B90A68B8
S21444C3B0012A05D12A4802602A4802602A480260B7
S21444C3C02A4A502010602A4A2A4810602A4A12688C
S21444C3D01A602A4B1B780B60294B1C6874B9294B8E
S21444C3E00021186804F042FB88B1274B07221A60E4
S21444C3F00122264B1C60264B1A6008E0012C07D10C
S21444C4000223214A1360214A1360214A136010BD57
S21444C410022C0FD11B4B0021186804F027FB002880
S21444C420F5D0194B03221A600022184B1A60184B99
S21444C4301C60ECE7032CEAD1124B0021186804F088
S21444C44015FB0028E3D0104B04221A6001220F4B40
S21444C4501A6002220E4BCFE73C1B4020381B40207C
S21444C460481B40204C1B4020541B4020341B40207B
S21444C470301B4020000048C2FC1940201E1E4020AD
S21444C4805C1C4020781C4020441B4020401B40201D
S21444C490641B40200000000038B5174B00211C6880
S21444C4A0204604F0EDFA08B104F10044134D20464A
S21444C4B02C6003F099FC0CA3D3E9002303F016FE8A
S21444C4C00BA3D3E9002303F0E7FC00220C4B03F054
S21444C4D0E3FC0C4B002203F009FE03F0D5FF0A4BA5
S21444C4E06860186038BD00BF5C8FC2F528DC274002
S21444C4F0B4A766033D39FB3F701E40200021402010
S21444C50000004E4000408F40781C402008B5074B42
S21444C510186804F0BFF8064B0649186004F0BAFAE7
S21444C52010B1054B01221A7008BD00BF181E4020EA
S21444C530501840200000F04154184020FE28D4BF34
S21444C54001300020704770B50022FF23064ED4B257
S21444C550551C8C4202D3D843C0B270BD025D5340D2
S21444C5602A46F35CF3E700BF408E460007210130BD
S21444C57008B5FFF7E8FFC0B208BDB0F5447F38B54C
S21444C580144617D1244D204695F8FC32FF2B14BF91
S21444C59001330023DBB285F8FC3253701F4A137014
S21444C5A0FFF7E4FF1E4BC0B285F8FD0220701870FA
S21444C5B0012038BD402818D0B0F5547FF8D1164D28
S21444C5C0204695F8F832FF2B14BF01330023DAB225
S21444C5D085F8F8226270134A1360FFF7C7FFC0B2AB
S21444C5E0114B85F8F902207014E00B4D204695F85F
S21444C5F0F032FF2B14BF01330023DAB285F8F02261
S21444C60062700A4A1360FFF7B1FF094BC0B285F85F
S21444C610F10220701860CBE7D08340203B194020BD
S21444C6203A1940203419402030194020C01940207F
S21444C630BC194020402838B5144616D1254D20460E
S21444C64095F82833FF2B14BF01330023DAB285F85C
S21444C65028236270204A1360FFF788FF1F4BC0B23E
S21444C66085F829032070186005E0B0F5547F04D09F
S21444C670B0F5447F17D0012038BD164D204695F8B6
S21444C6803033FF2B14BF01330023DAB285F830234E
S21444C6906270134A1360FFF769FFC0B2114B85F806
S21444C6A031032070DFE70B4D204695F83433FF2BDB
S21444C6B014BF01330023DBB285F8343353700A4A7F
S21444C6C01370FFF753FF094BC0B285F8350320704B
S21444C6D01870D0E7D08340201C19402018194020F9
S21444C6E0C4184020C0184020CB184020CA18402008
S21444C6F0402838B5144617D1254D204695F828339A
S21444C700FF2B14BF01330023DAB285F8642362702A
S21444C710204A1360FFF72AFF1F4BC0B285F8650313
S21444C72020701860012038BDB0F5547F18D0B0F59D
S21444C730447FF7D1164D204695F87033FF2B14BF2F
S21444C74001330023DBB285F870335370134A1370F9
S21444C750FFF70CFFC0B2124B85F87103207014E04B
S21444C7600B4D204695F86C33FF2B14BF0133002342
S21444C770DBB285F86C3353700A4A1370FFF7F6FE43
S21444C780094BC0B285F86D0320701870CAE700BF25
S21444C790D0834020AC184020A8184020A018402041
S21444C7A09F1840209C1840209B184020402838B5AD
S21444C7B0144616D1254D204695F87433FF2B14BFE6
S21444C7C001330023DAB285F874236270204A13607A
S21444C7D0FFF7CCFE1F4BC0B285F875032070186077
S21444C7E005E0B0F5547F04D0B0F5447F17D001205F
S21444C7F038BD164D204695F88033FF2B14BF0133C1
S21444C8000023DAB285F880236270134A1360FFF778
S21444C810ADFEC0B2114B85F881032070DFE70B4DA7
S21444C820204695F87C33FF2B14BF01330023DBB23C
S21444C83085F87C3353700A4A1370FFF797FE094B0A
S21444C840C0B285F87D0320701870D0E7D0834020AE
S21444C8509418402090184020801840207C1840208F
S21444C8608718402086184020502870B50546144640
S21444C87016D18C4A92F8B431FF2B14BF01330023EF
S21444C880D9B282F8B411884A2171136040F28533D4
S21444C8909D4200F0DD80162D00F0F080012070BD32
S21444C8A0642826D065283BD032284FD0702863D0E1
S21444C8B0712877D0332800F08C806A2800F09F8057
S21444C8C0B0F5617FE2D1774D204695F80033FF2BD3
S21444C8D014BF01330023DBB285F800335370734A28
S21444C8E01370FFF743FEC0B2714B85F80103207006
S21444C8F06DE06C4E204696F8B832FF2B14BF0133D9
S21444C9000023DBB286F8B83253706A4A1370FFF7D6
S21444C9102DFE694BC0B286F8BC0220701870B5E78D
S21444C920604E204696F82033FF2B14BF0133002375
S21444C930DBB286F820335370604A1370FFF716FE56
S21444C940C0B25F4B86F824032070E7E7554E204676
S21444C95096F8D032FF2B14BF01330023DBB286F89F
S21444C960D0325370574A1370FFF700FEC0B2564B8E
S21444C97086F8D1022070D1E74A4E204696F8C43253
S21444C980FF2B14BF01330023DBB286F8C432537046
S21444C9904E4A1370FFF7EAFDC0B24D4B86F8C50207
S21444C9A02070BBE73F4D204695F81433FF2B14BF49
S21444C9B001330023DBB285F814335370454A1370B1
S21444C9C0FFF7D4FD444BC0B285F8150320701870A9
S21444C9D064E7344D204695F83833FF2B14BF0133B3
S21444C9E00023DBB285F8383353703C4A1370FFF7A4
S21444C9F0BDFDC0B23A4B85F839032070E7E7294DB0
S21444CA002046D5F8E832D5F8E822C3F3C733FF2BDF
S21444CA1014BF01330023DBB263F3D632C5F8E822F1
S21444CA206370D5F8E8322F4AC3F3C7331360FFF771
S21444CA309DFDB5F8EA32C0B22B4A60F3CE13A5F892
S21444CA40EA322070B5F8EA32C3F3C713136025E719
S21444CA50144D2046254A95F85033FF2B14BF013316
S21444CA600023DBB285F8503363701370FFF77EFD06
S21444CA70C0B21F4B85F851032070A8E70949B1F8A6
S21444CA809C22C2F34313013303F00F0363F34812AB
S21444CA90A1F89C226370B1F89C32164AC3F3431340
S21444CAA0D4E700BFD08340202C1C40202C194020C3
S21444CAB02B1940207C1940207D1940201019402015
S21444CAC011194020C6194020C51940205D19402040
S21444CAD05C194020ED184020EC18402022194020D4
S21444CAE021194020701940206C194020B918402064
S21444CAF0B8184020C41A40200F28D4BF0130002064
S21444CB00704770B50022FF23074ED4B2551C8C42A2
S21444CB1005D3DB4383EA131303F00F0070BD025DB5
S21444CB2053402A46F35CF0E7408F46000721013025
S21444CB3008B5FFF7E6FFC0B208BDB0F5AE6F70B5F6
S21444CB40054614461AD1C04D204695F811221309BD
S21444CB50013363F3071203F00F0385F81122BB4A2F
S21444CB601360FFF7E3FF95F8123260F3030300F017
S21444CB700F0085F81232B64B1860C0E0B0F5B06FBF
S21444CB801DD0B0F5B26F35D1AF4D204695F8222270
S21444CB9002F00F03013363F3030203F00F0385F837
S21444CBA02222AC4A1360FFF7C1FF95F8223260F3A5
S21444CBB0071300F00F0085F82232A74BDCE7A24D9E
S21444CBC02046B5F81822C2F38313013363F389125F
S21444CBD003F00F03A5F81822A04A1360FFF7A6FF38
S21444CBE095F8193260F3850300F00F0085F8193282
S21444CBF09B4BC1E740F29553984222D040F285536E
S21444CC00984258D050287CD0512835D18E4D204655
S21444CC1095F83C2202F00F03013363F3030203F05A
S21444CC200F0385F83C228F4A1360FFF77FFF95F881
S21444CC303C3260F3071300F00F0085F83C328A4B11
S21444CC409AE7814E204696F82722C2F3830301339F
S21444CC5003F00F0363F3850286F82722834A137092
S21444CC60FFF764FF96F8283200F00F0060F30303E2
S21444CC7086F828327E4B1870602D5DD0612D35D1F4
S21444CC80714D204695F84C2202F00F03013363F3AE
S21444CC90030203F00F0385F84C22764A1360FFF72D
S21444CCA045FF95F84C3260F3071300F00F0085F803
S21444CCB04C32714B60E7644E2046D6F82C22C2F3C1
S21444CCC08333013363F3913203F00F03C6F82C2207
S21444CCD06A4A1360FFF72AFF96F82E3260F38503FC
S21444CCE000F00F0086F82E32654B1860132D3ED0A8
S21444CCF0142D57D0152D70D0162D00F089800120A4
S21444CD0070BD514D204695F8342202F00F0301338E
S21444CD1063F3030203F00F0385F83422594A136081
S21444CD20FFF704FF95F8343260F3071300F00F0062
S21444CD3085F83432544B1FE7434D204695F8442239
S21444CD4002F00F03013363F3030203F00F0385F885
S21444CD5044224E4A1360FFF7E9FE95F8443260F3E6
S21444CD60071300F00F0085F84432494B04E7364D6C
S21444CD702046B5F85622C2F38313013363F389126F
S21444CD8003F00F03A5F85622424A1360FFF7CEFE7F
S21444CD9095F8573260F3850300F00F0085F8573254
S21444CDA03D4BE9E6284D204695F85E2202F00F03F7
S21444CDB0013363F3030203F00F0385F85E22374A18
S21444CDC01360FFF7B3FE95F85E3260F3071300F086
S21444CDD00F0085F85E32324BCEE61B4D204695F862
S21444CDE0662202F00F03013363F3030203F00F03DA
S21444CDF085F866222B4A1360FFF798FE95F866324C
S21444CE0060F3071300F00F0085F86632264BB3E64E
S21444CE100D4D2046B5F89C22C2F34313013363F309
S21444CE20481203F00F03A5F89C22204A1360FFF72C
S21444CE307DFE95F89D3260F3440300F00F0085F8BC
S21444CE409D321B4B98E600BFD0834020101A4020EA
S21444CE500C1A4020341E4020301E4020EC1D40203A
S21444CE60E81D4020A41A4020A01A4020DB19402088
S21444CE70DA194020841A4020801A4020E4194020C1
S21444CE80E0194020B41A4020B01A4020941A40209A
S21444CE90901A4020041B4020001B4020E41A4020E7
S21444CEA0E01A4020CC1A4020C81A4020C41A402019
S21444CEB0C01A40200D4B0E490E4810B51C680E4B48
S21444CEC01A78A2421A460BD10B8801339BB2312BF7
S21444CED00B8008D932230B8001230370147010BDD5
S21444CEE000230B80F9E70023F7E700BF581D4020D6
S21444CEF09817402080174020881740200D4B0E4935
S21444CF000E4810B51C680E4B1A78A2421A460BD12E
S21444CF100B8801339BB2312B0B8008D932230B800C
S21444CF2001230370147010BD00230B80F9E700231F
S21444CF30F7E700BFB41D4020961740207F174020D7
S21444CF40871740200D4B0E490E4810B51C680E4BF3
S21444CF501A78A2421A460BD10B8801339BB2312B66
S21444CF600B8008D932230B8001230370147010BD44
S21444CF7000230B80F9E70023F7E700BFA41D4020F9
S21444CF80941740207E174020861740200D4B0E49AC
S21444CF900E4810B51C680E4B1A78A2421A460BD19E
S21444CFA00B8801339BB2312B0B8008D932230B807C
S21444CFB001230370147010BD00230B80F9E700238F
S21444CFC0F7E700BF881D4020921740207D17402079
S21444CFD08517402008B5FFF76DFFFFF78FFFFFF773
S21444CFE0B1FFBDE80840FFF7D1BF0D4B0D490E48D1
S21444CFF010B51C780D4B1A78A2421A460BD10B88F2
S21444D00001339BB2312B0B8008D932230B8001238A
S21444D0100370147010BD00230B80F9E70023F7E774
S21444D020101D402090174020281C40208417402084
S21444D0300D4B0E490E4810B51C780E4B1A78A2427A
S21444D0401A460BD10B8801339BB2312B0B8008D97F
S21444D05032230B8001230370147010BD00230B8011
S21444D060F9E70023F7E700BF9C1C40208E174020BA
S21444D070271C4020831740200D4B0E490E4810B500
S21444D0801C680E4B1A78A2421A460BD10B88013301
S21444D0909BB2312B0B8008D932230B8001230370BB
S21444D0A0147010BD00230B80F9E70023F7E700BF98
S21444D0B0541D40208C174020261C402082174020B8
S21444D0C00D4B0E490E4810B51C680E4B1A78A242FA
S21444D0D01A460BD10B8801339BB2312B0B8008D9EF
S21444D0E032230B8001230370147010BD00230B8081
S21444D0F0F9E70023F7E700BFD01C40208A174020FA
S21444D100251C4020811740201D4B1B78012B30D115
S21444D1101C4B1B78003B18BF01231B4A13701B4B48
S21444D1201B78012B27D1174B1B78003B18BF0123D4
S21444D130174A1370174B1B78012B1ED1114B1B78C3
S21444D140003B18BF0123144A1370144B1B78012B61
S21444D1500CD0134B1B78012B08D0124B1B78012B99
S21444D16004D0114B1B785A1E534253410F4A137036
S21444D17070470023D1E70023DAE70023E3E700BF44
S21444D180661F4020A81740202A1C4020651F4020C8
S21444D190291C4020641F4020241C40208017402027
S21444D1A07F1740207E1740207D1740207C17402064
S21444D1B00B4B1B68012B09D10A4A11680A4A1068AE
S21444D1C088420ABF094A116013607047022B06D191
S21444D1D0074B1B68012B02BF044B00221A607047A2
S21444D1E0581C4020701F4020941F40208C1F402015
S21444D1F07C1F40202C4B1B68012B10B52B4C0FD0AA
S21444D2002B4B1B88012B0BD02A4B1B68012B07D0BA
S21444D210294B1B68012B03D0284B1B78012B05D1C7
S21444D22002232360BDE81040FFF7D4BE244B1B689E
S21444D230013B022B0AD80323224A00212360002301
S21444D2401370214A1160214A137010BD204A214BA5
S21444D25012681B68012A22D11F4A1278012A1ED15D
S21444D260012B226805D12368032BEED101232360CA
S21444D270EBE7032AE9D1FFF7ADFE184B1B78012BE9
S21444D280E3D0174B1B78012BDFD0164B1B78012BB2
S21444D290DBD0154B1B78012BD7D00023E7E7012BB7
S21444D2A0E1D00323E3E700BF7C1F4020581C402006
S21444D2B0041840208C1D40208C1F4020A817402076
S21444D2C0241E4020251840205C1B40202418402063
S21444D2D09C1D4020881F4020741F402080174020FB
S21444D2E07F1740207E1740207D1740201A4B1A781F
S21444D2F01A4B1B7813432DD1194B1B78013B18BF8F
S21444D3000123184A1370184B184A1B68003B18BF71
S21444D31001231370164B1A78164B1B781343164B7F
S21444D32014BF012200221A70144B154A1B78013B85
S21444D33018BF01231370134B134A1B78003B18BFC6
S21444D34001231370114B124A1B78003B18BF01236C
S21444D350137070470123D4E7E61D4020E51D4020A6
S21444D3601C1E402067184020901E40206418402011
S21444D370D51D4020D41D4020651840201D1E402049
S21444D380661840201E1E402063184020281E402059
S21444D3906218402038B52A4B2A4D1B68012B30D1E1
S21444D3A0294B1C68294B012C1B6814D1002B42D1F5
S21444D3B0274B4FF07E51186803F06CFB00283AD098
S21444D3C0244B0021186803F051FB002833D02C600E
S21444D3D0214B1C7038BD1C432DD11D4B4FF07E5144
S21444D3E0186803F057FB30B31A4B0021186803F053
S21444D3F03DFB00B32C60194B1C68003C18BF01244D
S21444D400E6E7C3B9164B1C68164B012C1B6810D1B3
S21444D4108BB90F4B4FF07E51186803F03BFB50B16D
S21444D420114B0021186803F021FB20B10B4B1C6004
S21444D43001E01C43EDD02B68002BDCD00124C7E769
S21444D440581C4020641C4020781F40209C1F4020CD
S21444D450781C4020A01F402078174020141B4020F2
S21444D460981D4020C01D4020BC1D402038B50124D6
S21444D470204B00251C70204B1C70204B1C70204BEE
S21444D4801C70204B1D70204B1D70204B1C70204B75
S21444D4901C70204B1D70204B1D70204B186803F0E9
S21444D4A017FB1F4B18601F4B1C601F4B1C601F4B09
S21444D4B01C601F4B1A681F4B1A6015221E4B1C70AB
S21444D4C01E4B1C701E4B1C701E4B1C701E4B1D703E
S21444D4D01E4B1D701E4B1A7006221E4B1D701E4B93
S21444D4E01D701E4B1A7018221D4B1D701D4B1A7052
S21444D4F038BD00BFC41940202019402039194020A7
S21444D50038194020C9184020C81840209D1840208B
S21444D5109E18402084184020851840205C1B4020DC
S21444D520A8194020A419402094194020F8184020F7
S21444D5305C1C402000194020B41940201219402099
S21444D540A1184020881840202A1940202919402034
S21444D5502819402027194020261940202519402004
S21444D5602419402023194020064B01221A70064BEA
S21444D5701B78934204D1054A13707822044B1A80D0
S21444D580704700BF2B1B4020631840202A1B4020B6
S21444D590281B402008B5FFF7E7FFFEF767FE054B5C
S21444D5A01B68012B1EBF044B00221A60BDE80840CE
S21444D5B0FFF710BD8C1D4020081B402008B5FFF720
S21444D5C0D3FFFEF70FFE064B1B68012B1EBF054B11
S21444D5D000221A60044B1A68044B1A6008BD00BF48
S21444D5E07C1F4020601C4020681F4020741C402044
S21444D5F00D4B1A780D4B32B90D4A1278012A02BFE8
S21444D6001A8801321A801A88B2F5FA7F06D30022A5
S21444D6101A80074B1A700522064B1A700023064AD6
S21444D6201370064A13807047621840201A18402028
S21444D6302B1B4020681840202A1B4020281B4020D3
S21444D64008B5FFF7D5FFFEF755FE0023024A1360E0
S21444D650024A136008BD00BF601C4020081B4020DF
S21444D66038B5134A0223134D1360134A134C136000
S21444D67001232B602360FFF7BBFFFEF767FE104BCA
S21444D6801B88A3B90F4B104A1B68126813430F4AF2
S21444D690126813430BD10E4B1B7843B90D4A2B60CB
S21444D6A013600D4A2360136003220C4B1A6038BD86
S21444D6B0641B4020601C40205C1C4020081B40200B
S21444D6C0041840207C1F40208C1D40208C1F402086
S21444D6D0A8174020941B4020901B4020581C4020F4
S21444D6E008B5FFF7C3FEFFF785FDFEF7FFFAFCF724
S21444D6F0DFF9FEF7E3FB0C4B1B78032B13D8DFE86C
S21444D70003F002060A0EBDE80840FFF743BFBDE833
S21444D7100840FFF753BFBDE80840FFF7A1BFBDE888
S21444D7200840FFF78DBF08BD581C402010B5314C4B
S21444D730FFF7DCFD2378052B5AD8DFE803F0031601
S21444D74038474F5300F078F8FEF7E0FE2A4B1B7834
S21444D750012B3AD1294A1178294A12780A4334D1FE
S21444D760284A1360284A137018E0274B1A78511E2B
S21444D7704B424B4125490B7025490B7025490B708C
S21444D78025490B70254B1B78012B254B08D1012AC4
S21444D79006D11A700022234B1A700223237014E019
S21444D7A000221A70144B1B787BB90323F6E7FFF765
S21444D7B097FFFEF7F7FDFEF76FFE0F4B1B7823B976
S21444D7C0194B1B68023B012BEFD910BD174B0022A7
S21444D7D01A800122164B1A700423DFE7BDE8104076
S21444D7E0FFF706BF134B1B88042BEED80023B9E77C
S21444D7F00023D3E768184020691840206718402063
S21444D80063184020501B40202C1B40206E1840209C
S21444D8106D1840206C1840206B184020701840202B
S21444D8207518402072184020581C40201A18402072
S21444D83074184020C61D4020074B1A2206211A6041
S21444D8400123064A1360064A1160064A1360064BD3
S21444D850064A1A60704700BFA81B4020A41B4020FD
S21444D860A01B40209C1B4020981B4020EFAB03008D
S21444D8707047704730B53D4C85B03D48237801A984
S21444D8800193019B1B020193019A6378134401930D
S21444D890019B1B020193019AA37813440193019BB5
S21444D8A01B020193019AE37813440193237902936C
S21444D8B0029B1B020293029A637913440293029BCF
S21444D8C01B020293029AA37913440293029B1B02FF
S21444D8D00293029AE37913440293237A0193019BB9
S21444D8E01B020193019A637A13440193019B1B0222
S21444D8F00193019AA37A13440193019B1B0201935B
S21444D900019AE37A13440193237B0293029B1B02FE
S21444D9100293029A637B13440293029B1B02029374
S21444D920029AA37B13440293029B1B020293029A1D
S21444D930E37B1344029342F21273019342F213734D
S21444D940029300F0B0FB04F1100004F1080104F166
S21444D9501802082314F8015B013B00F8015B11F838
S21444D960015B02F8015BF5D105B030BDF8114220E9
S21444D970808080000C4A0823002102F1280030B43D
S21444D98002F1080502F12004013B02F8011B05F8E8
S21444D990011B13F0FF0304F8011B00F8011BF3D12D
S21444D9A030BCFFF767BF00BFF81142204F4BF0B5BD
S21444D9B01B688BB002934E4B1A6803925A680492C3
S21444D9C09B68059342F21273029A9A4200F0898049
S21444D9D0484800F013FBFFF7CDFF002346480AAA49
S21444D9E050F8231002EB83020133082B42F8201C24
S21444D9F0F5D1002340480AAA50F8231002EB8302CC
S21444DA000133082B42F8201CF5D102990025039ACD
S21444DA10049B0598394C00903948264600F0EEFAA7
S21444DA20029B38481B0E2370029B1B0C6370029BA0
S21444DA301B0AA370029BE370039B1B0E2371039B7C
S21444DA401B0C6371039B1B0AA371039BE371049B2A
S21444DA501B0E2372049B1B0C6372049B1B0AA3724B
S21444DA60049BE372059B1B0E2373059B1B0C63737D
S21444DA70059B1B0AA373059BE37300F0B6FA0135B6
S21444DA8016F8010B00F0DAFA082DF8D11E4D0026E0
S21444DA9000F0CBFA1D482F4600F0A7FA013617F8D7
S21444DAA0010B00F0CBFA082EF8D100F0BEFA184B62
S21444DAB0002203F1080703F1100003F1180194460D
S21444DAC0013214F8016B15F801EB082A03F8016BD0
S21444DAD007F801EB00F8016B01F801CBF0D10BB06D
S21444DAE0F0BD0C4800F08AFA77E700BF80808000DB
S21444DAF084808000A295460010808000F811422061
S21444DB00C6954600E395460000124220ED95460031
S21444DB1008124220B8954600194A08211948F0B51B
S21444DB2092F8A53100F1100C00F1080500F1180731
S21444DB30012B9CBF002382F8D431002310F8014BFC
S21444DB4001391CF8016B17F801EBB4422E7818BF64
S21444DB50013344EA060418BFDBB2764505F8014BA8
S21444DB601CBF0133DBB211F0FF01E7D133B1B2F889
S21444DB70BE301BB9BDE8F040FFF77CBEF0BD00BF29
S21444DB8034124220F81142201FB5144B01A953F811
S21444DB9020305A1E073312F8010F9A4201F8010B3F
S21444DBA0F9D19DF804300024502B8DF80C4007D052
S21444DBB0432B0CD0422B0DD0552B08BF4FF44004BA
S21444DBC00DF1050000F04CFA204404B010BD4FF4AB
S21444DBD08004F5E74FF40004F2E700BF0821402034
S21444DBE02DE9F04F5C4D8DB082462B6805F1080850
S21444DBF006AC09A963F07C4340462E46A9462B60F2
S21444DC004246082316F8017B013B04F8017B9BB28D
S21444DC1010F8017B01F8017B002BF3D1BAF10A0F0F
S21444DC200BD141464C4C0823FF20013B04F8010B22
S21444DC3001F8010B9BB2002BF7D1484BC8240021B6
S21444DC40013C03F8011BA4B2002CF9D126464449F2
S21444DC50DFF808B104F1080380279BB200932B78C1
S21444DC601F4203D198F800301F4248D051F8243060
S21444DC700DF10C0C581E073310F801EF98420CF8BF
S21444DC8001EBF9D14FF000038DF814309DF80C30B9
S21444DC90502B59D0432B59D0422B5AD0552B34D1E4
S21444DCA04FF440030DF10D00019300F0D9F9019BA8
S21444DCB095F800C0184498F800302A4A3B404FEA8A
S21444DCC0102E274918BF082317EA0C0F4FEA104CAA
S21444DCD018BF43F001030BF806C006F1010C1FFA07
S21444DCE08CFC0BF80CE006F1020C1FFA8CFC0BF8CB
S21444DCF00C00F01C043680B2B6B20BF80030013487
S21444DD00009B7F08A4B2A342A9D1013508F10108BB
S21444DD1095429FD1BAF10A0F0FD19DF81A30BDF83B
S21444DD20182089F80230A9F800209DF82630BDF85E
S21444DD30242089F80A30A9F80820084B00223046E7
S21444DD409A550DB0BDE8F08F0023ABE74FF480033F
S21444DD50A8E74FF40003A5E7F81142203E224020EE
S21444DD600821402000124220F0B50D4C0822002025
S21444DD7004F1080514F8016B082380210E4202D1F1
S21444DD802F78394201D0013080B2013B49089BB21A
S21444DD90002BF3D1013A013592B2002AEAD1F0BD04
S21444DDA0F81142202DE9F04FDFF8B480002685B004
S21444DDB08346A8F1080A3446284B022E4FF08009C1
S21444DDC04FF0000234BF082703272744BFB29AF80F
S21444DDD0001019EA010F04D198F8001019EA010F4F
S21444DDE02DD053F8241001AD481E073110F801CF4A
S21444DDF0814205F801CBF9D19DF804108DF80C202A
S21444DE00502914D0432914D0422915D055291CD161
S21444DE104FF440050DF1050000F022F905440F4B80
S21444DE2000225D450BD1E0B205B0BDE8F08F002579
S21444DE30F0E74FF48005EDE74FF40005EAE70134D8
S21444DE404FEA5909A4B2A742C1D1013608F10108E4
S21444DE500AF1010A082EB0D1FF20E5E70821402048
S21444DE60001242202DE9FF4700240746204EA146D3
S21444DE70022C4FF0000834BF4FF0080A4FF0030A54
S21444DE80336801A95A1E073312F8010F9A4201F863
S21444DE90010BF9D19DF804308DF80C90502B0DD021
S21444DEA0432B15D0422B16D0552B17D001340436AD
S21444DEB0082CDDD1FF2004B0BDE8F08700250DF125
S21444DEC0050000F0CDF80544BD420AD1E0B2F2E7C1
S21444DED04FF48005F3E74FF40005F0E74FF44005B0
S21444DEE0EDE708F101081FFA88F39A45C8D8DDE73C
S21444DEF0082140202DE9F04FDFF8C490002585B076
S21444DF008346A9F108082C462B4A022D4FF0800A76
S21444DF104FF0000134BF082703272744BFB298F8C0
S21444DF2000001AEA000F04D199F800001AEA000F1C
S21444DF3032D052F824000DF1040C461E073016F871
S21444DF4001EFB0420CF801EBF9D19DF804008DF8CE
S21444DF500C10502818D0432818D0422819D05528D9
S21444DF6020D14FF440060DF1050000F079F8064440
S21444DF70124B00215E45104A0ED15955E0B21D445D
S21444DF80297205B0BDE8F08F0026ECE74FF4800612
S21444DF90E9E74FF40006E6E701344FEA5A0AA4B22A
S21444DFA0A742BCD1013509F1010908F10108082D41
S21444DFB0ABD1FF20E5E700BF08214020F8114220FE
S21444DFC0001242207047092894BF30303730C0B220
S21444DFD0704707B501220DF107018DF807000020B0
S21444DFE013F052FE03B05DF804FB10B5441E14F85B
S21444DFF0010F00B910BDFFF7ECFFF8E70FB400B50A
S21444E000C3B044AA02A852F8041B019204F06CFC64
S21444E010002302A88DF805318DF80631FFF7E5FF99
S21444E02043B05DF804EB04B070470D2008B5FFF725
S21444E030D0FF0A20BDE80840FFF7CBBF10B5044622
S21444E0400009FFF7C0FFFFF7C4FF04F00F00FFF717
S21444E050BAFFFFF7BEFF2C20BDE81040FFF7B9BF5C
S21444E060002330B51A46441E184614F8011F3929B1
S21444E07008D82F290AD95D1C01F00F0303EB0010C2
S21444E0802B4606E0A1F14105052D06D900B943B15A
S21444E09008220132072AE8D930BD5D1CA1F13703B6
S21444E0A0ECE71D46EAE7002070470000034A92F872
S21444E0B09E30013382F89E30704700BF34124220AF
S21444E0C010B52A4C94F89A30642B94BF013300233D
S21444E0D084F89A3094F8C63043B1013BDBB284F8F6
S21444E0E0C6301BB984F8C53084F88A3194F8C730F2
S21444E0F053B1013BDBB284F8C7302BB994F88A217C
S21444E100032A08BF84F88A31B4F8E4315BB1013B92
S21444E1109BB2A4F8E43133B9012284F8CF3184F8B1
S21444E120C13184F8A52194F8C231013384F8C23150
S21444E130FFF7F2FC94F8A13123B1002084F8A10142
S21444E14001F01FFCB4F8BE3073B1013B9BB2A4F897
S21444E150BE304BB984F88A3184F8C53084F8A3318C
S21444E16084F8C13184F8DC3110BD00BF341242203B
S21444E170034A92F89830013382F89830704700BFCB
S21444E1803412422070470323002010B5064CA4F8EE
S21444E190EC3104F154020823E16CF4F7DDFB002370
S21444E1A084F8953010BD00BF34124220024B002242
S21444E1B0C3E91522704700BF3412422030B5224BC3
S21444E1C0002201244FF4FB604FF4FA61082583F8DB
S21444E1D0A541A3F89820A3F8B420C3F8D420A3F804
S21444E1E0CA20A3F8CC2083F88121A3F8822183F89F
S21444E1F08C2183F89C21C3F8A02183F8D62183F888
S21444E200DB2183F8DC21A3F8E42183F8EA21A3F890
S21444E210C220C3F8C420D864196083F89450A3F885
S21444E220C621C3F8D02183F8D421C3E972424FF4FF
S21444E2300C14C3E92E22C3E96122C3F8C04183F813
S21444E240C421C3E92B1030BD34124220144B0022A3
S21444E25093F88D1183F88A21E1B90322A3F8861135
S21444E26083F8542093F8882142F0400283F85520DE
S21444E27093F89C21012A01BF7F2283F8552000226F
S21444E28083F89C21B3F8862152BAA3F8562000227C
S21444E2909A65704746F60362A3F85420E8E700BF41
S21444E2A034124220054B3022A3F854200A2283F825
S21444E2B056200D2283F8C720704700BF34124220F0
S21444E2C0034B012283F8C5200B2283F8C6207047EF
S21444E2D03412422008B5FFF783FC0330284B81B242
S21444E2E0284AC0B207291DD85921C3F8982183F873
S21444E2F0540083F8551093F89E1183F85610FF2166
S21444E30083F85710117883F85810517883F85910C9
S21444E3109178D27883F85A1083F85B200422A3F8C5
S21444E320CA2008BDA3F8CC10090AC3F8982141F0C6
S21444E330100183F8550083F85410592183F8561079
S21444E34093F89E1183F85710FF2183F858101178DC
S21444E35083F859105178927883F85A1083F85B20E2
S21444E3600322A3F8CA20012283F8C520022283F898
S21444E3708A21212283F88C21222283F88821D0E71F
S21444E380341242203E224020024B002283F854207E
S21444E390704700BF3412422038B5CB1C40F6FF7499
S21444E3A09BB2A34228BF2346174C1D0A84F8553017
S21444E3B06223A4F8CC1045F0100584F8580084F87D
S21444E3C05630030A84F85450022163F00F03C4F80D
S21444E3D0982184F857300123A4F8CA301378A4F857
S21444E3E0CA1084F85930537884F85A300323A4F872
S21444E3F0CA30937884F85B30FFF762FF212384F8B1
S21444E4008A1184F88C3138BD34124220F0B5C84C99
S21444E41087B094F8C2310133DAB21B064ABF0023F0
S21444E42084F8C22184F8C231B4F8C63113B1013B32
S21444E430A4F8C63194F8A03123B1002384F8A0315F
S21444E440FFF798FA94F88A51012D40F0288194F801
S21444E45088312E2B3DD146F60362A4F854206289B7
S21444E460A4F8562094F88D210D2A0BD1002384F865
S21444E4708A31012384F8953040F2F513A4F8BE306F
S21444E48007B0F0BD0E2AF4D194F88911A948049136
S21444E490A9490391B4F8CA10CDE9012194F8C520DE
S21444E4A029460092B4F88421FFF7A8FD94F88931F0
S21444E4B0012B03D1002001F064FAD7E7022B03D1E5
S21444E4C0002001F079FAD1E7FF2BCFD184F8CB5165
S21444E4D0CCE7222BCAD1B4F88431B3F5A06F6BD104
S21444E4E0964D0022964915F8010B134601321F2813
S21444E4F092B204D9322A01F8010BF4D11346E21839
S21444E5002C213A2082F8E4105A1C422114FA82F252
S21444E51082F8E4109A1C4F2114FA82F282F8E4102E
S21444E520DA1C14FA82F282F8E4101A1D542114FA02
S21444E53082F282F8E4105A1D562114FA82F282F8C6
S21444E540E410991DDA1D14FA81F192B281F8E400C0
S21444E5507C49087842281FD022444E2182F8E41091
S21444E56003F10802302114FA82F282F8E41003F12F
S21444E5700A010933202289B214FA83F383F8E4208B
S21444E5806318002201314FF4A06083F8E42089B276
S21444E5906B4AFFF701FF6CE70B466B4D1878114644
S21444E5A001321F2892B2EBD901332144AB4281F8A1
S21444E5B0E400F3D11146E3E7644EB4F8862106EB53
S21444E5C04316B4F886C14FEA122E3789D0B29CFA65
S21444E5D09CFCF268FB1C99B2DBB207292FD984F85D
S21444E5E05530C1F30321622384F857E041F010010B
S21444E5F084F8580084F85630002384F854100221D6
S21444E600A4F8CA30C4F89821A4F8CC701378A4F8B7
S21444E610CA5084F859305378A4F8CA1084F85A304B
S21444E620937884F85B300323A4F8CA30FFF748FE97
S21444E630322384F88A1184F8C630212374E0622198
S21444E64084F85430A4F856C0013384F85510002199
S21444E650C4F89821DBB2A4F8CA10A4F8CC70107899
S21444E660A4F8CA5084F85800507884F85900022018
S21444E670A4F8CA00907884F85A000320A4F8CA0084
S21444E680D27884F85B200422A4F8CA20DAB2082A96
S21444E6903FF4ECAEE218013382F85410F6E7022D4C
S21444E6A07FF4EEAE94F8C530002B7FF4E9AE94F8D0
S21444E6B08831222B7FF4DDAE94F8C430012B06D982
S21444E6C0023BDBB284F8C430002B7FF4D9AE94F816
S21444E6D0C330072194F88C212E27B4F8CC50D4F8B4
S21444E6E09861134884F8C43084F85420B4F8CA3087
S21444E6F001390130AB4238BF16F803C003F10103B9
S21444E7002CBF80F8547080F854C09BB211F0FF01BF
S21444E710A4F8CA30EAD19D4202F10103DBB298BFA5
S21444E72084F88A112F2B88D884F88C31A1E600BF50
S21444E73034124220E6984600CC134220000144009E
S21444E74018134220201040003910400040904600E4
S21444E750FFF75CBE38B51B4C6389A4F89E31FFF7BF
S21444E76013FE94F89E5105F0F703022B05D10123BE
S21444E770002584F89D31284638BD012D0FD145F635
S21444E780061384F85650A4F8543094F89F3184F80D
S21444E7905730FFF7E9FA40BAA4F85800EBE7032DE0
S21444E7A012BF47F6027345F6021384F856504FF0EC
S21444E7B001051BBFA4F854301223A4F8543084F83F
S21444E7C05630D8E73412422008B5FFF7DDFD0B4B30
S21444E7D04CF20252A3F854209A7A012A83F856201F
S21444E7E004D1002283F8D421012008BD022A01D195
S21444E7F00122F7E77F2283F85520F5E734124220BA
S21444E800064B47F60372A3F85420012283F85600B9
S21444E81083F8571083F89C21704700BF3412422077
S21444E820074B93F8D621132A09D093F8A521032A37
S21444E8301FBF7F2283F8D621012283F89C2170478C
S21444E84034124220002310B56B4C84F8D63194F829
S21444E850CE30222B07D194F8D531032B09D013237D
S21444E86084F8D63105E0202B14D194F8D531022B08
S21444E870F5D894F8D63163B147F6037284F8573026
S21444E8800123A4F8542094F8CE2084F89C3184F8CC
S21444E890562010BD102B0BD194F8D531022BDED167
S21444E8A0A37A03F07F03013B022BE2D91223D7E776
S21444E8B0852B12D1A37A013B012B84BF122384F803
S21444E8C0D63194F8D531022B02D0132384F8D631AE
S21444E8D094F8D601FFF7A4FFCBE7272B05D194F88D
S21444E8E0D53103F0FB03022BB8E7192B18D194F863
S21444E8F0D531012BB3D0A27A0A2AF4D0032AF2D017
S21444E900022AAAD0042A08D1062BA8D1A37B012B1D
S21444E910AFD0FF2BADD03123A2E7012AC6D19CE766
S21444E920282B1DD194F8D511A27A032902F07F032F
S21444E93005D0002BC9D0032BC7D0022902D0591EBC
S21444E9400129C2D912F07C0F01D01223BEE7E27A25
S21444E950013A022ABCD90BB1032BB9D13123B5E70E
S21444E960142B1CD194F8D531042B7FF478AFE07A7D
S21444E970A37A00EB0323207B00EB03206FF07F4356
S21444E9809842C4F8D0013FF474AF1C4B98423FF40D
S21444E99070AFFFF767FAFF287FF46BAFBBE73E2BF9
S21444E9A011D194F8D531022B7FF459AFA37A13F0E2
S21444E9B07F0F4FF4FA7318BF1222A4F8E43118BF3D
S21444E9C084F8D62155E7312B09D194F8D531062B56
S21444E9D03FF645AFA37A013B022B9CD849E72E2B42
S21444E9E005D194F8D531022B7FF639AF41E70F2B8A
S21444E9F03FF63FAF112333E734124220FF00400076
S21444EA004FF287139842134B0ED10A290AD100229B
S21444EA1083F8D62193F8D621003A18BF012283F80A
S21444EA20DB2170471322F3E74FF28B12904201D159
S21444EA300429EBE74FF29512904201D10329E5E70A
S21444EA404FF293129042F9D04FF28C129042DED19C
S21444EA500729DBE7341242200B4B024693F90A009F
S21444EA60997A0028B3BF01F07F02012083F855202D
S21444EA700020B8BF9A724FF00102A8BF83F8540032
S21444EA8083F8A521704700BF34124220274B014625
S21444EA9010B593F90A009A7A0028BBBF02F07F02A9
S21444EAA0002001209A729A7A541E022C31D80624E9
S21444EAB083F85510022A4FF0000183F854404FF46F
S21444EAC0997483F85620A3F858404FF0F40483F81A
S21444EAD0571083F85A404FF4FA7483F8A521A3F8E4
S21444EAE0E44112D1124A1278422A06D102F5800233
S21444EAF002F6DF7212784F2A03D0012283F89C2153
S21444EB0003E00122084683F8CA21002283F8CF2175
S21444EB1010BD47F60372A3F8542093F8CE2083F82A
S21444EB205620122283F85720E7E700BF34124220CB
S21444EB302010400010B5214CA37AE07A00EB032065
S21444EB4080B2B0F5754FA4F886010BD14FF4A0639C
S21444EB50A4F884310123002084F88A31222384F8DF
S21444EB60883111E0B0F5704F12D300F0A9FD4FF68E
S21444EB70FF73984209D10223012084F85430637A03
S21444EB8043F0400384F8553010BDA4F88401E1E70F
S21444EB9040F2DF73D4F8E001C01A47F60373A4F8D2
S21444EBA0543018BF012094F8CE3084F856303123C0
S21444EBB084F85730012384F89C31E5E73412422028
S21444EBC02DE9F0414E4C2E23A27AE07A84F888311F
S21444EBD0130900EB0220217B0E2B84F88D3180B282
S21444EBE084F88911A4F886010DD10123002084F805
S21444EBF08A3194F8DB31012B71D1424A626584F83C
S21444EC009C31BDE8F081B0F5704F13D300F0C3FDDE
S21444EC100F230246A4F8840184F88D314FF6FF731F
S21444EC20984204D0384E06EB4013D96921B90323E1
S21444EC3084F8DB310120DCE794F8CF11012901D0B8
S21444EC400223F5E7002084F89C0194F8DB010028B1
S21444EC50F0D19B6894F8D5010333DBB2984207D0D1
S21444EC6013232A4884F8DB1184F8D631FFF7C6F913
S21444EC70B4F884310027DFF89C80042506EB431360
S21444EC80A4F8CA70DA689B68C4F89421A4F8CC3017
S21444EC90B4F8CA3018F8011BD4F89421D154B4F807
S21444ECA0CA30B4F8CC2001339BB29A42A4F8CA3096
S21444ECB0C0D90020FFF7CAFA94F89C3184F8DB7177
S21444ECC043B9B4F8843106EB4313DB69012B08BF20
S21444ECD084F8A131013D15F0FF05D9D1AAE7022BEE
S21444ECE003D10B4B6365012389E7032B01BF03F173
S21444ECF0445303F5391303F57C53636581E700BF3A
S21444ED0034124220037F2E13409046003799460023
S21444ED10037F2E3340124220204B014630B593F9F0
S21444ED200A009A7A0028BBBF02F07F020020012026
S21444ED309A72DA7A02F0FD04012C22D19A7A02F011
S21444ED40FD05012D11D183F8DC5193F8A521012A44
S21444ED504FF0020283F854201AD87F225A72222295
S21444ED609A72002283F8DC2130BD12B983F8DC2184
S21444ED70EBE7022A06BF002083F8DC4183F89C4177
S21444ED80E3E7022A1FBF7F225A7212229A72DCE7F6
S21444ED909A7A83F8551083F85620E5E734124220D1
S21444EDA0704770477047704750B123230549013B6D
S21444EDB000284FEA40009BB2B8BF4840002BF6D12B
S21444EDC0704700BF69696C6CF8B56C4B064693F89F
S21444EDD0A5211C46012A0BD847F60372A3F85420F3
S21444EDE05A7A83F856207F2283F8572001253DE03F
S21444EDF0997A01F0FB05012D4AD1062384F8550083
S21444EE0084F8561084F8543094F8CF31012B2FD11F
S21444EE1001292DD10023A4F8A631A4F8A83194F8EA
S21444EE20A661012994F8A72194F8A83118BF0221B5
S21444EE3084F8582002EB062294F8A90184F8593045
S21444EE4003EB022384F85A0000EB032084F857604F
S21444EE50FFF7AAFF030E84F8A631030C40BA84F8E1
S21444EE60A7310123A4F8A80184F8C1312846F8BD87
S21444EE7094F8C23103F1110284F8A63184F8A7212C
S21444EE8003F12202343384F8A82184F8A931C6E772
S21444EE90022DABD193F8C121012A4FF0000210D0C5
S21444EEA083F8C12147F603720125A3F8542093F84A
S21444EEB0CE2083F89C5183F85620242283F857208A
S21444EEC0D4E783F8C121DA7A93F8A6319A420AD174
S21444EED0227B94F8A7319A4205D1B4F8A821B4F815
S21444EEE00D309A421DD047F603730629A4F85430D1
S21444EEF094F8CE3084F856304FF0350384F85730C3
S21444EF004FF0010384F89C317FF470AF1C4B1B78A0
S21444EF10422B08D001231B4884F89C31FFF76EF837
S21444EF2001E00629F2D094F89C51002D7FF45EAFA0
S21444EF30A37A022784F8556084F8563084F85470CF
S21444EF40FFF721F9A37A062B0ED101230E4884F845
S21444EF50CF7184F8CA31FFF748F80B48FFF745F8F5
S21444EF600948FFF742F881E794F8A531023B012BA4
S21444EF709CBF012384F8CF3178E700BF3412422087
S21444EF80201040004B994600A9994600114B002298
S21444EF9093F89C1183F8D621012904BF7F2183F876
S21444EFA09C2193F8CE2008BF83F85510312A0DD102
S21444EFB093F8D511062903D9132283F8D62103E002
S21444EFC0997A01390229F8D801207047342AFBD1AE
S21444EFD01222F2E73412422070B5674C0025637A59
S21444EFE0264694F8DD2184F8CE30237A84F89C5162
S21444EFF09A4284F8D53101D800200FE0013B062B15
S21444F000FAD8FFF71FFC94F89C31012B0FD1D4F8A3
S21444F010E02140F2DF739A4201D0012070BD94F89B
S21444F020D631113B012BF8D884F89C51E4E7627A38
S21444F03094F8CE30102A43F0400003D1BDE8704027
S21444F040FFF724BD202A03D1BDE87040FFF704BD76
S21444F050852A03D1BDE87040FFF7B6BB2A2B0AD1F8
S21444F060E37A84F8C33146F60223A4F85430A37AEC
S21444F07084F85630D1E7222B04D16220BDE8704094
S21444F080FFF758BD2E2B04D16E20BDE87040FFF725
S21444F09097BD282B04D16820BDE87040FFF73CBEDE
S21444F0A02F2B0ED146F60673344AA4F85430062362
S21444F0B0013B12F8011B13F0FF0382F84B10F7D103
S21444F0C0ABE7142B15D1FFF75FF9D4F8D0016FF0F6
S21444F0D07F43984202D02A4B984207D1012386F8B0
S21444F0E0A03145F20143A6F8543096E7FEF702FFF6
S21444F0F0F7E7272B04D16720BDE87040FFF764BECE
S21444F100192B03D1BDE87040FFF724BB312B0BD13C
S21444F1101C4A0723013B12F8011B13F0FF0382F835
S21444F120DA10F7D1712079E7112B0FD145F202138B
S21444F130A4F85430A37A84F85630FFF724F81248DB
S21444F140FEF753FF1148FEF750FF66E73E2B0FD1FC
S21444F15094F90A10A37A0029FFF64EAF022142F032
S21444F160400284F8563084F8541084F8552054E706
S21444F170FEF79CFF40E700BF341242203E12422076
S21444F180FF0040003D124220559946006A994600C9
S21444F19038B5424C0F2384F88D312546237A217B9B
S21444F1A003F00F02637AE07A03EB022304F1E402ED
S21444F1B001EB0020C4F8942142F2030280B2A4F882
S21444F1C0CC30A4F88A2194F8CE202F2A23D1033BAE
S21444F1D02E22A4F87A019BB284F8882104F22F12D6
S21444F1E0A4F88601A4F8CC3084F87931A37BC4F81B
S21444F1F0942184F831310423627BA4F8CA30E37B3B
S21444F20084F87C2184F82F1184F8302184F8323134
S21444F210FFF748F814E0A4F8860100F051FA4FF6D8
S21444F220FF7398420ED147F603723123A5F8542053
S21444F23095F8CE2085F8D63185F8562085F857308F
S21444F240012038BD164B03EB4013DA69002AEAD096
S21444F2502E22A4F8840184F88821032284F88A2183
S21444F260DA689B68C4F89421A4F8CC300123A4F847
S21444F270CA30637B1370B4F8CA30D4F89421591C4E
S21444F280A4F8CA10A17BD154B4F8CA30D4F8942157
S21444F290591CA4F8CA10E17BD154B9E73412422071
S21444F2A04090460008B51A4B0022197A83F88D21FF
S21444F2B001F00F00597AA3F8842101EB00219A7AD1
S21444F2C0C82983F888211A7B88BFC82183F8E5209B
S21444F2D0A3F8CC10D97A02EB01205A7B83F8E410C9
S21444F2E083F8E6209A7BA3F8860142F2030083F86B
S21444F2F0E720DA7BA3F88A0183F8E820052205484C
S21444F300A3F8CA20C3F89401FEF7CCFF012008BD39
S21444F310341242203E224020184B0022987A83F82A
S21444F320D62183F89C21A0F12E0283F8CE00D1B2D8
S21444F33008291DD840F24912CA40D24312F00102AD
S21444F34016D12E2883F8DB2114D193F8A521012A5F
S21444F35002D993F8CF216AB97E2283F8D62102F1E6
S21444F3607E2202F5381285325A65012283F89C21A2
S21444F370012070470020FFF70BBF00BF3412422025
S21444F380002340F2F51210B5884C84F8983084F87F
S21444F3909C31A4F8BE204FF4FA72C4E915332368AE
S21444F3A0A4F8E421B3F5FA6F17D1431E04F108021A
S21444F3B0073013F8011F984202F8011BF9D14FF4A5
S21444F3C0FA63C4F8E031227A12F0F0032BD1FFF747
S21444F3D003FE002840F08B804CE040F2DF729342FC
S21444F3E020D1037813F0F00F1CD14278A2F1100319
S21444F3F0DBB2182B11D9852A01D03E2A12D140F20D
S21444F400DF736B4AC4F8E031431E073013F8011F1C
S21444F410834202F8011BF9D1D5E7664A22FA03F380
S21444F420DB07ECD410BD102B02D1FFF775FFD0E7F5
S21444F430202B40F08F8094F8CE302E3BD9B206294C
S21444F4405CD84923CB40DB4313F0010356D194F8F0
S21444F4508A1103290ED194F8DD11072910D8B4F87F
S21444F460CA3001391944B4F8CC30994202D2002348
S21444F47084F88A31002384F89C3184F89830D1E7A4
S21444F48094F88B11914205D14B4884F88A31FEF7A3
S21444F490ACFDEFE784F88B210D2284F8C72094F85E
S21444F4A0DB2132B9E218D4F89411507AB4F8CA2061
S21444F4B08854B4F8CA20B4F8CC10013292B29142BF
S21444F4C0A4F8CA2042D894F8DB31012B1AD147F667
S21444F4D00372A4F8542094F8CE2084F856201322BD
S21444F4E084F8572084F89C31002384F8DB3194F860
S21444F4F09C31012B04BF7F2384F85530012384F8C4
S21444F5009530B7E7022B0CD147F60373A4F8543072
S21444F51094F8CE3084F85630332384F85730012399
S21444F520E0E70020FEF792FEB4F88421234B94F8DB
S21444F5309C1103EB42132248DA69012A08BF84F877
S21444F540A12194F8A131FEF759FDCDE70133072BED
S21444F550A5D18FE7302B8DD194F8DD31022B86D997
S21444F560312A03D10B2384F8C63083E794F8C53098
S21444F5705BB9322A09D146F20323A4F85430B4F8CE
S21444F58086315BBAA4F856304CE7A37A0021312A78
S21444F59003F1030384F8C51084F8C610DBB284F87C
S21444F5A0C33084F8C4303FF662AF63E73412422077
S21444F5B03C124220130204017A99460040904600C9
S21444F5C0929946000A4810B5FEF718FD72B64FF0F9
S21444F5D0005308491022084C0848C3E90012FEF7B5
S21444F5E00DFDFAF75EFA2046FEF708FDFBE700BF7E
S21444F5F0A49946007154CA3DCB994600B199460039
S21444F60038B52C4B93F8C8211C4632B9FEF7D6FDC4
S21444F6102948BDE83840FEF7E8BC93F89820002A0D
S21444F6203FD0002293F89D1183F8982081B193F837
S21444F6309E0183F89D21FEF74DFE012384F8953004
S21444F64040F2F513A4F8BE30BDE83840FEF79BBD43
S21444F65093F89550002DF3D1184A13780133DBB252
S21444F660022B01D8137038BD1570FEF7CFFE94F800
S21444F670993094F8C22101330132DBB284F8C221B6
S21444F680042B84F899300CD984F89950FEF718FD69
S21444F690B4F89C30C72B96BF0133A4F89C50A4F80A
S21444F6A09C3094F8CA2194F8CB311343DBD0FFF74F
S21444F6B089FF00BF34124220DA99460004224020D3
S21444F6C04FF22803984218D84FF20F03984259D95C
S21444F6D0A0F57040113817280DD8DFE800F05629F9
S21444F6E02B2D2F3131333537393B3D3F414345454B
S21444F6F047494B4D4F51042070474FF2931398425D
S21444F70045D00CD84FF28713984242D04FF2881215
S21444F7104FF6FF73904214BF1846012070474FF2CD
S21444F72095124FF6FF73904214BF18460220704756
S21444F7300620704707207047082070470920704706
S21444F7400A2070470B2070470C2070470D207047E6
S21444F7500E2070470F2070471020704711207047C6
S21444F76012207047132070471420704715207047A6
S21444F7701620704717207047182070471920704786
S21444F7801A2070474FF6FF707047052070470320D5
S21444F790704700207047FFF793BF1C280146F0B51A
S21444F7A085B037D83F4B420103EB40169C584FF682
S21444F7B0FF739C422ED0F369012B2BD1756804F558
S21444F7C00004B368AD082246009337482B46FEF73C
S21444F7D015FCD6E903639A1E012A1DD8002315E0BA
S21444F7E036F82310023389B2029102990904029131
S21444F7F05088029901440291918889B203910399F1
S21444F80009040391D188039A0A4403929D4206EB65
S21444F8108302E5D805B0F0BD043B012B3FD9002751
S21444F820BD4206EB8701F5D916F827302046023745
S21444F8300834DBB20293029B1B0602934A78029B6F
S21444F84003EB024302938A78029B03EB0223029360
S21444F850CB78029A134402930B79DBB20393039B4F
S21444F8601B0603934A79039B03EB024303938A796B
S21444F870039B03EB02230393CB7902A9039A134415
S21444F8800393FEF710FCCBE756F82310023302919D
S21444F890526803929D4206EB8302F5D8BAE70023EA
S21444F8A0F8E700BF40904600E59946001C2801460C
S21444F8B030B403D92C4830BCFEF7A0BB42012B4BD6
S21444F8C003EB40109B584FF6FF7293421FD0C26919
S21444F8D0012A1CD10169072919D0826803F500035F
S21444F8E0C468881E012814D8520802340021914264
S21444F8F00DD253F8040B050C24F8025C4D1C9542BB
S21444F90005D2023180B28A4224F8040BEFD830BCC8
S21444F91070470439012925D822F003022244944230
S21444F920F5D053F8041B44F8041BF8E75858050E62
S21444F93025704D1CAA42EAD9C0F3074565708D1C54
S21444F940AA42E4D9C0F30725A570CD1CAA42DED945
S21444F9500431C0B204348A4204F8010CD7D9914227
S21444F960E4D3D4E70021FAE7069A460040904600DE
S21444F97010B50024A0B20134FFF798FF1D2CF9D12E
S21444F98010BD1FB50024A0B20134FFF706FF1D2C9E
S21444F990F9D1074B02A902934FF47C730393054BAA
S21444F9A001930198FEF77FFB002004B010BD00BF12
S21444F9B055EFCDAB1000800008B508B9FFF7D8FF67
S21444F9C0002008BD124B00B51B688BB00293114B48
S21444F9D01A6803925A6804929B6805930299039A9C
S21444F9E0049B059800900C48FEF708FB039BB3F570
S21444F9F07C7F06D10948FEF701FB01200BB05DF879
S21444FA0004FB0748FEF7FAFA4FF0FF30F6E700BF6C
S21444FA101000800014008000169A46002E9A460075
S21444FA20399A460008B5FFF7CDFF012805D1FFF700
S21444FA309FFFBDE80840FDF7B9BFFFF7C3FF0128A5
S21444FA40F5D00020FFF79DFFFFF7BCFFF1E700BFAE
S21444FA5010F8012B11F8013B012A28BF9A42F7D02F
S21444FA60D01A7047034613F8012B002AFBD1181A04
S21444FA70013870470000000000000000000000004D
S21444FA8001F0FF01102A2BDB10F0070F08D010F806
S21444FA90013B013A8B422DD010F0070F42B3F6D10A
S21444FAA0F0B441EA012141EA014122F007047FF023
S21444FAB000070023F0E80256083C85EA010586EA7A
S21444FAC0010685FA47F5A3FA87F586FA47F6A5FAB6
S21444FAD087F68EB9EED1F0BC01F0FF0102F00702C2
S21444FAE032B110F8013B013A83EA010313B1F8D16D
S21444FAF00020704701387047002D06BF354603384E
S21444FB00073815F0010F07D1013015F4807F02BF86
S21444FB10013015F4C03F0130F0BC0138704700BFD7
S21444FB2081F0004102E000BF83F0004330B54FEA65
S21444FB3041044FEA430594EA050F08BF90EA020FD2
S21444FB401FBF54EA000C55EA020C7FEA645C7FEA65
S21444FB50655C00F0E2804FEA5454D4EB5555B8BF88
S21444FB606D420CDD2C4480EA020281EA030382EAF9
S21444FB70000083EA010180EA020281EA0303362D8B
S21444FB8088BF30BD11F0004F4FEA01314FF4801C5E
S21444FB904CEA113102D0404261EB410113F0004F70
S21444FBA04FEA03334CEA133302D0524263EB430327
S21444FBB094EA050F00F0A780A4F10104D5F1200EC5
S21444FBC00DDB02FA0EFC22FA05F2801841F1000120
S21444FBD003FA0EF2801843FA05F359410EE0A5F1F4
S21444FBE020050EF1200E012A03FA0EFC28BF4CF025
S21444FBF0020C43FA05F3C01851EBE37101F00045DB
S21444FC0007D54FF0000EDCF1000C7EEB00006EEBE7
S21444FC100101B1F5801F1BD3B1F5001F0CD3490871
S21444FC205FEA30004FEA3C0C04F101044FEA4452C8
S21444FC3012F5800F80F09A80BCF1004F08BF5FEA4F
S21444FC40500C50F1000041EB045141EA050130BD2F
S21444FC505FEA4C0C404141EB0101013C28BFB1F541
S21444FC60801FE9D291F0000F04BF01460020B1FA8C
S21444FC7081F308BF2033A3F10B03B3F120020CDA5F
S21444FC800C3208DD02F1140CC2F10C0201FA0CF03D
S21444FC9021FA02F10CE002F11402D8BFC2F1200CA2
S21444FCA001FA02F120FA0CFCDCBF41EA0C01904058
S21444FCB0E41AA2BF01EB0451294330BD6FEA0404A1
S21444FCC01F3C1CDA0C340EDC04F11404C4F120028C
S21444FCD020FA04F001FA02F340EA030021FA04F39E
S21444FCE045EA030130BDC4F10C04C4F1200220FAF5
S21444FCF002F001FA04F340EA0300294630BD21FA33
S21444FD0004F0294630BD94F0000F83F4801306BFF8
S21444FD1081F480110134013D4EE77FEA645C18BFEC
S21444FD207FEA655C29D094EA050F08BF90EA020F83
S21444FD3005D054EA000C04BF1946104630BD91EA7B
S21444FD40030F1EBF0021002030BD5FEA545C05D17E
S21444FD504000494128BF41F0004130BD14F58004BD
S21444FD603CBF01F5801130BD01F0004545F0FE4131
S21444FD7041F470014FF0000030BD7FEA645C1ABF66
S21444FD80194610467FEA655C1CBF0B46024650EA9D
S21444FD90013406BF52EA033591EA030F41F40021C9
S21444FDA030BD00BF90F0000F04BF0021704730B54F
S21444FDB04FF4806404F132044FF000054FF0000124
S21444FDC050E700BF90F0000F04BF0021704730B5E5
S21444FDD04FF4806404F1320410F0004548BF4042BA
S21444FDE04FF000013EE700BF42004FEAE2014FEA0F
S21444FDF031014FEA02701FBF12F07F4393F07F4FEA
S21444FE0081F06051704732F07F4208BF704793F0EC
S21444FE107F4F04BF41F40021704730B54FF46074FF
S21444FE2001F0004521F000411CE700BF50EA010202
S21444FE3008BF704730B54FF000050AE050EA0102AB
S21444FE4008BF704730B511F0004502D5404261EB1B
S21444FE5041014FF4806404F132045FEA915C3FF45C
S21444FE60D8AE4FF003025FEADC0C18BF03325FEAF9
S21444FE70DC0C18BF033202EBDC02C2F1200300FAAA
S21444FE8003FC20FA02F001FA03FE40EA0E0021FACF
S21444FE9002F11444BDE600BF70B54FF0FF0C4CF4BD
S21444FEA0E06C1CEA11541DBF1CEA135594EA0C0F6F
S21444FEB095EA0C0F00F0DEF82C4481EA030621EAAA
S21444FEC04C5123EA4C5350EA013518BF52EA0335E5
S21444FED041F4801143F4801338D0A0FB02CE4FF097
S21444FEE00005E1FB02E506F00042E0FB03E54FF0C7
S21444FEF00006E1FB03569CF0000F18BF4EF0010EBF
S21444FF00A4F1FF04B6F5007F64F5407404D25FEABA
S21444FF104E0E6D4146EB060642EAC62141EA55516D
S21444FF204FEAC52040EA5E504FEACE2EB4F1FD0CAF
S21444FF3088BFBCF5E06F1ED8BEF1004F08BF5FEA2D
S21444FF40500E50F1000041EB045170BD06F00046DF
S21444FF5046EA010140EA020081EA0301B4EB5C048C
S21444FF60C2BFD4EB0C0541EA045170BD41F4801184
S21444FF704FF0000E013C00F3AB8014F1360FDEBFA9
S21444FF80002001F0004170BDC4F10004203C35DA85
S21444FF900C341BDC04F11404C4F1200500FA05F308
S21444FFA020FA04F001FA05F240EA020001F00042A9
S21444FFB021F0004110EBD37021FA04F642EB06011F
S21444FFC05EEA430E08BF20EAD37070BDC4F10C0449
S21444FFD0C4F1200500FA04F320FA05F001FA04F20D
S21444FFE040EA020001F0004110EBD37041F10001F9
S21444FFF05EEA430E08BF20EAD37070BDC4F1200504
S21445000000FA05F24EEA020E20FA04F301FA05F26A
S21445001043EA020321FA04F001F0004121FA04F212
S21445002020EA020000EBD3705EEA430E08BF20EAE2
S214450030D37070BD94F0000F0FD101F0004640001C
S21445004041EB010111F4801F08BF013CF7D041EA9E
S214450050060195F0000F18BF704703F000465200A2
S21445006043EB030313F4801F08BF013DF7D043EA73
S2144500700603704794EA0C0F0CEA135518BF95EA29
S2144500800C0F0CD050EA410618BF52EA4306D1D1B0
S21445009081EA030101F000414FF0000070BD50EACF
S2144500A0410606BF1046194652EA430619D094EA59
S2144500B00C0F02D150EA013613D195EA0C0F05D143
S2144500C052EA03361CBF104619460AD181EA030197
S2144500D001F0004141F0FE4141F470014FF000004F
S2144500E070BD41F0FE4141F4780170BD70B54FF0EA
S2144500F0FF0C4CF4E06C1CEA11541DBF1CEA13556A
S21445010094EA0C0F95EA0C0F00F0A7F8A4EB05044B
S21445011081EA030E52EA03354FEA013100F0888042
S2144501204FEA03334FF0805545EA131343EA12630B
S2144501304FEA022245EA111545EA10654FEA0026C0
S2144501400EF000419D4208BF964244F1FD0404F579
S214450150407402D25B084FEA3202B61A65EB0305D5
S2144501605B084FEA32024FF480104FF4002CB6EB92
S214450170020E75EB030E22BFB61A754640EA0C0012
S2144501805B084FEA3202B6EB020E75EB030E22BF52
S214450190B61A754640EA5C005B084FEA3202B6EB93
S2144501A0020E75EB030E22BFB61A754640EA9C0052
S2144501B05B084FEA3202B6EB020E75EB030E22BF22
S2144501C0B61A754640EADC0055EA060E18D04FEAE0
S2144501D0051545EA16754FEA06164FEAC30343EA80
S2144501E052734FEAC2025FEA1C1CC0D111F4801F4D
S2144501F00BD141EA00014FF000004FF0004CB6E746
S21445020011F4801F04BF01430020B4F1FD0C88BFE4
S214450210BCF5E06F3FF6AFAEB5EB030C04BFB6EBEF
S214450220020C5FEA500C50F1000041EB045170BDE2
S2144502300EF0004E4EEA113114EB5C04C2BFD4EB0F
S2144502400C0541EA045170BD41F480114FF0000E93
S214450250013C90E645EA060E8DE60CEA135594EA0F
S2144502600C0F08BF95EA0C0F3FF43BAF94EA0C0F12
S2144502700AD150EA01347FF434AF95EA0C0F7FF487
S21445028025AF104619462CE795EA0C0F06D152EADB
S21445029003353FF4FDAE1046194622E750EA4106BF
S2144502A018BF52EA43067FF4C5AE50EA41047FF4D0
S2144502B00DAF52EA43057FF4EBAE12E74FF0FF3C35
S2144502C006E000BF4FF0010C02E000BF4FF0010C06
S2144502D04DF804CD4FEA410C7FEA6C5C4FEA430C7F
S2144502E018BF7FEA6C5C1BD001B050EA410C0CBFCE
S2144502F052EA430C91EA030F02BF90EA020F002030
S214450300704710F1000F91EA030F58BF994208BF96
S21445031090422CBFD8176FEAE37040F00100704753
S2144503204FEA410C7FEA6C5C02D150EA013C07D1AA
S2144503304FEA430C7FEA6C5CD6D152EA033CD3D0F5
S2144503405DF8040B704700BF8446104662468C46EF
S2144503501946634600E000BF01B5FFF7B7FF002822
S21445036048BF10F1000F01BD4DF808EDFFF7F4FF4B
S2144503700CBF012000205DF808FB00BF4DF808EDD6
S214450380FFF7EAFF34BF012000205DF808FB00BFF9
S2144503904DF808EDFFF7E0FF94BF012000205DF81B
S2144503A008FB00BF4DF808EDFFF7CEFF94BF0120D0
S2144503B000205DF808FB00BF4DF808EDFFF7C4FFC9
S2144503C034BF012000205DF808FB00BF4FEA410C12
S2144503D07FEA6C5C02D150EA013C0AD14FEA430CF5
S2144503E07FEA6C5C02D152EA033C02D14FF0000032
S2144503F070474FF0010070474FEA410212F5001270
S21445040015D211D56FF47873B3EB625212D94FEA11
S214450410C12343F0004343EA505311F0004F23FAFB
S21445042002F018BF404270474FF00000704750EA50
S214450430013005D111F0004008BF6FF0004070470D
S2144504404FF00000704700BF4A0011D212F5001267
S21445045011D20DD56FF47873B3EB62520ED44FEAD2
S214450460C12343F0004343EA505323FA02F0704752
S2144504704FF00000704750EA013002D14FF0FF3090
S21445048070474FF0000070474FEA4102B2F1E04333
S21445049024BFB3F5001CDCF1FE5C0DD901F0004C21
S2144504A04FEAC0024CEA5070B2F1004F40EB830071
S2144504B008BF20F00100704711F0804F21D113F19D
S2144504C03872BCBF01F00040704741F480114FEAD6
S2144504D05252C2F11802C2F1200C10FA0CF320FA5F
S2144504E002F018BF40F001004FEAC1234FEAD3237C
S2144504F003FA0CFC40EA0C0023FA02F34FEA4303E6
S214450500CCE77FEA625307D150EA01331EBF4FF06E
S214450510FE4040F44000704701F0004040F0FE4089
S21445052040F40000704700BF80F0004002E000BF86
S21445053081F0004142001FBF5FEA410392EA030F84
S2144505407FEA226C7FEA236C6AD04FEA1262D2EBCE
S2144505501363C1BFD218414048404140B8BF5B42D3
S214450560192B88BF704710F0004F40F4000020F06C
S2144505707F4018BF404211F0004F41F4000121F082
S2144505807F4118BF494292EA030F3FD0A2F10102CC
S21445059041FA03FC10EB0C00C3F1200301FA03F10A
S2144505A000F0004302D5494260EB4000B0F5000F2D
S2144505B013D3B0F1807F06D340084FEA310102F1EC
S2144505C00102FE2A51D2B1F1004F40EBC25008BF9E
S2144505D020F0010040EA03007047490040EB000068
S2144505E0013A28BFB0F5000FEDD2B0FA80FCACF169
S2144505F0080CB2EB0C0200FA0CF0AABF00EBC25096
S21445060052421843BCBFD0401843704792F0000F83
S21445061081F4000106BF80F400000132013BB5E7D6
S2144506204FEA41037FEA226C18BF7FEA236C21D04C
S21445063092EA030F04D092F0000F08BF08467047B1
S21445064090EA010F1CBF0020704712F07F4F04D17F
S214450650400028BF40F00040704712F100723CBF92
S21445066000F50000704700F0004343F0FE4040F4BC
S214450670000070477FEA226216BF08467FEA23637A
S2144506800146420206BF5FEA412390EA010F40F465
S214450690800070474FF0000304E000BF10F00043B1
S2144506A048BF40425FEA000C08BF704743F0964398
S2144506B001464FF000001CE050EA010208BF7047B3
S2144506C04FF000030AE000BF50EA010208BF70473A
S2144506D011F0004302D5404261EB41015FEA010C4F
S2144506E002BF84460146002043F0B64308BFA3F147
S2144506F08053A3F50003BCFA8CF2083AA3EBC25329
S21445070010DB01FA02FC634400FA02FCC2F1200247
S214450710BCF1004F20FA02F243EB020008BF20F07E
S2144507200100704702F1200201FA02FCC2F12002E4
S21445073050EA4C0021FA02F243EB020008BF20EAD9
S214450740DC7070474FF0FF0C1CEAD0521EBF1CEA07
S214450750D15392EA0C0F93EA0C0F6FD01A4480EAF5
S214450760010C400218BF5FEA41211ED04FF00063DE
S21445077043EA501043EA5111A0FB01310CF000400A
S214450780B1F5000F3EBF490041EAD3715B0040EA30
S214450790010062F17F02FD2A1DD8B3F1004F40EB00
S2144507A0C25008BF20F00100704790F0000F0CF0D3
S2144507B0004C08BF49024CEA502040EA51207F3A97
S2144507C0C2BFD2F1FF0340EAC250704740F4000072
S2144507D04FF00003013A5DDC12F1190FDCBF00F063
S2144507E000407047C2F10002410021FA02F1C2F111
S2144507F0200200FA02FC5FEA310040F1000053EAAD
S2144508004C0308BF20EADC70704792F0000F00F0FA
S214450810004C02BF400010F4000F013AF9D040EA00
S2144508200C0093F0000F01F0004C02BF490011F494
S214450830000F013BF9D041EA0C018FE70CEAD15392
S21445084092EA0C0F18BF93EA0C0F0AD030F0004C12
S21445085018BF31F0004CD8D180EA010000F00040C6
S214450860704790F0000F17BF90F0004F084691F084
S214450870000F91F0004F14D092EA0C0F01D14202BE
S2144508800FD193EA0C0F03D14B0218BF084608D187
S21445089080EA010000F0004040F0FE4040F40000D1
S2144508A0704740F0FE4040F4400070474FF0FF0C64
S2144508B01CEAD0521EBF1CEAD15392EA0C0F93EAAB
S2144508C00C0F69D0A2EB030280EA010C49024FEAFD
S2144508D0402037D04FF0805343EA111143EA1013B6
S2144508E00CF000408B4238BF5B0042F17D024FF46E
S2144508F0000C8B4224BF5B1A40EA0C00B3EB510F49
S21445090024BFA3EB510340EA5C00B3EB910F24BF31
S214450910A3EB910340EA9C00B3EBD10F24BFA3EBB6
S214450920D10340EADC001B0118BF5FEA1C1CE0D17E
S214450930FD2A3FF650AF8B4240EBC25008BF20F031
S214450940010070470CF0004C4CEA50207F32C2BF85
S214450950D2F1FF0340EAC250704740F400004FF022
S2144509600003013A37E792F0000F00F0004C02BF53
S214450970400010F4000F013AF9D040EA0C0093F01D
S214450980000F01F0004C02BF490011F4000F013B77
S214450990F9D041EA0C0195E70CEAD15392EA0C0FDF
S2144509A008D142027FF47DAF93EA0C0F7FF470AF17
S2144509B0084676E793EA0C0F04D14B023FF44CAF5A
S2144509C008466EE730F0004C18BF31F0004CCAD1EF
S2144509D030F000427FF45CAF31F000437FF43CAF2B
S2144509E05FE700BF4FF0FF3C06E000BF4FF0010C4D
S2144509F002E000BF4FF0010C4DF804CD4FEA40022F
S214450A004FEA41037FEA226C18BF7FEA236C11D078
S214450A1001B052EA530C18BF90EA010F58BFB2EB2B
S214450A20030088BFC81738BF6FEAE17018BF40F0AB
S214450A30010070477FEA226C02D15FEA402C05D15F
S214450A407FEA236CE4D15FEA412CE1D05DF8040BE4
S214450A50704700BF844608466146FFE70FB5FFF777
S214450A60C9FF002848BF10F1000F0FBD4DF808ED2F
S214450A70FFF7F4FF0CBF012000205DF808FB00BF20
S214450A804DF808EDFFF7EAFF34BF012000205DF87A
S214450A9008FB00BF4DF808EDFFF7E0FF94BF0120C7
S214450AA000205DF808FB00BF4DF808EDFFF7D2FFC4
S214450AB094BF012000205DF808FB00BF4DF808ED07
S214450AC0FFF7C8FF34BF012000205DF808FB00BFD4
S214450AD042000ED2B2F1FE4F0BD34FF09E03B3EB5E
S214450AE0126209D44FEA002343F0004323FA02F08A
S214450AF070474FF00000704712F1610F01D1420276
S214450B0002D14FF0FF3070474FF00000704700BFEE
S214450B1053B94AB9002908BF00281CBF4FF0FF311A
S214450B204FF0FF3000F0A6B9ADF1080C6DE904CEE4
S214450B3000F03EF8DDF804E0DDE9022304B0704736
S214450B4038B505460C462846214600220023FFF7C1
S214450B5015FC28B928462146BDE8384000F00AB8B5
S214450B60284604F1004100F005F8404261EB41019A
S214450B7038BD00BFD0B50C4B002206460F46FFF7E2
S214450B808BF9FFF761FC0446FFF70CF9074B00228B
S214450B90FFF782F902460B4630463946FEF7C4FF54
S214450BA0FFF752FC2146D0BD0000F03D0000F04165
S214450BB02DE9F047089D0E4604468C46002B40F02E
S214450BC081808A42174645D9B2FA82F24AB1C2F1C5
S214450BD0200106FA02F320FA01F1974041EA030C98
S214450BE094404FEA174E230CBCFBFEF6B9B20EFBFB
S214450BF016CC43EA0C4306FB01F0984209D9FB188C
S214450C0006F1FF3C80F01581984240F21281023E83
S214450C103B441B1AA4B2B3FBFEF00EFB103344EA6A
S214450C20034400FB01F1A14209D93C1900F1FF3309
S214450C3080F00181A14240F2FE8002383C44641AAD
S214450C4040EA064000211DB1D4400023C5E90043D3
S214450C50BDE8F08702B9FFDEB2FA82F2002A4FD12C
S214450C60CB1B4FEA174E1FFA87F80121B3FBFEFC54
S214450C70260C0EFB1C3346EA034608FB0CF3B34230
S214450C8007D9BE190CF1FF3002D2B34200F2EB8011
S214450C908446F61AA3B2B6FBFEF00EFB106643EA90
S214450CA0064408FB00F8A04507D93C1900F1FF3378
S214450CB002D2A04500F2D2801846A4EB080440EACA
S214450CC00C40C0E78B4208D9002D00F0AF800021CC
S214450CD0C5E900060846BDE8F087B3FA83F1002962
S214450CE049D1B34202D3824200F2BB80841A66EBF6
S214450CF0030301209C46002DAAD0C5E9004CA7E772
S214450D00C2F120039740D8409140DE404FEA174E47
S214450D1008434FEA104CB6FBFEF11FFA87F80EFB68
S214450D2011664CEA064601FB08F3B34204FA02F4A0
S214450D3009D9BE1901F1FF3C80F08E80B34240F2DE
S214450D408B8002393E44F31A86B2B3FBFEF00EFBA7
S214450D50103346EA034600FB08F3B34207D9BE19EB
S214450D6000F1FF3C74D2B34272D902383E44F31ABE
S214450D7040EA01417AE7C1F1200703FA01F422FA75
S214450D8007F31C4320FA07F906FA01F34FEA144C19
S214450D90FE4049EA03094FEA1943B6FBFCFE1FFA33
S214450DA084F80CFB1E6643EA06460EFB08FAB24577
S214450DB002FA01F200FA01F308D9A6190EF1FF303E
S214450DC048D2B24546D9AEF1020E2644A6EB0A06EF
S214450DD01FFA89F9B6FBFCF00CFB106649EA064695
S214450DE000FB08F8B04507D9A61900F1FF3C2DD2FF
S214450DF0B0452BD90238264440EA0E40A6EB0806F5
S214450E00A0FB02894E45C446CE4618D315D075B3C9
S214450E10B3EB0C0266EB0E0606FA07F722FA01F369
S214450E20CE401F43C5E90076002111E729462846EE
S214450E300EE76646EDE6184601E74345E7D2B8EBCA
S214450E40020C69EB04040138A646E0E76046D3E7A2
S214450E5060468CE78646B9E7614674E702383C4407
S214450E602BE7084647E7ACF1020C3E4411E7294616
S214450E70EEE600BF704700BF2DE9F04788B0002B6F
S214450E801F461446B8BF03F10043129A109DDDF87D
S214450E904CA0B6BF1F4600232D231370149B23F08A
S214450EA02008B8F1460F05D0B8F1450F00D10135F9
S214450EB0022300E0032307AA049206AACDE902A26C
S214450EC0CDE9003522463B4601F0A6FDB8F1470F71
S214450ED0064602D1119BDB0722D5B8F1460F06EB35
S214450EE0050910D13378302B0AD10022002320463D
S214450EF03946FFF739FA18B9C5F10105CAF8005061
S214450F00DAF8003099440022002320463946FFF798
S214450F102BFA08B1CDF81C903022079B4B4507D3DA
S214450F20079B159A9B1B3046136008B0BDE8F087B3
S214450F30591C07911A70F0E7F7B503460029B8BF64
S214450F40494203F8022BB4BF2D222B2209294270B1
S214450F502ADD0DF10704A4460A27A6460A4691FB54
S214450F60F7F607FB16153035632A04F1FF340EF8FD
S214450F70015C3146F1DC3031AEF1020504F8011C66
S214450F80441C294661450AD30DF10902A2EB0E021F
S214450F90654588BF00221344181A03B0F0BD11F802
S214450FA0012B04F8012FEDE7302330318370C170F3
S214450FB0031DF1E72DE9F04F91B00C46DDF868804A
S214450FC016461F46054602F04DFE03680993184629
S214450FD0FEF748FD00230E93D8F800300A900733F5
S214450FE023F0070303F1080294F81890D4F800B0EC
S214450FF0C8F80020D3E90023C4E91223D4E9128AAD
S2144510002AF000430B930B999C4B4FF0FF3240461A
S214451010FFF7DCF970BB994B0B994FF0FF32404612
S214451020FFF7B6F930BB0022002340465146FFF78E
S214451030A5F910B12D2384F84330914B9148B9F169
S214451040470F94BF98468046032323612BF004033D
S21445105023604FF0000A009733460FAA21462846DC
S21445106000F0D2F9013040F08F804FF0FF3011B0DC
S214451070BDE8F08F4246534640465146FFF7A6F92F
S21445108040B1BAF1000FBCBF2D2384F843307E48EB
S2144510907E4BD4E763685A1C09F0DF0142D106232C
S2144510A06360002206920EAACDE904920DAA4BF47F
S2144510B0806303920DF13302CDE901322360636804
S2144510C000934246534628460B91FFF7D5FE0B99AB
S2144510D0472980460D9908D1C81C02DB63689942AA
S2144510E040DDA9F102095FFA89F9B9F1650F1FD804
S2144510F001394A4604F150000D91FFF71DFF0E9A3F
S2144511001318012A8246236102DC2268D20701D5DC
S214451110013323619DF83330002B9CD02D2384F872
S214451120433098E74729BCD1002BBAD10123B7E70E
S214451130B9F1660F18D1002963680BDD216113B933
S2144511402268D00702D501330B442361A1654FF0D1
S214451150000ADFE713B92268D20701D50233F4E760
S2144511600123F2E74FF067090E9B994205DB23689A
S2144511702161D807EAD54B1CE7E70029D4BFC1F162
S214451180020201221344E0E723685A0507D423697F
S214451190424631462846B84701302BD165E7B9F176
S2144511A0650F40F2DC80D4E9120100220023FFF7E8
S2144511B0DBF8002833D0364A012331462846B8475F
S2144511C001303FF452AFDDE90D239A4202DB236836
S2144511D0D8070FD5DDE9092331462846B8470130FB
S2144511E03FF443AF4FF0000804F11A090E9B013B4C
S2144511F0434509DC23689B0700F10181E0680F9BA6
S2144512009842B8BF184632E701234A463146284633
S214451210B84701303FF429AF08F10108E6E70D9BD2
S214451220002B37DC1A4A012331462846B847013099
S2144512303FF41BAFDDE90D23134302D12368D907DD
S214451240D8D5DDE9092331462846B84701303FF46D
S2144512500CAF4FF0000904F11A0A0D9B5B424B4553
S21445126001DC0E9B94E70123524631462846B84793
S21445127001303FF4FAAE09F10109EEE7FFFFEF7FD3
S214451280469A46004A9A4600529A46004E9A460064
S214451290569A46000E9AA36D9A42A8BF1A46002A49
S2144512A0914637DC4FF0000B29EAE97904F11A023A
S2144512B0D4F858A0AAEB09035B4533DCDDE90D23DA
S2144512C09A423BDB2368DA0738D40E9A0D99A2EB8F
S2144512D00A03A2EB01099945A8BF9946B9F1000F43
S2144512E034DC4FF0000829EAE97904F11A0ADDE909
S2144512F00D239B1AA3EB090343457FF77BAF0123D9
S214451300524631462846B84701303FF4AEAE08F15E
S2144513100108ECE71346314642462846B8470130B1
S214451320C0D1A2E60123314628460B92B847013084
S2144513303FF49BAE0B9A0BF1010BB9E7DDE90923A8
S21445134031462846B8470130BFD18EE64B4608EBB6
S2144513500A0231462846B8470130C2D185E60E9A7C
S214451360012A01DCDB0737D50123424631462846AC
S214451370B84701303FF479AEDDE9092331462846C2
S214451380B84701303FF471AED4E91201002200237C
S214451390FEF7EAFFD8B90E9B08F10102013B31463C
S2144513A02846B84701300ED15FE601234A46314606
S2144513B02846B84701303FF458AE08F101080E9B61
S2144513C0013B4345F1DC534604F15002E1E64FF05C
S2144513D0000804F11A09F2E701234246DFE7012334
S2144513E04A4631462846B84701303FF43EAE08F1F6
S2144513F00108E3680F995B1A4345F0DCFEE64FF0BB
S214451400000804F11909F4E72DE9F0471646994610
S2144514108A680B69DDF820809342B8BF134633606F
S21445142091F8432007460C460AB1013333602368DA
S214451430990642BF336802333360256815F00605C2
S21445144006D104F1190AE36832689B1AAB4226DCDA
S21445145094F84320131E226818BF012392062BD406
S21445146004F1430249463846C04701301ED023683A
S214451470E568326803F00603042B08BFAD1AA36877
S21445148022690CBF25EAE57500259342C4BF9B1A21
S214451490ED1800261A34B5421AD1002008E001237B
S2144514A0524649463846C047013003D14FF0FF30D3
S2144514B0BDE8F0870135C6E7E1185A1C302081F8AB
S2144514C04300224494F8451082F843100233C7E798
S2144514D00123224649463846C0470130E6D0013604
S2144514E0D9E700002DE9FF470C469146277E0C9923
S2144514F0782F80469A4604F1430207D8622F0AD8C9
S214451500002F00F0D880582F00F0A38004F1420643
S21445151084F842703AE0A7F16303152BF6D801A08C
S21445152050F823F07D154500911545000D154500ED
S2144515300D1545000D1545000D1545009115450041
S2144515400D1545000D1545000D1545000D154500B5
S2144515509D164500C11545007F1645000D154500ED
S2144515600D154500BF1645000D154500C11545002E
S2144515700D1545000D154500871645000B681A1DC7
S2144515801B680A6004F1420684F842300123A3E052
S214451590256808682E0600F104030AD505680B6021
S2144515A0002D03DA2D236D4284F843305E480A2326
S2144515B019E015F0400F05680B6018BF2DB2EFE730
S2144515C00B682568181D0860280601D51D6802E0C9
S2144515D06906FBD51D8854486F2F0CBF08230A2380
S2144515E0002184F843106668A660002EA2BF2168D5
S2144515F021F0040121600DB9002E4DD01646B5FBED
S214451600F3F103FB1157C75D06F8017D2F46BB4234
S2144516100D46F4D9082B0BD12368DF0708D5236977
S21445162061689942DEBF302306F8013C06F1FF3675
S214451630921B2261CDF800A04B4603AA21464046A0
S214451640FFF7E2FE01304CD14FF0FF3004B0BDE865
S214451650F087354884F8457023680E681F0656F8A7
S214451660045B0E6014D5D90744BF43F020032360BE
S2144516701DB9236823F0200323601023B0E72368B1
S21445168043F0200323607823284884F84530E3E771
S2144516905E0648BFADB2E6E71646BBE70B6826686A
S2144516A060691D1D0D6035061B6801D5186002E092
S2144516B07106FBD51880002323611646BAE70B68EA
S2144516C01A1D0A601E68626800213046FEF7D8F982
S2144516D008B1801B606063682361002384F843304B
S2144516E0A8E72369324649464046D0470130ABD045
S2144516F023689B0713D4E068039B9842B8BF1846F7
S214451700A4E70123324649464046D04701309BD0A0
S2144517100135E36803995B1AAB42F2DCEBE700253B
S21445172004F11906F5E700BF589A4600699A46003F
S2144517302DE9F04F87B0174603938B685A1EB2F5CE
S214451740AE7F83BF6FF4AE755B190293002386BFE9
S21445175040F25D138B6002930B688B46002543F47D
S214451760F0634BF81C3BCDE9045580460C465E4677
S214451770AA46A9460195A26852B13B681B784E2BEE
S21445178064D8402B3CD8A3F12B01C8B20E283AD9D1
S214451790B9F1000F03D0236823F4807323600AF160
S2144517A0FF3ABAF1010F00F213815E4500F205815A
S2144517B00125284607B0BDE8F08FA3F161020D2A42
S2144517C0E6D801A151F822F00719450091174500C2
S2144517D09117450091174500671945003F19450083
S2144517E09117450091174500151945009117450075
S2144517F0911745009117450091174500CD184500AE
S214451800A3F14102DBE70E29C2D801A050F821F02A
S214451810BF18450091174500BF18450053194500A8
S214451820911745006D184500A9184500A9184500AB
S214451830A9184500A9184500A9184500A918450046
S214451840A9184500A9184500A91845006E2B09D8C2
S214451850602BB2D8542B77D0592B99D1072D97D1D9
S214451860082529E0742B6FD0792BF6E72168C80543
S2144518701AD5029B21F08001216009F101091BB1AF
S214451880013B01320293A260A368013BA360236932
S214451890013323617B68013B002B7B6040F38480EA
S2144518A03B6801333B6066E71AEB050F7FF470AF84
S2144518B0226822F4C072226006F8013BE4E72268FB
S2144518C010067FF565AF22F08002F4E7BAF1000F07
S2144518D00ED1B9F1000F0ED1226802F4E061B1F5E0
S2144518E0E06F08D122F4F06222604FF0010AE3E788
S2144518F0BAF1020F55D0012D02D0042D7FF448AF22
S2144519000135EDB2D8E7BAF1010F7FF441AF4FF09C
S214451910020AD1E77DB9B9F1000F7FF43CAF2268E2
S21445192002F4E061B1F5E06F7FF439AF22F4F0627E
S21445193022600125C0E7032DE2D0052DDEE7022D06
S2144519407FF426AF0325B7E7062D7FF421AF07259D
S214451950B2E7226891057FF51BAF22F4207222601C
S214451960CDF80490A8E7226802F4A061B1F5806F2F
S21445197006D050057FF50CAFB9F1000F3FF40FAF19
S214451980910558BF019922F4F06258BFA9EB0101B1
S21445199042F4C07258BFCDE9041622604FF00009E4
S2144519A08AE74FF0030A87E7D4F880313946404640
S2144519B0984700283FF4DFAEEAE6D4F87C3116F8BF
S2144519C0011D3A46404698472369013B2361ECE6AC
S2144519D06B1E062B25D8022D36D85E457FF6E8AE1B
S2144519E0D4F87C3116F8011D3A4640469847236997
S2144519F0013B2361F1E70298D4F87C3110F8011DCC
S214451A0002903A46404698472369013B23610AF1CE
S214451A10FF3A5FFA8AFABAF1020FECD1033DEDB20E
S214451A20761B2368DA052FD55B0510D55E457FF610
S214451A30BFAED4F87C3116F8011D3A464046984765
S214451A402369013B2361F1E7AA460296DFE716F8CC
S214451A50011C2369652903F1FF3306F1FF35236130
S214451A600CD045290AD0D4F87C313A4640469847AA
S214451A70236916F8021C013BB51E2361D4F87C3158
S214451A803A46404698472E46256815F0100559D1E2
S214451A903570236803F4C063B3F5806F1CD1019B92
S214451AA04B45A3EB090224D100225946404600F097
S214451AB083FED4F800C0039B1CF0020F1B68064645
S214451AC00F4621D003991A1D0A601B68C3E90067B3
S214451AD0E3680133E3606CE6049B002BE4D005998C
S214451AE00A232A460131404600F0E6FE049B059E41
S214451AF0C21A04F26F139E4228BF04F5B776124900
S214451B00304600F029F8CFE71CF0040F03F1040E29
S214451B1003D00399C1F800E0D7E7039AC2F800E07E
S214451B20D3F8008002460B46FEF750FC28B107481E
S214451B3000F00EF8C8F80000CAE730463946FEF70A
S214451B40A3FCF7E7002534E67A9A460064954600F6
S214451B50004870470000C07F0EB400B59AB01BAB76
S214451B60019005906FF00041094806910391094997
S214451B7053F8042B04910068009301A902F0E4FD94
S214451B80019B00221A701AB05DF804EB03B070474B
S214451B90182340200802FFFF2DE9F0410F469046E6
S214451BA002F084FB04460D46B8F1000F11D0C7F38A
S214451BB00A53C3F16B03002B0BDD1B0503F17F5561
S214451BC0002405F5401522462B46FEF765F90446E2
S214451BD00D4620462946BDE8F0810000000000007D
S214451BE02DE9F04FA1B09B4600231C939E4B1792C0
S214451BF01F68824638460E46FDF734FF4FF000080C
S214451C0004464FF000091B961B9B1A782B2A4CD08E
S214451C103AD80D2A33D8082A33D8002A3DD000238F
S214451C200C931B9D2B78302B40F0A9806B7803F0E6
S214451C30DF03582B66D10C9B01931CAB00938B4A54
S214451C40CDF808B01DAB1BA9504601F01FFD10F09E
S214451C500706044605D0062E29D1013500231B95D7
S214451C600C93179B002B40F08E850C9BD3B14246B8
S214451C7009F100431046194621B0BDE8F08F202AE9
S214451C80CDD101331B93BFE72D2AC8D101220C9233
S214451C905A1C1B925B78002BC3D1179B1B96002BB7
S214451CA040F06F8542464B46E4E70022EFE71C9A34
S214451CB03AB135211EA802F0F0FB1C99504602F0B9
S214451CC031F8013E042E06D8DFE806F00A0314175D
S214451CD00A00DDE91E892107C3D549F00049C0E75A
S214451CE0DDE91E831D9A23F4801302F2334243EA4C
S214451CF00259F0E7DFF87891EDE76FF000494FF0CD
S214451D00FF38E8E71B9B5A1C1B925B78302BF9D0B3
S214451D10002BA6D0012307931B9B08930023CDE9F0
S214451D2005339B460A221B980578A5F13003D9B2A0
S214451D30092926D92246394602F01CFE002832D00B
S214451D4000202B465C4604900246652B01D0452B69
S214451D5013D11CB9079B03439FD000241B9E731CBD
S214451D601B9373782B2B78D02D2B7BD00027A3F194
S214451D703001092940F282801B9600259EE000230B
S214451D80C9E7BBF1080FD5BF0699059902FB013394
S214451D9002FB013300F10100D4BF069305930BF116
S214451DA0010B1B90BFE71B9B1A191B921B5DBBF1D2
S214451DB0000F36D004905C46A3F13002092A12D9AA
S214451DC00122C2E71B9B5A1C1B925B780130302BC5
S214451DD0F8D0A3F13102082A00F2DA841B9A04905F
S214451DE0002008920446303B00F1010213D00499C6
S214451DF011440491224605190A21954213D1221809
S214451E00082A04F1010404441BDC06990A2202FB55
S214451E100133069300221B9B591C1B915B78104689
S214451E20CAE75846D3E7082A04DC069F4F43069779
S214451E300132E2E7571C102FDEBF059F4F4305973B
S214451E40F6E7102CDFBF05990A2202FB01330593FE
S214451E50E0E70023049301227CE70027B31C1B938D
S214451E60B37884E70127F9E7E09B4600809A460069
S214451E700000F07F1B9B591C1B915B78302BF9D0DB
S214451E80A3F1310108293FF678AFA3F1300C1B9B2F
S214451E9009934FF00A0E1B9B591C1B915B78A3F1C7
S214451EA03005092D35D9099D491B082944F61F6576
S214451EB002DC6545A8BF654607B16D42002C4CD18E
S214451EC0079901437FF4CDAE002A7FF4E6AE692B31
S214451ED026D023DC492B23D04E2B7FF4DEAE9C49FF
S214451EE01BA801F00FFE00283FF4D7AE1B9B1B78BE
S214451EF0282B2CD197491EAA1BA801F017FE0528AA
S214451F0025D11F9BDDF8788043F0FF4949F4E00969
S214451F10A7E60EFB0C3CACF1300CBCE76E2BDCE7C1
S214451F208D491BA801F0EEFD00283FF4B6AE1B9B7D
S214451F308A49013B1BA81B9301F0E4FD10B91B9B86
S214451F4001331B93DFF824924FF0000889E6844856
S214451F5002F00AFD8046894683E6049B0698EB1AFE
S214451F60BBF1000F08BFA346102C07932646A8BF13
S214451F701026FDF717FF092C8046894613DD794B59
S214451F8003EBC60353E91223FDF786FF8046059803
S214451F908946FDF707FF02460B4640464946FDF78C
S214451FA0C5FD804689460F2C36DC079B002B3FF443
S214451FB058AE22DD162B09DC6A4C04EBC304D4E983
S214451FC0000142464B46FDF767FFC3E7079AC4F153
S214451FD02503934220DB634DC4F10F0405EBC40192
S214451FE042464B46D1E90001FDF756FF079B1C1BB1
S214451FF005EBC405D5E90023E5E7079B16330BDB60
S214452000049B584A5D1B02EBC505D5E900234046AF
S2144520104946FEF76BF89DE7079BA61B1E44002E18
S21445202071DD16F00F030AD04E4901EBC301424657
S2144520304B46D1E90001FDF72FFF8046894636F02D
S2144520400F0650D0B6F59A7F27DD4FF0000BCDF83A
S21445205010B0CDF820B0CDF818B02223DFF80C919B
S214452060CAF800304FF00008089B002B3FF4F9AD46
S2144520701C99504601F056FE0699504601F052FE10
S2144520800499504601F04EFE0899504601F04AFE26
S2144520905946504601F046FEE3E5002336114046D4
S2144520A049461F46012E21DC0BB1804689462E4BFC
S2144520B0A9F1547903EBC70742464B46D7E90001D9
S2144520C0FDF7EAFE294B0A460B4029498B428046D6
S2144520D0BBD8A1F580118B4286BFDFF898904FF0AC
S2144520E0FF3802F15479002305937EE0F20707D5C1
S2144520F01D4B03EBC703D3E90023FDF7CDFE0123B4
S21445210001377610CEE7EED0764216F00F020AD0AB
S214452110144B03EBC20340464946D3E90023FDF77B
S214452120E5FF804689463611DDD01F2E24DD4FF06B
S214452130000BCDF810B0CDF820B0CDF818B022235E
S2144521404FF000084FF00009CAF800308CE700BF92
S214452150539A4600949A46004B9A4600D49B4600AE
S21445216064954600209C4600F89B46000000F07F9C
S2144521700000A07CFFFFEF7F16F0100318BF6A2310
S214452180B34F0593404649460023F20704D5D7E9A1
S2144521900023FDF781FE0123761007F10807F4D1E9
S2144521A00BB180468946059BBBB1C9F30A53C3F1BB
S2144521B06B03002B494610DD1F2B40F32881342B3B
S2144521C0DEBF203B4FF0FF3202FA03F34FF0000824
S2144521D0CCBF4FF05C7903EA010900220023404654
S2144521E04946FEF7C1F80028A1D1069B00930899F9
S2144521F023465A46504601F0EAFD089000283FF42B
S21445220024AF049B5D1B079B002BB4BF2B460023C6
S2144522100E93079B4FF0000B23EAE3731693CDF816
S21445222010B0089B5046596801F048FD06900028B6
S2144522303FF413AF089B1A69023203F10C01920072
S2144522400C3001F02DFD1EAB01931DAB00934246AD
S2144522504B465046CDE90A8902F0A2F81C90002864
S2144522603FF4FBAE0121504601F03DFE0490034687
S21445227000283FF4F2AE1D9D1E9A002DABBF0E9B67
S214452280169B169C0E9EACBFEE185C1B059BED1A66
S2144522901544704B013D9D42C2F1360280F2C9801D
S2144522A05B1B1F2BA2EB03024FF0010700F3B68022
S2144522B007FA03F30F930025B718059BBE4214444F
S2144522C01C443346A8BF3B46A342A8BF2346002B23
S2144522D0C2BFFF1AE41AF61A0E9B002B17DD0499A7
S2144522E01A46504601F0A4FE049000283FF4B5AEC9
S2144522F001461C9A504601F0FFFD099000283FF420
S214452300ACAE1C99504601F00DFD099B1C93002F61
S21445231000F39380079B002B08DD169A06995046D6
S21445232001F086FE069000283FF497AE002C08DDA7
S21445233006992246504601F0C9FE069000283FF40D
S2144523408CAE002E08DD04993246504601F0BEFE9E
S214452350049000283FF481AE069A1C99504601F039
S2144523602FFF834600283FF478AE0024C3680499BF
S214452370C4600D9301F009FFA04271DA0D9B53EA44
S214452380080340F09780C9F31303002B40F0928072
S21445239029F000431B0D1B05B3F1D66F40F28A802A
S2144523A0DBF8143023B9DBF81030012B40F382807C
S2144523B059460122504601F089FE0499834601F0AC
S2144523C0E4FE002876DD0599234A4B46002900F0B1
S2144523D0928002EA0901B1F1D66F00F38C80B1F123
S2144523E05C7F7FF7ACAE1D4A0023CDE914324046EC
S2144523F0DDE914234946FDF74FFD0B46034308BF69
S21445240022238046894608BFCAF8003030E64FF09A
S214452410FF3202FA03F303EA0808DEE6C5F17F4514
S21445242005F57F0505F57B45E23507FA05F50F9772
S21445243042E7012300250F933EE71C993A4650464E
S21445244001F044FE1C9000287FF464AF05E600BF0B
S214452450A89A460002FCFFFF0000F07F00005039B6
S214452460CDF8249066D10D9AC9F313035AB39C4A06
S21445247093422CD1059B404603B39A4A4B461A4095
S214452480B2F1D46F4FF0FF311BD8120DC2F16B037A
S21445249001FA03F398421AD1934B099A9A4202D10C
S2144524A001303FF4DAAD8F4B099A1A4002F5801990
S2144524B04FF00008059B002B95D1D9E54FF0FF332B
S2144524C0E8E70B46E6E753EA08033FF47CAFE5B199
S2144524D0099B1D42EED00D9B059A40464946C3B121
S2144524E0FFF75AFB02460B46DDE90A01FDF71EFBE0
S2144524F080468946DEE71340A3F580136FEA1359F5
S2144525006FEA09594FF0FF38D4E70F9B13EA080FD7
S214452510E0E7FFF741FB02460B46DDE90A01FDF71A
S21445252003FB0022002380468946FDF71DFF002851
S214452530C0D004E60499584601F081FF00224FF0CA
S214452540804306460F46FDF723FF002875D00D9BB2
S214452550002B47D0654F0026644D099B23F000436A
S2144525601B0D1B050F930F9A614B9A4240F0C8808E
S214452570DDE90A23CDE91423099BA3F154794046A6
S214452580494601F093FE02460B4630463946FDF76E
S21445259083FC42464B46FDF7C9FA0B465149554A18
S2144525A01940914280465ED90B9B02F15472934284
S2144525B003D10A9B01333FF450ADDFF82C914FF021
S2144525C0FF381C99504601F0ADFB0699504601F080
S2144525D0A9FB0499504601F0A5FB5946504601F023
S2144525E0A1FB1EE6B8F1000F19D1099BC3F31303EF
S2144525F0E3B93E4B002230463946FDF7BFFEC8B923
S2144526003D4B002230463946FDF746FC04460D460E
S21445261005F1004318941993DDE918679DE7B8F16D
S214452620010F03D1099B002B3FF489AD334F00269C
S214452630002491E70D9C304DEAE72F4B00223046AB
S2144526403946FDF729FC0D9B04460D4633B901F185
S214452650004310901193DDE910677EE702460B466E
S214452660CDE91023F7E703F15479059B002BA8D154
S21445267029F000430F9A1B0D1B059A42A1D120460F
S2144526802946FEF75DFAFDF7D9FB02460B4620467E
S2144526902946FDF749FA0D9AC9F3130343EA080399
S2144526A0134304460D4666D009A3D3E90023FDF738
S2144526B065FE00287FF4DCAC07A3D3E9002320465B
S2144526C02946FDF779FE00283FF47BAFD0E400BFEE
S2144526D09535A094FFFFDF3F35E5AF350000E03F79
S2144526E0FFFF0F000000F07FFFFFEF7F0000F03F89
S2144526F00000E07FFFFF9F7C0000E03F0000F0BF4A
S214452700059B13B30F9BB3F1D46F1ED826A3D3E90D
S214452710002320462946FDF73BFE90B12946204634
S214452720FDF792FE012838BF0120FDF73BFB0D9BC8
S21445273004460D46D3B901F1004312901393DDE9E3
S21445274012670F9A07F1D6639F1ADDE90A0101F071
S214452750ADFD02460B4630463946FDF79DFBDDE9A5
S2144527600A23FDF7E3F9804689467EE702460B468F
S214452770CDE91223E3E70EA3D3E90023FDF7FEFDDB
S214452780A1E700230C93179A1B9B1360FFF76DBABE
S214452790652B3FF45EAB452B3FF45BAB0122FFF761
S2144527A08FBB00BFAFF300800000C0FFFFFFDF41D7
S2144527B09535A094FFFFCF3F014BFFF711BA00BFF9
S2144527C0802340202DE9F0473A4E86468C466046A3
S2144527D01CF8014BA55D15F00805F8D12D2C33D115
S2144527E09CF800404FF0010800F1020C002B5CD02D
S2144527F0102B0CD1302C0AD19CF8000000F0DF00DD
S21445280058284DD19CF8014010230CF1020C08F1D4
S2144528100047013F0026B7FBF3F9304603FB197A1C
S214452820A4F13005092D18D82C46A34224DD751C85
S21445283007D081451DD301D1A2451ADB00FB0340D5
S21445284001261CF8014BEBE72B2C08BF9CF80040F3
S214452850A84608BF00F1020CC8E7A4F14105192DAA
